:020000040800F2
:1000000000200010F5D402088DC30108A14A0008A1
:1000100089C3010885C3010881C3010800000000ED
:100020000000000000000000000000007DC3010887
:1000300079C301080000000075C301085D110008C4
:100040005DD502085DD502085DD502085DD50208C0
:100050005DD502085DD502086924000895250008D1
:10006000592500081D250008E12400083139000841
:10007000213900081139000801390008F138000859
:10008000DD380008C93800085DD502085DD50208D2
:1000900091C601085DD502085DD50208A5240008B7
:1000A000CD500008FD500008BD5000080D5100085B
:1000B000ED500008DD5000085DD502085DD502084E
:1000C0005DD502085DD502085DD502085DD5020840
:1000D0005DD50208891200080D1200089111000870
:1000E0002D2400085DD5020865C301085DD502080E
:1000F0005DD502085DD502085DD502085DD5020810
:100100000000000000000000000000005DD50208B3
:100110005DD502085DD5020861A3020845A3020867
:10012000B5380008A13800088D3800087938000873
:10013000653800085DD502080000000000000000DE
:100140005DD502085DD502085DD5020800000000FB
:10015000000000000000000000000000000000009F
:1001600000000000000000005DD502085DD5020817
:100170005DD5020800000000000000000000000043
:08018000000000005DD502083B
:1001880070B4EFF31186502383F31288436B1A6817
:10019800D20720D45D686DB9446A826A944217D048
:1001A80081691144D9600ED9A21A5A60846200226A
:1001B80080F850201A6842F00102F1B21A6081F307
:1001C800118870BC704701698A1A5A608562EEE727
:1001D800012380F85030F1B281F3118870BC704768
:1001E800436A8269D154436A0169426B01338B4285
:1001F80028BF00234362002A2FD0EFF31181502338
:1002080083F31288436B1A68D2072CD470B45E68E3
:100218006EB9456A826A954217D084691444DC60D5
:100228000ED9AA1A5A608562002280F850201A68EE
:1002380042F00102C9B21A6081F3118870BC70479C
:100248000469A21A5A608662EEE7012380F85030EA
:10025800C9B281F3118870BC7047C26C136843F04F
:10026800800313607047C9B281F31188704700BFDB
:10027800026B10B462B1036CC2684469D11A013BC5
:10028800615C5DF8044B08BF13460364C8B270474D
:10029800016A4369C4685B5C0131A14228BF114609
:1002A80001625DF8044BD8B2704700BF436B13B1CD
:1002B80090F850007047836A406A181AB0FA80F0C4
:1002C80040097047416A836A99420AD3CB1A416B45
:1002D800026961B14968501E0B4483420AD2C01AB0
:1002E800704702691144CB1A416B0029F2D1501EA4
:1002F800C01A704700207047036B43B1026C5B68FB
:1003080093422FBF981AC0689B1AC0187047C269D9
:10031800036A9A422FBFD01AC0688018C01A704763
:100328000A4B30B503F1140493F900205D78072ACD
:10033800C8BF143A811804330D7313F8025C85544E
:1003480013F8012C0A76A342EED130BD8CFD0208C9
:1003580003682DE9F041DF691FB13B46BDE8F04174
:100368001847002A164611DD04460D460E4400E0E3
:1003780023689B68204698470028F9D0236815F819
:10038800011B1B6820469847AE42F1D1BDE8F081B9
:10039800002324212522017042708370C3707047A6
:1003A800232383702423437125230372704700BFDE
:1003B80030B4836813B11C689B882385436840F276
:1003C800E93401E0002C3FD01D89013C15F0020FF3
:1003D800A4B2F7D0197303F10C0540F2E93101E03A
:1003E80000293BD01C89013914F0010F89B2F7D0DC
:1003F8002B78436840F2E93100E0D9B11C89013912
:1004080014F0020F89B2F8D01A7303F10C0440F209
:10041800E93200E072B11989013A11F0010F92B284
:10042800F8D02378836813B11A689B8893610120F8
:1004380030BC70470F4A9342F4D10F4A538D0133B1
:100448009BB25385538DEDE70A498B42D2D10A4CB2
:10045800618D013189B26185618DCBE705498B4298
:10046800C7D105494B8D01339BB24B854B8D4368F2
:10047800C0E700BF003C004084640020002870B53D
:100488001EDB0928044620DD012303EB83035B0000
:10049800B0FBF3F2092AF8D87BB10E4EB4FBF3F0A7
:1004A8000928CCBF57223022A6FB03E5024403FBF0
:1004B8001044EB0801F8012BF0D100230B7070BD3C
:1004C8002D230B7040420131DBE7303001F8010B7E
:1004D800F3E700BFCDCCCCCC884230B44FF0010458
:1004E8002ED301FB04F4B0FBF4F58D42F9D284B1AC
:1004F800AAB901E0B0FBF4F5092DCCBF5722302290
:100508002A4404FB150003F8012BB4FBF1F4002C7A
:10051800F0D100221A7030BC7047B0FBF4F5092DF9
:10052800CCBF372230222A4404FB150003F8012BE4
:10053800B4FBF1F4002CF0D100221A7030BC7047E3
:100548000546002AEBD1D7E703685A1C02601970E8
:10055800704700BF2DE9F047089C2578002B80469E
:1005680089460CBF4FF0200A4FF0300A661C35B39D
:10057800002A29DD334601E0024698B113F8011B31
:10058800501E0029F8D1971E60B13D46013D5146E5
:100598004046C8476B1C002BF8DC257827EAE77033
:1005A800013055B1041B29464046C847301916F892
:1005B800015B002DF7D1BDE8F087BDE8F087002A80
:1005C80004DC2846BDE8F0870020EBE7571EDCE78F
:1005D80083684268D0ED037A00EB830101339342CC
:1005E80081ED040A836004BF0023836000EB83036A
:1005F80093ED047A036870EE277A9A42C0ED037A85
:1006080077EEC77AC0ED037A0CDA013307EE103AB9
:10061800F8EEC76AB7EE007A87EEA60A036030EEF6
:10062800070A704707EE102AB8EEC77A87EE870ADE
:10063800704700BF90ED057A90ED004AD0ED066A4C
:10064800D0ED014AD0ED047A90ED035AD0ED025A6C
:10065800A4EE007AB0EE406AB0EE470AB0EE667AD1
:10066800A6EE247A67EEC07AA0EE457AE6EE257A01
:1006780080ED057AC0ED067A704700BFD0ED057AA7
:1006880090ED013AD0ED003AD0ED064A90ED024ADD
:1006980090ED077A90ED035A90ED086AD0ED045A70
:1006A800C0ED067AF0EE406A27EE830AC0ED056ACF
:1006B800A3EEA60A80ED087AA4EE240AA5EE470A5E
:1006C800A5EEC60A80ED070A704700BFD0ED007A94
:1006D80090ED017A30EE670AE7EE007AB0EE670A2D
:1006E800C0ED007A704700BF704700BF0A449142CE
:1006F80014D030B40139551E41F2210211F8014FCE
:10070800082380EA042004044CBF82EA4000400029
:10071800013B80B2F7D18D42F0D130BC704700BFA9
:100728004FF40063838270474FF4006383827047FD
:1007380090F8203033B1012B03D14FF4006383824A
:10074800704770474FF480638382704770B50446E2
:1007580082B01430E56D06236A464321A847B0B13C
:100768009DF804009DF800609DF801109DF8025066
:100778009DF803209DF8053041EA062143EA00234D
:1007880042EA0522A187E287A4F84030012002B09E
:1007980070BD00BF70B5044682B00830656A062394
:1007A8006A463B21A847A8B19DF804009DF800605F
:1007B8009DF801109DF802509DF803209DF8053022
:1007C80041EA062143EA002342EA0522E182228324
:1007D8006383012002B070BD10B490E80600047B6A
:1007E80040690223A3404B6013685DF8044B4FF641
:1007F800FE710B401360C3E470B40468037B226885
:10080800022101FA03F31A4213D042690A49582017
:1008180000FB02124FF6FE7650685289C5680068E0
:10082800296831402960C168D24392B20A40C26047
:10083800636070BC704700BFD865002030B4094BB6
:100848001C7864B1084B002503EBC4041A68998826
:100858005562D06808330143A342D160F6D130BC59
:10086800704700BF986800209C68002010B4026898
:10087800047B11680223A340194209D00649406845
:1008880000240C7001684FF6FE742140016053602B
:100898005DF8044B704700BFC3540020F0B4334CDC
:1008A80000EB800004EB80046468002C5BD0304EC1
:1008B80049004FF42040CDB23060A169090444D406
:1008C80060682C4F45F08071384041F49031014305
:1008D8004FF420406160306003E0411E002838D0AA
:1008E8000846A1698F07F8D54FF42040A26230600E
:1008F80002E0421E68B31046A2691106F9D5626883
:100908001C4945F0007545F480350A4015434FF4FD
:1009180020406560306002E0421ED0B11046A269F6
:100928009207F9D5A362A3694FF420409B06306073
:1009380005D4431E68B11846A3699B06F9D5202340
:100948003060E3610120F0BC7047411E08B10846E1
:10095800B3E7094A138801339BB24FF0FF31316086
:100968001380F0BC70472046F0BC7047D06100206F
:10097800F8610020009800FCFC610020134601206B
:100988000A4668218AE700BF30B50446C06C617129
:100998000368A26823F00103036087B0A37900927B
:1009A80013F004023DD04FF4805213F00203019279
:1009B80044D102934FF480630022039311F00103A2
:1009C800059237D1049308238D07694648BF0493DD
:1009D80028F034FA6079E36CA17900F00202002A69
:1009E80015BF4FF440324FF480324FF400340024E6
:1009F80010F0010F586808BF2246CC074CBF0243CD
:100A080020EA02025A609A6809074CBF42F00802BD
:100A180022F008029A601A6842F001021A6007B0D0
:100A280030BD13F0020301920BD04FF4005513466A
:100A38000295C1E7042304930C23C5E74FF4005340
:100A4800B7E70293B8E700BF10B50446C06CA160D1
:100A5800036823F001030360A37986B013F004024E
:100A6800009141D04FF4805213F00203019244D117
:100A780002934FF4806362790393D1074FF0000328
:100A88000493059345BF0423049308230C23694664
:100A9800920748BF049328F0D1F96079E36CA179F3
:100AA80000F00202002A15BF4FF440324FF48032A2
:100AB8004FF40034002410F0010F586808BF224694
:100AC800CC074CBF024320EA02025A609A68090721
:100AD8004CBF42F0080222F008029A601A6842F0FD
:100AE80001021A6006B010BD13F00203019207D08C
:100AF8004FF4005113460291BDE74FF40053B7E796
:100B08000293B8E7002303604360192343701A2354
:100B1800C37001234371C37170472DE9F34105691F
:100B280006460F467DBBD0F80080C8F30A0323B3FE
:100B38000023D6F80080019326F006F8042819D17E
:100B4800214C236943F001032361BBB2A8F80030AC
:100B580025F0FAFF04282ED108F102030193019B26
:100B68003F0C1F8025F0F0FF2369042823F00103C0
:100B7800236125D06FF0010505E025F0E5FF042885
:100B880005D04FF0FF35284602B0BDE8F0810E4C85
:100B9800236943F002032361C4F81480236943F0F6
:100BA8004003236125F0D0FF2369042823F00203C2
:100BB8002361BDD0E5E7236923F001032361D9E769
:100BC800336804333360DEE700200240F8B504469A
:100BD8000D468E180027B54201D12069F8BDE3689B
:100BE800591CE160234415F8012B1A720429F2D12B
:100BF800A1682046FFF791FFE7602061EBE700BF9F
:100C080000B5002183B00A2023F076F80F210A20CE
:100C180023F072F801AA0321102023F091F89DF91E
:100C28000430DFED277ADFED275A06EE103A9DF9FA
:100C3800053006EE903A9DF9063007EE103AB8EE08
:100C4800C66AF8EEE66AB8EEC77A76EEE76A36EE76
:100C5800676A37EE677AF7EE007AB0EE675AA6EE63
:100C6800255A194B0021B0EE456AB0EE675AA6EE38
:100C7800A55A0A20E7EE257AF3EE0E5A26EE256AE3
:100C880025EE257A67EEA57A83ED006A83ED017A71
:100C9800C3ED027A23F030F80DF10302012102209E
:100CA80023F04EF80DF103020121092023F048F842
:100CB80001210A2023F020F8012003B05DF804FB8D
:100CC800000000430000803B0000002070B582B0A7
:100CD80004466946143022F0C5FFB0B19DF80500FE
:100CE8009DF801609DF802109DF803509DF80420BE
:100CF8009DF8063041EA062143EA002342EA05222C
:100D0800A187E287A4F84030012002B070BD00BF7F
:100D18000846194624F0EEB82DE9F04FDFF830C147
:100D2800474A4849484E494D8046102718F1FF3830
:100D3800C0F08480DCF80430C3F30803002B5CD1D6
:100D4800EFF31183002B58D10B68946800BF086833
:100D58008342F9D1D6F800904FF47A7000FB09FE6F
:100D6800AEEB040EBEFBF9FE00FB03EEDCF804302C
:100D7800C3F308034FF47A740120FBB9EFF311832E
:100D8800E3B90B68D2F808A000BFD1F800904B4532
:100D9800F7D1D6F800B004FB0BF9A9EB0A09B9FBA7
:100DA800FBF904FB0393A3EB0E03B3F57A7FBDD2E3
:100DB800DCF80430C3F30803002BDFD0EFF3118A0B
:100DC80087F31288D2F808B01368DB0344BF2860A1
:100DD800D2F808B00B68D5F800905FFA8AFA8AF35F
:100DE8001188D6F800A0994404FB0AF3A3EB0B037F
:100DF800B3FBFAF304FB0933D5E7EFF3118487F368
:100E08001288D2F808901368D80303D501232B6001
:100E1800D2F808900B682868E4B284F31188D6F8F1
:100E280000A04FF47A7400EB030E04FB0AF3A3EB63
:100E38000903B3FBFAF304FB0E3E97E7BDE8F08F16
:100E480010E000E0A4610020A8610020A06100205B
:100E580000ED00E038B5044600F11405236E802249
:100E68006B21284698476420FFF756FF236E072218
:100E78006821284698476420FFF74EFF236E00221A
:100E88006B21284698476420FFF746FF236E01220E
:100E98006B21284698470F20FFF73EFF94F8532010
:100EA800236E032A8CBF1A2218221B212846984732
:100EB8000F20FFF731FF236E18221C212846984780
:100EC8000F20FFF729FF236E94F852201A21284695
:100ED80098470F20FFF720FF236E94F8542019211C
:100EE800284698476420FFF717FF236E1022372102
:100EF800284698470F20FFF70FFF2846236E012248
:100F0800382198470F20BDE8384005E770B50446FA
:100F180000F11405236E80226B212846984764202F
:100F2800FFF7FAFE236E284603226B219847236EAB
:100F380094F854201921284698470F20FFF7ECFE13
:100F4800236E94F8522028461A219847236E284683
:100F580018221B219847236E284618221C219847DF
:100F6800236E28460222372198472846236E0122FD
:100F78003821BDE870401847204B5B68C3F308036D
:100F880030B4BBB9EFF31183A3B91D4B1D4C1868DE
:100F9800A16800BF1A689042F9D11B4B1C684FF436
:100FA8007A7202FB04F3591AB1FBF4F130BC02FB6C
:100FB80000107047EFF31182102383F31288114950
:100FC8008C680B6813F4803F104B02D00120186026
:100FD8008C680B49D2B20D68186882F311880A4BE5
:100FE80019684FF47A72284402FB01F31B1B30BCCA
:100FF800B3FBF1F302FB0030704700BF00ED00E0E7
:10100800A461002010E000E0A8610020A061002099
:101018002DE9F84F8046FFF7AFFF254E2549DFF849
:10102800A0E0254A254D844610274FF47A74012004
:10103800DEF80430C3F30803D3B9EFF31183BBB967
:101048000B68D2F808A000BFD1F800904B45F7D143
:10105800D6F800B004FB0BF9A9EB0A09B9FBFBF9B8
:1010680004FB0393A3EB0C034345E1D3BDE8F88FDE
:10107800EFF3118A87F31288D2F808B01368DB03FC
:1010880044BF2860D2F808B00B68D5F800905FFA22
:101098008AFA8AF31188D6F800A0994404FB0AF367
:1010A800A3EB0B03B3FBFAF304FB0933DAE700BF46
:1010B800A8610020A461002010E000E0A0610020E9
:1010C80000ED00E010B504460120A269138823F062
:1010D80040031B041B0C138013889BB223F03803B6
:1010E80043F03003138013889BB243F0400313800E
:1010F800FFF78EFF2046FFF7ADFE102204F1140023
:101108006A21FFF755F96420FFF706FEA2691388E4
:1011180023F040031B041B0C1380138823F03803AF
:101128001B041B0C138013889BB243F040031380ED
:101138000120BDE810406BE708B5FFF71DFF044B21
:101148005B68C01AC0F5FA5020EAE07008BD00BF1D
:10115800545E002030B4EFF31183102282F312881A
:101168000649074C0A680748013200250A602560CD
:10117800DBB2026883F3118830BC7047A461002099
:10118800A061002010E000E01D4B70B59C68E36C86
:10119800226BDD69C2B1636B2BB12B0702D5E36CFF
:1011A80008221A6270BD2A06F7D5A26A616A8A42C5
:1011B8001FD0511CA069A162825C2069E66C814243
:1011C8003285EAD3A362E8E7A906E4D5E26A1AB150
:1011D800988C80B29047DEE7E1699B8C6069DBB24E
:1011E8004E1CE6614354E169E368994228BFE26115
:1011F800D1E7E26C136823F080031360CDE700BFEA
:10120800782C00201D4B70B55C68E36C226BDD699F
:10121800C2B1636B2BB12B0702D5E36C08221A62AB
:1012280070BD2A06F7D5A26A616A8A421FD0511C8E
:10123800A069A162825C2069E66C81423285EAD3AA
:10124800A362E8E7A906E4D5E26A1AB1988C80B2ED
:101258009047DEE7E1699B8C6069DBB24E1CE66172
:101268004354E169E368994228BFE261D1E7E26C3F
:10127800136823F080031360CDE700BF782C0020AB
:101288001D4B70B51C68E36C226BDD69C2B1636BE2
:101298002BB12B0702D5E36C08221A6270BD2A060F
:1012A800F7D5A26A616A8A421FD0511CA069A1625F
:1012B800825C2069E66C81423285EAD3A362E8E762
:1012C800A906E4D5E26A1AB1988C80B29047DEE7A5
:1012D800E1699B8C6069DBB24E1CE6614354E169AD
:1012E800E368994228BFE261D1E7E26C136823F012
:1012F80080031360CDE700BF782C002003685B6A89
:1013080003B11847704700BF03681B6A03B1184749
:10131800704700BF03682DE9F041DF691FB13B4604
:10132800BDE8F0411847002A164611DD04460D466F
:101338000E4400E023689B68204698470028F9D0AF
:10134800236815F8011B1B6820469847AE42F1D167
:10135800BDE8F08103689B69184700BF03685B69B3
:10136800184700BF0368DB68184700BF03689B681D
:10137800184700BF03685B68184700BF03681B680D
:10138800184700BF014B1868F8E700BFD86A00206B
:10139800054B53F8203033B11A689B88918A0B4269
:1013A80018BF1B0493617047B864002003682DE9D7
:1013B800F04F03F13845644EAD0A0124755D05F020
:1013C8001F066D09022D04FA06F400F0A280032D11
:1013D80000F0A480012D52D08088B0FA80F4C4F1C6
:1013E8001F04A4B2E50803EB850504F007042E6A80
:1013F800A4000F27A74026EA07062E622E6A01F0EE
:10140800030702FA04F47A1E3443012AC1F3810C5B
:10141800C1F300182C62C1F3411135D9C60700F198
:101428009780850700F1A380440700F1B180020787
:1014380000F1BF80C60600F1CD80850600F1DB8093
:10144800440600F1E980020600F1F780C60500F1C4
:101458000581850500F11381440500F1218102050C
:1014680000F12F81C60400F13D81850400F14B8114
:10147800440400F15981020455D4BDE8F08F334D7E
:101488006E6934436C61A7E7002422464FF0010ED1
:101498004FF0030904E00132102A04F10204ECD0F1
:1014A8000EFA02F636EA0005F5D1D3F808A009FAD3
:1014B80004F5ED430AEA050AC3F808A0D3F808B012
:1014C8000CFA04FA4AEA0B0AC3F808A0B3F804A015
:1014D8001FFA8AFA2AEA06069E80B3F804A008FAD8
:1014E80002F646EA0A06B6B29E801E682E401E60C4
:1014F800D3F800A007FA04F646EA0A061E60D3F8F5
:101508000CA001FA04F605EA0A0A46EA0A05DD60B3
:10151800C1E70E4DAE693443AC615DE70B4DEE6932
:101528003443EC6158E71A6822F040421A601A689E
:1015380042EA87771F60DA6822F0404242EA817106
:10154800D960BDE8F08F00BF602103080010024099
:101558001A6822F003021A601A683A431A60DA68B5
:1015680022F003020A438507DA607FF55DAF1A6847
:1015780022F00C021A601A6842EA87021A60DA68D6
:1015880022F00C0242EA81024407DA607FF54FAF8D
:101598001A6822F030021A601A6842EA07121A60C2
:1015A800DA6822F0300242EA0112DA6002077FF5B7
:1015B80041AF1A6822F0C0021A601A6842EA87121C
:1015C8001A60DA6822F0C00242EA8112C606DA60BE
:1015D8007FF533AF1A6822F440721A601A6842EA3B
:1015E80007221A60DA6822F4407242EA012285066C
:1015F800DA607FF525AF1A6822F440621A601A682B
:1016080042EA87221A60DA6822F4406242EA8122BA
:101618004406DA607FF517AF1A6822F440521A6060
:101628001A6842EA07321A60DA6822F4405242EA3B
:101638000132DA6002067FF509AF1A6822F44042E7
:101648001A601A6842EA87321A60DA6822F440425D
:1016580042EA8132C605DA607FF5FBAE1A6822F4E9
:1016680040321A601A6842EA07421A60DA6822F4BD
:10167800403242EA01428505DA607FF5EDAE1A682C
:1016880022F440221A601A6842EA87421A60DA682D
:1016980022F4402242EA81424405DA607FF5DFAE57
:1016A8001A6822F440121A601A6842EA07521A604D
:1016B800DA6822F4401242EA0152DA6002057FF544
:1016C800D1AE1A6822F440021A601A6842EA8752B8
:1016D8001A60DA6822F4400242EA8152C604DA60EB
:1016E8007FF5C3AE1A6822F040721A601A6842EA9F
:1016F80007621A60DA6822F0407242EA01628504E1
:10170800DA607FF5B5AE1A6822F040621A601A688E
:1017180042EA87621A60DA6822F0406242EA81622D
:101728004404DA607FF5A7AE1A6822F040521A60C6
:101738001A6842EA07721A60DA6822F0405242EAEE
:101748000172DA6097E600BF036803F138422DE9B9
:10175800F04F920A584DAA5C02F01F055209012465
:10176800022A04FA05F400F08C80032A00F08E8027
:10177800012A3CD001F003077A1E012AC1F3810C2B
:10178800C1F300188088C1F3411135D9C60700F1AB
:101798009780850700F1A380440700F1B180020714
:1017A80000F1BF80C60600F1CD80850600F1DB8020
:1017B800440600F1E980020600F1F780C60500F151
:1017C8000581850500F11381440500F12181020599
:1017D80000F12F81C60400F13D81850400F14B81A1
:1017E800440400F15981020455D4BDE8F08F334A0E
:1017F80055692C435461BDE7002422464FF0010E81
:101808004FF0030904E00132102A04F10204ECD07D
:101818000EFA02F636EA0005F5D1D3F808A009FA5F
:1018280004F5ED430AEA050AC3F808A0D3F808B09E
:101838000CFA04FA4AEA0B0AC3F808A0B3F804A0A1
:101848001FFA8AFA2AEA06069E80B3F804A008FA64
:1018580002F646EA0A06B6B29E801E682E401E6050
:10186800D3F800A007FA04F646EA0A061E60D3F881
:101878000CA001FA04F605EA0A0A46EA0A05DD6040
:10188800C1E70E4A95692C43946173E70B4AD56901
:101898002C43D4616EE71A6822F040421A601A6835
:1018A80042EA87771F60DA6822F0404242EA817193
:1018B800D960BDE8F08F00BF602103080010024026
:1018C8001A6822F003021A601A683A431A60DA6842
:1018D80022F003020A438507DA607FF55DAF1A68D4
:1018E80022F00C021A601A6842EA87021A60DA6863
:1018F80022F00C0242EA81024407DA607FF54FAF1A
:101908001A6822F030021A601A6842EA07121A604E
:10191800DA6822F0300242EA0112DA6002077FF543
:1019280041AF1A6822F0C0021A601A6842EA8712A8
:101938001A60DA6822F0C00242EA8112C606DA604A
:101948007FF533AF1A6822F440721A601A6842EAC7
:1019580007221A60DA6822F4407242EA01228506F8
:10196800DA607FF525AF1A6822F440621A601A68B7
:1019780042EA87221A60DA6822F4406242EA812247
:101988004406DA607FF517AF1A6822F440521A60ED
:101998001A6842EA07321A60DA6822F4405242EAC8
:1019A8000132DA6002067FF509AF1A6822F4404274
:1019B8001A601A6842EA87321A60DA6822F44042EA
:1019C80042EA8132C605DA607FF5FBAE1A6822F476
:1019D80040321A601A6842EA07421A60DA6822F44A
:1019E800403242EA01428505DA607FF5EDAE1A68B9
:1019F80022F440221A601A6842EA87421A60DA68BA
:101A080022F4402242EA81424405DA607FF5DFAEE3
:101A18001A6822F440121A601A6842EA07521A60D9
:101A2800DA6822F4401242EA0152DA6002057FF5D0
:101A3800D1AE1A6822F440021A601A6842EA875244
:101A48001A60DA6822F4400242EA8152C604DA6077
:101A58007FF5C3AE1A6822F040721A601A6842EA2B
:101A680007621A60DA6822F0407242EA016285046D
:101A7800DA607FF5B5AE1A6822F040621A601A681B
:101A880042EA87621A60DA6822F0406242EA8162BA
:101A98004404DA607FF5A7AE1A6822F040521A6053
:101AA8001A6842EA07721A60DA6822F0405242EA7B
:101AB8000172DA6097E600BF10B50409013C052CF5
:101AC80017D80D4B33F8142000F00F0042FA00F33A
:101AD80013F001030DD0012303FA00F00138104080
:101AE8002BF0F0FC054A064B125D104403EBC000D6
:101AF80010BD002010BD00BF482103085421030871
:101B08002C6000202DE9F04F4A484B4B4B4C4FF0CE
:101B180090414FF0010A4FF002094FF004084FF0CE
:101B2800080C4FF0100E20274026802530F8022B95
:101B380012F0010F03D01960A3F804A0083312F0C3
:101B4800020F03D01960A3F80490083312F0040FB1
:101B580003D01960A3F80480083312F0080F03D0EB
:101B68001960A3F804C0083312F0100F03D01960ED
:101B7800A3F804E0083312F0200F02D019609F8008
:101B8800083312F0400F02D019609E80083312F01B
:101B9800800F02D019609D80083312F4807F05D031
:101BA8004FF4807B1960A3F804B0083312F4007F67
:101BB80005D04FF4007B1960A3F804B0083312F481
:101BC800806F05D04FF4806B1960A3F804B0083318
:101BD80012F4006F05D04FF4006B1960A3F804B03D
:101BE800083312F4805F05D04FF4805B1960A3F8C6
:101BF80004B0083312F4005F05D04FF4005B19609D
:101C0800A3F804B0083312F4804F05D04FF4804B8A
:101C18001960A3F804B00833D20B04D04FF4004283
:101C280019609A80083301F58061A1427FF47EAF84
:101C3800BDE8F08F482103082C60002000180048F8
:101C4800002867D003682DE9F04F03F138445C4E53
:101C5800A40A0125345D04F01F066409022C05FA64
:101C680006F558D0032C00F0A580012C58D08088A8
:101C7800B0FA80F4C4F11F04A4B2E50803EB8505AB
:101C880004F007042E6AA4000F27A74026EA0706D7
:101C98002E622E6A01F00307A2407C1E3243012CFB
:101CA800C1F3810CC1F300182A62C1F341113CD978
:101CB800C60700F18980850700F19580440700F187
:101CC800A380020700F1B180C60600F1BF80850637
:101CD80000F1CD80440600F1DB80020600F1E980C6
:101CE800C60500F1F780850500F10581440500F17E
:101CF8001381020500F12181C60400F12F818504BA
:101D080000F13D81440400F14B81020400F1598146
:101D1800BDE8F08F70472B4CA6693543A561A6E74F
:101D2800284C666935436561A1E7002422464FF0D7
:101D3800010E4FF0030904E00132102A04F10204F5
:101D4800E6D00EFA02F636EA0005F5D1D3F808A077
:101D580009FA04F5ED430AEA050AC3F808A0D3F81E
:101D680008B00CFA04FA4AEA0B0AC3F808A0B3F858
:101D780004A01FFA8AFA2AEA06069E80B3F804A08D
:101D880008FA02F646EA0A06B6B29E801E682E4097
:101D98001E60D3F800A007FA04F646EA0A061E6099
:101DA800D3F80CA001FA04F605EA0A0A46EA0A057D
:101DB800DD60C1E7034CE6693543E56157E700BFDD
:101DC80060210308001002401A6822F003021A601A
:101DD8001A683A431A60DA6822F003020A43850750
:101DE800DA607FF56BAF1A6822F00C021A601A6885
:101DF80042EA87021A60DA6822F00C0242EA81029B
:101E08004407DA607FF55DAF1A6822F030021A6085
:101E18001A6842EA07121A60DA6822F0300242EAC7
:101E28000112DA6002077FF54FAF1A6822F0C0028C
:101E38001A601A6842EA87121A60DA6822F0C00249
:101E480042EA8112C606DA607FF541AF1A6822F4C9
:101E580040721A601A6842EA07221A60DA6822F4A5
:101E6800407242EA01228506DA607FF533AF1A68CC
:101E780022F440621A601A6842EA87221A60DA6815
:101E880022F4406242EA81224406DA607FF525AFF7
:101E98001A6822F440521A601A6842EA07321A6035
:101EA800DA6822F4405242EA0132DA6002067FF52B
:101EB80017AF1A6822F440421A601A6842EA873259
:101EC8001A60DA6822F4404242EA8132C605DA60D2
:101ED8007FF509AF1A6822F440321A601A6842EA9C
:101EE80007421A60DA6822F4403242EA0142850564
:101EF800DA607FF5FBAE1A6822F440221A601A688D
:101F080042EA87421A60DA6822F4402242EA8142B1
:101F18004405DA607FF5EDAE1A6822F440121A60C3
:101F28001A6842EA07521A60DA6822F4401242EA52
:101F38000152DA6002057FF5DFAE1A6822F440022A
:101F48001A601A6842EA87521A60DA6822F4400274
:101F580042EA8152C604DA607FF5D1AE1A6822F0EF
:101F680040721A601A6842EA07621A60DA6822F058
:101F7800407242EA01628504DA607FF5C3AE1A68EE
:101F880022F040621A601A6842EA87621A60DA68C8
:101F980022F0406242EA81624404DA607FF5B5AE1D
:101FA8001A6822F040521A601A6842EA07721A60E8
:101FB800DA6822F0405242EA0172DA6002047FF5E0
:101FC800A7AE1A6822F040421A601A6842EA877778
:101FD8001F60DA6822F0404242EA8171D960BDE8A8
:101FE800F08F00BF002852D0036803F138422DE972
:101FF800F04F920A504DAA5C02F01F0552090124C5
:10200800022A04FA05F443D0032A00F09080012A3A
:1020180043D001F003077A1E012AC1F3810CC1F3F2
:1020280000188088C1F341113CD9C60700F18880A7
:10203800850700F19480440700F1A280020700F1AF
:10204800B080C60600F1BE80850600F1CC8044064B
:1020580000F1DA80020600F1E880C60500F1F6809A
:10206800850500F10481440500F11281020500F1A3
:102078002081C60400F12E81850400F13C814404CE
:1020880000F14A81020400F15881BDE8F08F7047E1
:102098002A4A95692C439461BBE7284A55692C4321
:1020A8005461B6E7002422464FF0010E4FF00309B1
:1020B80004E00132102A04F10204E6D00EFA02F616
:1020C80036EA0005F5D1D3F808A009FA04F5ED437E
:1020D8000AEA050AC3F808A0D3F808B00CFA04FA0B
:1020E8004AEA0B0AC3F808A0B3F804A01FFA8AFA50
:1020F8002AEA06069E80B3F804A008FA02F646EA21
:102108000A06B6B29E801E682E401E60D3F800A054
:1021180007FA04F646EA0A061E60D3F80CA001FA8C
:1021280004F605EA0A0A46EA0A05DD60C1E7034A39
:10213800D5692C43D4616CE7602103080010024084
:102148001A6822F003021A601A683A431A60DA68B9
:1021580022F003020A438507DA607FF56CAF1A683C
:1021680022F00C021A601A6842EA87021A60DA68DA
:1021780022F00C0242EA81024407DA607FF55EAF82
:102188001A6822F030021A601A6842EA07121A60C6
:10219800DA6822F0300242EA0112DA6002077FF5BB
:1021A80050AF1A6822F0C0021A601A6842EA871211
:1021B8001A60DA6822F0C00242EA8112C606DA60C2
:1021C8007FF542AF1A6822F440721A601A6842EA30
:1021D80007221A60DA6822F4407242EA0122850670
:1021E800DA607FF534AF1A6822F440621A601A6820
:1021F80042EA87221A60DA6822F4406242EA8122BF
:102208004406DA607FF526AF1A6822F440521A6055
:102218001A6842EA07321A60DA6822F4405242EA3F
:102228000132DA6002067FF518AF1A6822F44042DC
:102238001A601A6842EA87321A60DA6822F4404261
:1022480042EA8132C605DA607FF50AAF1A6822F4DD
:1022580040321A601A6842EA07421A60DA6822F4C1
:10226800403242EA01428505DA607FF5FCAE1A6821
:1022780022F440221A601A6842EA87421A60DA6831
:1022880022F4402242EA81424405DA607FF5EEAE4C
:102298001A6822F440121A601A6842EA07521A6051
:1022A800DA6822F4401242EA0152DA6002057FF548
:1022B800E0AE1A6822F440021A601A6842EA8752AD
:1022C8001A60DA6822F4400242EA8152C604DA60EF
:1022D8007FF5D2AE1A6822F040721A601A6842EA94
:1022E80007621A60DA6822F0407242EA01628504E5
:1022F800DA607FF5C4AE1A6822F040621A601A6884
:1023080042EA87621A60DA6822F0406242EA816231
:102318004404DA607FF5B6AE1A6822F040521A60BB
:102328001A6842EA07721A60DA6822F0405242EAF2
:102338000172DA6002047FF5A8AE1A6822F0404202
:102348001A601A6842EA87771F60DA6822F040420A
:1023580042EA8171D960BDE8F08F00BF10B103680F
:1023680082881A85704700BF10B1036882889A6115
:10237800704700BF38B100298388026814BF002164
:1023880010218B40936170470E4B1B8801463BB967
:102398000D4B0E4A1B7810680BB981F00101E9E773
:1023A8000B4B5A691AB118B91A68106058747047FB
:1023B800084A18681188084A92FBF1F20121026064
:1023C80059747047C4640020C6640020C8640020A3
:1023D800CC640020E464002020A1070010B40A4B5C
:1023E8000A4A1C7801238340234052F8200029B967
:1023F800B3FA83F149095DF8044BBBE7191C18BF10
:1024080001215DF8044BB5E7B4640020B8640020EE
:1024180030B1036882881B8A1A4214BF0120002049
:10242800704700BF2DE9F0410B4E346873691C40BA
:102438000FD0DFF828800127B4FA84F3C3F11F0313
:1024480007FA03F558F8230003689847AC43756109
:10245800F2D1BDE8F08100BF00040140FC1D00205E
:102468002DE9F0410B4E346873691C400FD0DFF83A
:1024780028800127B4FA84F3C3F11F0307FA03F590
:1024880058F8230003689847AC437561F2D1BDE85A
:10249800F08100BF00040140FC1D00202DE9F0413F
:1024A8000B4E346873691C400FD0DFF82880012771
:1024B800B4FA84F3C3F11F0307FA03F558F82300AD
:1024C80003689847AC437561F2D1BDE8F08100BF5D
:1024D80000040140FC1D00202DE9F0410B4E34683A
:1024E80073691C400FD0DFF828800127B4FA84F301
:1024F800C3F11F0307FA03F558F823000368984748
:10250800AC437561F2D1BDE8F08100BF0004014021
:10251800FC1D00202DE9F0410B4E346873691C4006
:102528000FD0DFF828800127B4FA84F3C3F11F0322
:1025380007FA03F558F8230003689847AC43756118
:10254800F2D1BDE8F08100BF00040140FC1D00206D
:102558002DE9F0410B4E346873691C400FD0DFF849
:1025680028800127B4FA84F3C3F11F0307FA03F59F
:1025780058F8230003689847AC437561F2D1BDE869
:10258800F08100BF00040140FC1D00202DE9F0414E
:102598000B4E346873691C400FD0DFF82880012780
:1025A800B4FA84F3C3F11F0307FA03F558F82300BC
:1025B80003689847AC437561F2D1BDE8F08100BF6C
:1025C80000040140FC1D00200B490C4A8B6943F0B4
:1025D800010310B58B611368094C43F480531360F1
:1025E8002046402200212DF018FB4FF0FF332364D2
:1025F800C4F8433010BD00BF001002400000014085
:10260800FC1D00202DE9F041044618460D461646EB
:1026180098462AF0ADFA2768E6722844A07229463F
:102628007D69434632462046AC46BDE8F0416047E6
:10263800036810B504461B689847236820469B68C2
:102648009847A37B0133A37310BD00BFF0B48489FE
:102658004FF6FF764FF47A740BB300292ED00F781B
:10266800013101E0B44217D00589013CAD07A4B29D
:10267800F8D507734FF47A7402E0BCB2B4420BD0B9
:102688000589ED0704F1FF37F7D5057BEDB20AB1EF
:1026980015700132013BDFE7094B984202D0012057
:1026A800F0BC7047074A538D01339BB25385508D58
:1026B80080B2003018BF0120F0BC7047FF27D3E775
:1026C800003C00408464002070B50646806810B164
:1026D80004688088208541F08001706840F2E93400
:1026E80000E0F4B10589013C15F0020FA4B2F8D05E
:1026F800017300F10C0540F2E93100E0D9B1048919
:10270800013914F0010F89B2F8D0297870680021D6
:10271800FFF79CFFB36813B11A689B889361012087
:1027280070BD0A498842F2D1094C618D013189B2E4
:102738006185618DEBE705498842E7D10448418D01
:10274800013189B24185418D7068E0E7003C004065
:102758008464002038B50B4C2378054653B90A4ADF
:102768006378106849212A4600252570FFF7ACFFD9
:10277800012038BDFEF7E0FC0028F0D0FEF748FC49
:10278800EDE700BF545E0020505E0020F0B54D4CD0
:1027980094F84750012D83B013D02AD3022D0DD1C0
:1027A800494B1B780646002B7BD16846FFF7D2FFC2
:1027B80020B19DF8063013F0030025D0002003B0A7
:1027C800F0BD414E3378002B66D16846FFF7C2FF53
:1027D8009DF8003008B1DB0768D4002384F847303F
:1027E800337853B100230133002084F8473003B015
:1027F800F0BD354E3378002BF4D10121022021F0B1
:10280800C9FA94F84730EEE79DF801E09DF800100A
:102818009DF803709DF802209DF805509DF804303E
:1028280084F8470041EA0E2142EA072243EA0523D9
:1028380009B212B21BB2494252425B42234806EE29
:10284800901A07EE102A07EE903A90ED005AD0ED54
:10285800015A90ED026AF8EEE66AB8EEC77AF8EE29
:10286800E77A66EE856A27EE257A67EE867AFDEEC8
:10287800E66ABDEEC77AFDEEE77A16EE901A17EE15
:10288800102A17EE903A31807280B38001210A2015
:1028980021F032FA03B0F0BDFEF74EFC002894D0C8
:1028A8008CE7FEF749FC002888D17EE733782BB9FE
:1028B8000721032021F06EFA94F84750013584F877
:1028C80047507BE7FC1D0020545E002000000020DC
:1028D800427A02B9704710B504460368406804F1AB
:1028E8000A0198470023637210BD00BF437A5A1C3F
:1028F8000344D2B242729972037A934200D802B961
:10290800704710B504460368406804F10A01984707
:102918000023637210BD00BF30B40B4D002305F1D6
:10292800140101E0272B0BD011F8132082424FEA43
:10293800430403F10103F5D12C44607D30BC70479A
:10294800002030BC704700BF8CFD020870B5448879
:1029580006460D46C4F30B042246002128462DF0F6
:102968005CF93369094A934209D3094A934206D26A
:10297800224628461946BDE870402AF0CDBE23B14C
:1029880021462846BDE87040184770BDF85D030829
:10299800EC5E0308064B07498B4202D30023184616
:1029A80070471A88C2F30B029042F8D01433F3E749
:1029B800C0590308F85D0308024A136823EA0000B7
:1029C80010607047806F0020F8B5174D2B78A32B47
:1029D80028D16B78BE2B25D1022229464FF6FF70ED
:1029E800FDF784FE114FAC1C22884AB1A618BE42DE
:1029F80018D2052A16D92146FDF778FE3446F3E7A2
:102A080021460222FDF772FE0222A118FDF76EFE92
:102A18000634074B641B1C8041F60F53C31A5842F7
:102A28005841F8BD0020F8BD00F003080000040874
:102A3800903400202DE9F04FDFF848914C4F8BB0CF
:102A48000326A7EB09071822002104A82DF0E5F8B2
:102A5800484BCDF8109005971A69120604D5464AD6
:102A68005A6002F188325A6001228DF824203422FB
:102A7800DA60424B424C1B88ADF8003002226946AE
:102A880004A8FEF7A3F8022269464FF6FF70FDF787
:102A98002DFEDFF8F4A080464FF0000B544536D3E6
:102AA8000AAC002524F8245D0222214604A8FEF77A
:102AB8008DF8022221464046FDF718FE40BAC04371
:102AC800ADF80800022202A904A8FEF77FF80798CB
:102AD80060B106ABC0F10402294618442DF09DF8F8
:102AE800069904A8FEF719F8079508909DF8243070
:102AF800089A23B11F490B6943F080030B61013E1B
:102B08002DD0002A9FD1FFF75FFF50B32CE06588D6
:102B18008DF80DB0C5F30B05AB1DADF80830238853
:102B2800C3F30B02ADF80A201B0B062202A904A866
:102B38008DF80C30FEF74AF8062202A94046FDF748
:102B4800D5FD616880462A4604A8FEF73FF861680B
:102B580040462A46FDF7CAFD143480469EE7002AFF
:102B6800D1D0052002F084FC0BB0BDE8F08F00BF87
:102B7800000004080020024023016745EEFD02081A
:102B8800C059030800F00308F85D03080378202BF8
:102B9800024600F10100F9D0092BF7D02D2B2CD0DB
:102BA8002B2B03BF5378B7EE000A0246B7EE000A94
:102BB800A3F13001C8B209289FED467A10D8F2EE89
:102BC800046A07EE901AF8EEE77A12F8013FE7EE8A
:102BD800267AA3F13001C8B20928B0EE677AF0D995
:102BE8002E2B4CD003F0DF03452B0BD0F7EE007AE9
:102BF80067EE276A20EE260A70475378BFEE000A70
:102C08000246D5E710B451782D2959D02B290ABF8F
:102C18009178501C901C0024A1F13003092B53D843
:102C2800002303EB830301EB430310F8011FA1F119
:102C38003002092AA3F13003F3D9B3F59A7F28BFEC
:102C48004FF49A73072B42D9DFED236A1A46F7EE41
:102C5800007A083A072A67EEA67AFAD803F007033B
:102C68002BB1F2EE046A013B67EEA67AFBD124B3DE
:102C7800C7EE276A5DF8044B20EE260A70475378A2
:102C8800A3F13001C8B2092802F10102AAD8F2EE74
:102C9800046AF0EE665A07EE901AF8EEE77A12F830
:102CA800013F87EEA66AA3F13001C8B2092866EE93
:102CB800A56A37EE067AEED994E767EE276AD9E770
:102CC800901C91780124A7E7F7EE007ACFE7F7EE9A
:102CD800007AC5E70000000020BCBE4CB5EEC00A73
:102CE800DFED317AF1EE10FACCBF30EE270A30EE84
:102CF800670ADFED2E7A20EE270A30B5FDEEC07A9E
:102D080087B017EE904A054684EAE470002303A9C9
:102D1800A0EBE4700193009302931BF0E3FB002CFB
:102D2800ACBF20232D2303A88DF8003029F020FF05
:102D3800012803A924D002282DD0032805BF302359
:102D4800684668468DF801302CF08DFF684629F0FA
:102D58000FFF0338C4B22246694628462CF0E1FF2B
:102D680000232B55284629F003FF2E22431C2A5402
:102D78000DEB0401E8182CF093FF284607B030BD8E
:102D8800302368468DF801308DF802308DF8033015
:102D98002CF069FFDAE7302368468DF801308DF8AA
:102DA80002302CF060FFD1E76F12033A00007A443A
:102DB8002DE9F041064615460846B6FBF2F43CB943
:102DC80005FB1464124B1B5D00F8013BBDE8F08164
:102DD800B4FBF2F767B90E4B05FB174705FB146404
:102DE800DA5D00F8012B1B5D00F8013BBDE8F081BE
:102DF800B7FBF2F8B8F1000F02D04046FFF7D8FF52
:102E080005FB1878024B13F8082000F8012BE3E7BC
:102E1800A426030830B402681146531C036011F855
:102E2800024B0160D31C517803609378151D05602F
:102E38001B0443EA0123D078234343EA006030BCF3
:102E4800704700BF0368591C1A46016012F8021B3C
:102E58000260587841EA0020704700BF03685A1C96
:102E680002601878704700BF38B5044600681546F8
:102E78002AF052FC22682A44226038BD036810B444
:102E88000A0A5C1C04601A7003685A1C02601970F4
:102E98005DF8044B704700BF03685A1C026010B409
:102EA800197003680A0A5C1C04601A7003680A0C2B
:102EB8005C1C04601A700368090E5A1C02601970C1
:102EC8005DF8044B704700BF03685A1C0260197014
:102ED8000368090A5A1C0260197070472DE9F04707
:102EE800002488B080460F461E46A14605AD531CF7
:102EF8000393117839B3252933D1931CCDF8109059
:102F08000393507830284ED04FF0000AA0F13003D8
:102F1800DBB2092B42D96C2819D0642800F09380C1
:102F280024D825281CD063D9582876D063281BD1EB
:102F380031784046B847039A531C039311780436F6
:102F480001340029D7D1204608B0BDE8F087039B9B
:102F58005A1C03921B78642B7CD02AD8252B54D179
:102F6800252140460134B847039AC0E7732833D077
:102F780044D975284FD106F1040E30682B4600223B
:102F88000A217646FDF7A8FA049A00955346394671
:102F98004046FDF7DFFA039A0444A8E704AA03A908
:102FA8001BF07CFAB7E7D31C039390784FF0010A23
:102FB800ACE7732B10D05BD9752B3AD0782B96D110
:102FC800A3F15802B2FA82F2306852092B46102156
:102FD8000436FDF781FAD7E73368049A0093394637
:102FE80000234046FDF7B6FA04360444039A7EE708
:102FF8000028B9D1204608B0BDE8F0876E28B3D1C3
:10300800039A336804361C6071E72AD9582BD7D045
:10301800632B8DD06BE77828A6D1A0F15802B2FABD
:1030280082F2306852092B461021FDF755FA043612
:10303800AAE706F1040E30682B4600220A217646DC
:10304800FDF74AFAA0E7331D306829461E46FDF70A
:1030580015FA99E7331D306829461E46FDF70EFA22
:1030680092E7002B7FF443AF204608B0BDE8F08715
:103078006E2BC6D03BE700BF0EB400B584B005ABDD
:10308800019053F8042B0649039301A8FFF726FF84
:10309800019B00221A7004B05DF804EB03B070477E
:1030A800510500080FB430B583B006AB0A490B4888
:1030B80053F8042B096800680193FFF70FFF084CC9
:1030C80005462068FEF74AF90028FAD0284603B0DA
:1030D800BDE8304004B070476C2C0020702C0020F4
:1030E800D86A0020DFED2B7AB4EEE70AF1EE10FA89
:1030F8004ADDDFED296A9FED297A01E0B0EE670A23
:10310800B4EEC70AF1EE10FA70EE667AF6DC9FEDBF
:10311800247AF4EEC77AF1EE10FA38D5DFED1E6A9C
:103128009FED207A01E0F0EE407AF4EEC77AF1EEF6
:1031380010FA37EEA60AF6D4DFED1B7AB4EEE70AEA
:10314800F1EE10FA14DDDFED137A37EEC00A60EE07
:10315800006A9FED166A9FED167ADFED167AA6EEE5
:10316800867A20EE266AE6EE877AA6EE270A704768
:10317800DFED117AB4EEE70AF1EE10FA44BFDFEDA5
:10318800087A37EEC00AE2E7F0EE407ABFE7B0EE21
:10319800670AD1E7DB0F4940DB0FC940E4CB164192
:1031A800DB0F49C0E4CB16C1DB0FC93F92E741B939
:1031B8009730083C15A82ABEDB0FC9BF09B909E03A
:1031C800194690FBF1F301FB13030846002BF7D1D6
:1031D800084670470146FBE710B507EE901A2DED3B
:1031E800028BB8EE678ADFED217A28EE008A044662
:1031F80028EE278AB0EE480A2AF04EFCF0EE408A04
:10320800B0EE480A2AF0AAFBF7EE007A9FED187A8A
:10321800F0EE675AE8EE875A0023A361B0EE676ABA
:10322800C7EEA56A63612362E361A8EEC76ABDECD5
:10323800028B77EEC07AB6EE007AF8EE005A27EEE7
:10324800877A20EE250A27EE267A26EE266A67EE8A
:10325800A67A20EE260A84ED046AC4ED017A84ED8C
:10326800007A84ED027A84ED030A10BD27D4D236A1
:10327800F304353F10B44C09012250F8243001F012
:103288001F0102FA01F10B4340F824305DF8044BAA
:10329800704700BF4B0901F01F0150F8232001239C
:1032A80003FA01F1114214BF18460020704700BF0D
:1032B800F8B5494B1B78022B00F085804749484AEE
:1032C80002238B701370474B1B7B002B59D1464B45
:1032D8004648012219460524DC741A721A7516F03C
:1032E80027FA434B1B78012B66D0424B5A2003F137
:1032F800EA042C213C22187059709A70D870197100
:103308005A714E33A342F6D13B4D3C4C95E80F0021
:1033180005F1100684E80F0096E80F0004F1100785
:1033280005F1200687E80F0096E80F0004F1200752
:1033380005F1300687E80F0096E80F0004F1300722
:1033480005F1400687E80F0096E80F0004F14007F2
:1033580005F1500687E80F0096E80F0004F15007C2
:1033680005F1600687E80F0096E80F00703504F154
:10337800600686E80F0095E80F00703484E80F00B7
:10338800F8BD1F49184A0B681E4D1F4C1F4F204897
:1033980043F480630B6002260023167253721146B1
:1033A800442201262A827B71A370667016F0C0F948
:1033B8000F4B1B78012B98D11649094A4FF4FA4054
:1033C8000880137091E7144B0022282029211870D7
:1033D8005970DA709A7076E702380020E0680020A9
:1033E800E43D002000000020446A0020CC260308A9
:1033F80044310020326E0020F0FD02088C5100207C
:10340800806F0020285F00208C2C002000440020C2
:10341800D8260308B06500206446002010B5222095
:10342800FEF74AFB144CA06418B1112200238271E4
:10343800C3712021FEF7D6FD1520FEF73DFBE064A1
:1034480018B1112200238271C3712021FEF7CAFD31
:1034580021F0FEFAA06CFEF7DBFF084B002814BF32
:1034680001220222E06C1A70FEF7D2FF10B1044B61
:1034780000221A7310BD00BFFC1D00200238002076
:1034880000000020B0F1FF3F0AD0022810B403DC8E
:103498005DF8044BFDF702BA00205DF8044B704755
:1034A80000207047F0B55B4B5B4A97B019689142B2
:1034B80000AF00F0A3805949594A00234FF4700027
:1034C800C1F888003B607B60136843F48033136065
:1034D80003E03B68B3F5A04F09D0136803F4003349
:1034E8007B603B6801333B607B68002BF1D04C4B21
:1034F8001B6813F4003318BF01237B607B68012B22
:1035080052D0464C464B474AE260474A596A1160D6
:103518005A6A42F080725A625A6942F4FC025A614D
:103528000025032207F10801012341F6FF764FF039
:103538009040FD60BE603A73BB7325F0DBFC4FF62C
:10354800FF7307F108013948BB6025F0D3FC07F188
:1035580008013748374E25F0CDFC07F108013648F9
:1035680025F0C8FC07F10801344825F0C3FC07F131
:103578000801334825F0BEFC07F1080025F070FA71
:10358800BB683049304AA1FB031330499B0CF0203B
:103598004FF0070E5C370B60566084F82300956087
:1035A800C2F800E0BD46F0BD294A1D4B122111604A
:1035B8005A685A605A685A605A6842F480625A6077
:1035C8005A6822F47C125A605A6842F4E8125A6027
:1035D8001A6842F080721A601A689201FCD559681C
:1035E8000F4A21F003015960596841F002015960FE
:1035F800536803F00C03082BFAD182E700221A6003
:1036080062B6144B1B6883F30888134B1B689847F2
:10361800FEE700BFFC9F0020EFBEADDE00ED00E03E
:10362800001002400005FA053C460020000400484E
:10363800000800483F190100000C0048001000482D
:103648000014004883DE1B4310E000E0A86100205E
:103658000020024000D8FF1F04D8FF1F70B50F4C90
:103668000F4DC0EBC00004EB800468692669304345
:10367800686182B09209667BA1600025012101A8DA
:1036880063618DF804608DF805208DF806508DF87B
:10369800071025F001F902B070BD00BFC805002071
:1036A80000100240074BC0EBC00030B403EB8000B1
:1036B800054C056963692B4363610176427630BC2A
:1036C800704700BFC8050020001002402DE9F04FE8
:1036D8005E4C54F8204083B0002C71D0666D98463B
:1036E80091465B4B7268E264A160236004F15A0161
:1036F8004FF4807304F5AD726161A261E3602361E8
:103708000746307E21F0F2F9F068A8B1514B00214C
:103718005A68904203F11C0300F0928001310C2991
:10372800F6D100207A1CD2B20C21FFF7BBFFE36C64
:10373800F26822632433A364B068D8B1454B0021F2
:103748005A68904203F11C0378D001310C29F7D153
:1037580000257A1CD2B20B212846FFF7A3FF234687
:10376800F27E3D492846FFF779FFE36CB268626351
:103778002833636494F85900FEF79EF9054694F8D7
:103788005800FEF799F918F0080F824696F819B014
:103798001AD0CDB118F0110F4FF00B0307F1010744
:1037A80014BF4E213E21EF715A46AB712846FEF7F1
:1037B80047FA18F0010F45D0236B5BB3636B4BB32B
:1037C800204603B0BDE8F08F18F0010F0CBF4FF092
:1037D8002E084FF04E0819F0020F09D045B10B2200
:1037E8007B1CAA71EB7128465A464146FEF728FA17
:1037F80019F0010FE0D0BAF1000FDDD001370C232A
:103808008AF807705A4641468AF806305046FEF74D
:1038180017FAD1E7337FB27E8DF804209B09002187
:10382800012201A88DF805308DF806108DF80720C3
:1038380025F032F8204603B0BDE8F08FCDB288E716
:10384800C8B26FE72846FEF789FDB5E7782C002057
:1038580070FE0208C8050020E10700080348D0F8F8
:103868003C3113B100F59A7018477047C80500201D
:103878000348D0F8203113B100F58C701847704711
:10388800C80500200348D0F804310BB1FC301847B4
:10389800704700BFC80500200348D0F8E8300BB1D6
:1038A800E0301847704700BFC80500200348D0F82B
:1038B800CC300BB1C4301847704700BFC805002092
:1038C8000348D0F8B0300BB1A8301847704700BF94
:1038D800C80500200348D0F894300BB18C30184745
:1038E800704700BFC80500200248836F0BB17030D5
:1038F80018477047C80500200248C36D0BB1543003
:1039080018477047C80500200248036C0BB13830CF
:1039180018477047C80500200248436A0BB11C309D
:1039280018477047C80500200248836803B1184744
:10393800704700BFC80500201749184B184A194896
:1039480010B4D1F8884044F47004C1F888401C6869
:1039580044F001041C605C6822405A601A6822F036
:10396800847222F480321A601A6822F480221A6063
:103978005A6822F4FE025A60DA6A22F00F02DA620A
:103988001A6B002410404FF0006218639C608A6034
:103998005DF8044B704700BF00ED00E000100240E6
:1039A8000CC07FF8CCFC00FF38B50B4C23688BB1FA
:1039B8005A68821A002A054604DA0CE05A68AA1ADC
:1039C800002A07DB9A68226018461A68904723681D
:1039D800002BF3D138BD38BD803700200B4B0022B7
:1039E80010B4027203F1C804042102E0072A09DCBA
:1039F8009979890702D51979815401329C4203F1DA
:103A08001403F3D15DF8044B704700BF6821030825
:103A180010B40D4C04232146002200E08B7913F0EA
:103A2800010301F1140106D101320B2AF6D103700A
:103A38005DF8044B704702EB820204EB82025DF8EA
:103A4800044B13790370704768210308012214237B
:103A580002704370704700BF08B512F0E7F8024BD8
:103A6800024ADA60FEE700BF00ED00E00400FA0554
:103A7800024A034B1278197817F076BD7423002098
:103A8800752300202DE9F0470569C3681D4028D03B
:103A98000F4606464FF000484FF00009B5FA85F387
:103AA80028FA03F2D2431B3B32611540042B16D887
:103AB800DFE803F03129211903007B6A002B32D09B
:103AC80003F1FF3A1FFA8AFAC7F824903C6A34B126
:103AD80023682046514698476468002CF8D1002D89
:103AE800DCD1BDE8F0873868716B036889B2984704
:103AF800002DD3D1F5E77868B16B036889B2984790
:103B0800002DCBD1EDE7B868F16B036889B298470F
:103B1800002DC3D1E5E7F868316C036889B298478E
:103B2800002DBBD1DDE7F36A1FFA83FACEE700BFA9
:103B38002DE9F04F2DED028BA0F10A0389B00C4658
:103B4800E72B00F23E86DFE813F01C013C063C063A
:103B58003C063C063C063C063C063C063C063C064D
:103B68003C063C063C063C063C063C063C063C063D
:103B78003C063C063C063C063C062D013C063C0641
:103B88003C0651053C063C063C064B013C065801E8
:103B98003C062C023C0621023C0619023C06C103E5
:103BA8003C06F1013C063C063C06EB01E4013C0600
:103BB800DD013C063C06D6013C06AE013C063C064F
:103BC8003C069C013C063C063C063C06C7053C06F8
:103BD800FC003C063B04E7053C063C063C063C066C
:103BE8003C063C063C060F053C06D2043C069E04F7
:103BF8003C064A043C0605023C063C063C063C06DC
:103C08009C056105BF050B06E8003C063C068C03D5
:103C18000E033C06D702BB023C063C063C063C06AB
:103C2800B0023C063C068F023C063C063C0680027D
:103C38006902780336033C063C063C0627033C062B
:103C480018031B043C063C063C063C063C063C06A6
:103C58003C063C063C063C063C063C063C063C064C
:103C68003C069C053C063C063C063C063C063C06DD
:103C78003C063C063C063C063C063C063C063C062C
:103C88003C063C063C063C063C063C063C063C061C
:103C98003C063C063C063C063C063C063C063C060C
:103CA8003C063C063C063C063C063C063C063C06FC
:103CB8003C063C063C063C063C063C063C063C06EC
:103CC8003C063C063C063C063C063C063C063C06DC
:103CD8003C063C063C063C063C063C063C063C06CC
:103CE8003C063C063C063C063C063C063C063C06BC
:103CF8003C063C063C063C063C063C063C063C06AC
:103D08003C063C063C063C063C063C063C063C069B
:103D18003C063C063C061004E603AE4E337853B12D
:103D2800AD4F002537F8021F2046FFF7CDF833784E
:103D38000135AB42F6DC012009B0BDEC028BBDE8D1
:103D4800F08FA44E3378002BF5D0A44F0025B84649
:103D5800236817F81520591C21601A7098F801106B
:103D680001EB810101EB810101F2EE2189B22046CC
:103D7800FFF7AAF833780135AB4208F10208E7DC0F
:103D8800D9E7974D284628F0F3FE0028D3DD2B46C7
:103D98000544226813F8011B501C9D4220601170D5
:103DA800F7D1C8E78F4D05F15006287823F0D0FDEC
:103DB8002368027A591C21601A7023686A78591C92
:103DC80021601A702368AA78591C21601A70236828
:103DD800EA780435591CAE4221601A70E5D1AAE789
:103DE8000B68814A581C1178206019702368527832
:103DF800591C216001201A709EE77C4D0B682A7AB5
:103E0800591C21601A70A98B2046FFF75DF8298B91
:103E18002046FFF759F8698B2046FFF755F82368C5
:103E2800EA7C591C21601A70A98C2046FFF74CF8CF
:103E3800E98C2046FFF748F82368AA7F591C2160BF
:103E48001A70236895F82020591C21601A70698C13
:103E58002046FFF739F82368EA7A591C21601A705E
:103E6800E9682046FFF718F823682A7C591C216066
:103E78001A70236895F82120591C216001201A70B6
:103E88005AE70B6800255A1C0A60204629461D700F
:103E9800FFF702F829462046FEF7FEFF294620468E
:103EA800FEF7FAFF47E70B684F4A514D1178514A20
:103EB800581C2060197011682046FEF7EDFF236832
:103EC8004A4A591C127A21601A7029882046FEF73E
:103ED800FBFFA9882046FEF7F7FF29892046FEF751
:103EE800F3FF00212046FEF7EFFF20460021FEF7F2
:103EF800EBFF012020E7084608223C49FEF7B4FF03
:103F0800012019E70B683C4A581C91782060197009
:103F18006CE70B6801229918216010461A700BE7AC
:103F280008460021FEF7B8FF012005E7334D344E5F
:103F380005F1300795F90210324B93F906208A42B1
:103F480003F1080300F040849E42F6D10835BD42D3
:103F5800F0D1F0E60B682C4A2C49D0782C4A5D1C2D
:103F68002560187023684979581C206019702368E7
:103F7800D278591C216001201A70DDE60B681B4AB3
:103F8800591C527D216001201A70D5E6214D05F19A
:103F9800800655F8041F2046FEF77EFFAE42F8D192
:103FA800C9E61D4D05F14006B5F880102046FEF71C
:103FB8008BFF236895F88220591C21601A702368AA
:103FC80095F883200435591CAE4221601A70EBD154
:103FD800B1E600BF286D0020D65200201C590020F1
:103FE800CC3D0020303E00202C3E0020446A0020BA
:103FF800A42C0020806F00200C3E0020285F0020A9
:10400800F84E0020C84E0020F03D0020FC5600204D
:10401800003E0020BC530020C05300200A689C4B7F
:104028009C491878551C2560107022685878551CD2
:104038002560107022689B78501C20601370204601
:10404800C988FEF741FF012076E6924D0846298887
:10405800FEF73AFF69882046FEF736FF2046A98812
:10406800FEF732FF012067E68B4D05F16006A9884F
:104078002046FEF729FFE9882046FEF725FF298913
:104088002046FEF721FF2368AA7A591C21601A707E
:104098002368EA7A591C21601A7055F80C1B2046CF
:1040A800FEF7FAFEB542E2D145E67C495223226882
:1040B800501C2060137011F8013F002BF7D13AE62D
:1040C800774800232268056803EB4301561C6D5CA2
:1040D80026601570026825680A446E1C52782660AE
:1040E8002A70026825680A4401339278691C0A2BF1
:1040F80021602A70E6D11EE66A4D0B682A68591CB1
:10410800127821601A702B6822689978531C2360F2
:10411800002311702A6821681A4401335279481C17
:10412800032B20600A70F5D123682A68591C127A7B
:1041380021601A7023682A68591CD27821601A7085
:1041480023682A68591C127921601A702B68204646
:104158005989FEF7B9FE2A682368527A591C2160EA
:104168001A702A6842E600212046FEF795FE20468E
:104178000021FEF7A9FE0120DEE54B4B4B49B3F9C0
:10418800003081FB0321DB17C3EBA101204689B274
:10419800FEF79AFE0120CFE5454D0846298AFEF72D
:1041A80093FE698A2046FEF78FFE2046A98AFEF70D
:1041B8008BFE0120C0E5DFF810E10027FEB2714652
:1041C80000232268501C206016702268501C206052
:1041D8001370226811F8010F0133551C062B256056
:1041E8001070EED10137062F0EF1060EE6D13149D7
:1041F80000232268501C206017702268501C206021
:104208001370226811F8010F0133551C0B2B256020
:104218001070EED12368284A581C072120601970B5
:1042280023680021581C20601970236892F8F02038
:10423800591C216001201A707EE50B681F4A20492D
:104248001078194A5D1C2560187023688978581CF5
:104258002060197023689278591C216001201A7017
:104268006AE5184D08462988FEF72EFE698820461B
:10427800FEF72AFEB5F904300C4AD91782FB03234E
:10428800C1EBA301204689B2FEF71EFE012053E5CB
:10429800E83D00201C340020442E002098FE02082F
:1042A8009C6C0020DC6D0020003E0020676666667E
:1042B800B0650020A3540020C0530020E06800200F
:1042C800F03D0020206D00207F5400209F4B03F11B
:1042D8005A0522685979501C206011702268197893
:1042E800501C2060117022685978501C2060117091
:1042F80022689978501C206011702268D978501C67
:1043080020601170226819790633501C9D42206084
:104318001170DED10FE58E4B03F170052268197814
:10432800501C2060117022685978501C2060117050
:1043380022689978501C206011702268D978501C26
:104348002060117022681979501C20601170226851
:104358005979501C20601170226899790733501CD4
:104368009D4220601170D9D1E5E47A4D0846E9896B
:10437800FEF7AAFD2046A989FEF7A6FD0120DBE489
:104388000B68754F591C3A7821601A703B78002BDE
:104398003FF4D1AC0025EEB2304619F025FA236877
:1043A8004278591C216030461A7019F01DFA0189AB
:1043B8002046FEF789FD3B780135AB42EBDCBAE4D9
:1043C8000B6800255A1C0A601D700B685A1C0A608D
:1043D8001D700B685A1C0A6029461D705BE5002198
:1043E8002046FEF771FD00212046FEF76DFD0021F5
:1043F8002046FEF769FD2368584D00265A1C2260A6
:104408001E7023682A68591C92F82C2021601A70A3
:1044180023682A68591C92F8362021601A7023688C
:104428002A68591C92F8372021601A7023685A1C90
:1044380022601E7023685A1C22601E7023685A1C52
:1044480022601E702B682046598FFEF73DFD2B68B1
:104458002046198FFEF738FD23682A68591C92F800
:104468002E2021601A7023685A1C22601E702B6847
:104478002046598EFEF728FD2B682046998EFEF7B8
:1044880023FD012058E4364E0B687279334D591CD0
:1044980021601A702B682046198CFEF715FD2B68D1
:1044A8002046D98BFEF710FD71892046FEF70CFDDA
:1044B800B1892046FEF708FD2B682046598CFEF787
:1044C80003FD2B682046998CFEF7FEFCF1892046F7
:1044D800FEF7FAFC318A2046FEF7F6FC2A682368C4
:1044E80092F82620591C216001201A7024E41C4EE1
:1044F800F378002B00F060820B680822591C2160B9
:104508001A7023680122991821601A702368154DC2
:10451800591C2A7921601A702368AA78591C2160CD
:104528001A7029882046FEF7CFFCE9892046FEF755
:10453800CBFC2368F279591C21601A702368EA7849
:10454800591C216001201A70FFF7F6BBD4310020F6
:10455800382F0020F03D0020964300209C6C00205E
:10456800E0680020B065002016F0F2FFFF2806463C
:1045780000F02E8208A9002501F8125D0DF10D004A
:104588008DF80D5016F0C4FF08A800F8115D16F05C
:10459800B3FF08A800F8105D16F0A2FF08A820F8DD
:1045A800085D16F091FF23685A1C22601E7023686C
:1045B8009DF80D20591C21601A7023689DF80E2063
:1045C800591C21601A7023689DF80F20591C21601E
:1045D8001A7023689DF81020591C21601A70204613
:1045E800BDF81810FEF770FCFFF7A5BBA54D0846EF
:1045F8002988FEF769FCA9882046FEF765FC204655
:104608002989FEF761FC0120FFF796BB9E4B9B8A28
:10461800B3F5006F00F2CE81B3F5806F00F2EF8141
:10462800B3F5007F34BF01270227984D05F10C062A
:1046380055F8041B91FBF7F1204689B2FEF744FCBC
:10464800AE42F5D1924D934F05F10C06B5EC010A37
:10465800D7ED087A80EE270A29F0D2F981B22046F0
:10466800FEF732FCAE42F1D18B4D05F10C0655F840
:10467800041B204689B2FEF727FCAE42F7D1FFF7AC
:104688005ABB00258146DFF84882DFF848B2059515
:1046980004950695079501214FF6FF7A05E0013547
:1046A8000B2D00F0AF8018F9011F4F1C4AFA05F3D3
:1046B800F5D0DE07F3D5BBF800302B41D807EED58F
:1046C80006A8FEF7D7FDEAE7084610227349FEF769
:1046D800CBFB0120FFF730BB0B68714D591C2A79C1
:1046E80021601A7023686A79591C21601A70298818
:1046F8002046FEF7E9FB2368AA79591C21601A7045
:1047080069882046FEF7E0FB2368EA79591C216096
:1047180001201A70FFF710BB0B68624E01255A1C66
:104728000A601D700B68B278591921601A7015F06B
:10473800C7F923685C4A5D495F1927601870B1F9A9
:104748000010B2F90000FEF739FD23685A192260FB
:10475800187031882046FEF7B7FB2846FFF7ECBAF9
:10476800534D544E9FED548ADFF86C81DFED538A28
:1047780005F120070EE0FCEEE77ACDED017ABDF8F1
:10478800041020460435FEF79FFBAF4206F11806D9
:104798003FF4D1AA717C0029F3D0494BD5ED007ABA
:1047A8001B78012BE7D1474B1B68DB0440F1FA80EB
:1047B800F5EE407AF1EE10FA40F0238140F2DC5138
:1047C800DFE70020FFF7B8BA23685A1C2260197087
:1047D80029882046FEF778FB2368EA78591C21606F
:1047E8001A7023682A79591C21601A702368AA79DB
:1047F800591C21601A7023686A79591C21601A7043
:10480800FFF7A4BBDFF8D4A000254FF00808013556
:10481800C5F1200208FA02F2A5F120032AFA05F6EA
:10482800164328FA03F31E43252D06F001024FF024
:1048380000030BD01343EAD0E8B226F0B7FE0028F5
:10484800E5D0294606A8FEF715FDE0E71E4B1B78C4
:10485800DA0700F1C48000251C4E2F4602E001351E
:10486800252D3DD029463046FEF714FD0028F6D008
:10487800294606A8FEF70EFD002840F08E80013775
:10488800EDE700BFA42C0020C86C0020006D0020BC
:10489800F868002000620020106D0020F83B00201E
:1048A800343400204E6F00204E3C0020503C002045
:1048B800083C0020F06400200000404200E08244F0
:1048C800D465002004690020FC6B0020506B002098
:1048D800C8FE0208EE540020DB9B914190E33FF4B0
:1048E800664B674DB3F850102046FEF7EDFA654B5E
:1048F8001988204689B2FEF7E7FA634B19684B011D
:1049080003F02002C1F340031343C1F3800243EADA
:104918004203C1F3C00243EA8203C1F3401243EAEF
:10492800C20301F0100119432046FEF7CDFA04A98D
:1049380004222046FEF798FA23682978534A581C1F
:104948002060197011886429A8BF64212046FEF7E9
:10495800BBFAB9F1960F47D000212046FEF7B4FA0A
:104968002168B7F1190348BFA7F11203A3F3C403E1
:104978004A1C226020461A460B7005A9FEF774FAF5
:104988002368434A581C102120601970204611885A
:10499800FEF782FA0120FFF7CFB9394604A8FEF7DF
:1049A80069FC6CE7F4EEC87AF1EE10FA45DA4FF4D8
:1049B8007A71E6E6082738E60B68B178354A581C5C
:1049C8002060197023681278591C21601A709DE5BF
:1049D80023685A1C226001201E70FFF7ADB9069BA0
:1049E80043F00103069336E723680322591C21602C
:1049F8001A7023686A78591C21601A70B0E7042776
:104A080013E6F4EEC87AF1EE10FA3FF5D7AEF4EEFD
:104A1800E87AFDEEE77AF1EE10FA17EE901A1ED852
:104A28006FF4F973303903FB01F140F2E73391FB7E
:104A3800F3F101F2DB5189B2A3E6FDEEE77A40F229
:104A4800E73217EE903A303B02FB03F388FB031280
:104A5800D917C1EB622101F2E93189B291E640F23E
:104A6800F313A1F5836103FB01F140F2E73391FBF6
:104A7800F3F101F2DD5189B283E600BFC4010020E1
:104A8800906C0020FC610020C46C0020923400204F
:104A9800746D0020E43D002008B501210220FDF7D7
:104AA8009DFC094B1B7803F00503052B08D000215A
:104AB8000120FDF793FC00210846FDF78FFCFEE777
:104AC80011F046F9F3E700BF742C0020022828BF34
:104AD800022010B4084C094B207000EB8002C0EB98
:104AE800C20207495DF8044B013003EB4203C0B230
:104AF8000B601EF007BE00BF906C0020326E0020D5
:104B08009C6C002008B51DF09BF8FDF793FFBDE8ED
:104B180008401DF07DB800BF38B5434B5A899989C4
:104B2800914224BF00225A81198ADA89914224BF0E
:104B38000022DA81DA788AB3072A2FD03B493C4D24
:104B480091F85700012400210A282C709C70D97113
:104B58003DD00C2865D0DFED377A8ABB364C9FED07
:104B6800370AA278002918BFF0EE407A062A04D83E
:104B7800334901EB820191ED0F0A217959B3013ACA
:104B8800032A4DD8F7EE007A87EE800A28F038FF1E
:104B98002388984228BF1846208038BDD97921B18A
:104BA80098780428B8BF04209870204890F85700D7
:104BB8000A280CD00C28CED1DFED227A002ACDD0DD
:104BC800072ACBD00A282CD1DFED1F7AC6E70A20A6
:104BD800DFED1E7AC1E79B78154A07EE103A117887
:104BE800B8EEC77A27EE277A07EE901AF8EEE77A3A
:104BF80067EE877AB4EEE70AF1EE10FA10DDC0EE40
:104C0800077AFDEEE77A17EE903A102BA8BF10232B
:104C1800012BB8BF0123DBB28B4238BF0B461370A0
:104C280038BDDFED0B7A99E7E068002000620020CC
:104C3800E43D00206F120339B06500206F1203387D
:104C480098FE02080AD7A3390F506E3A5304E93880
:104C58006F12833A38B50D4C0D4DAC4206D26168DF
:104C680020461434FDF772FEAC42F8D3FEF720FB61
:104C7800084A094B094C1460002209491A705A70F5
:104C880008480860BDE8384026F030B8C059030825
:104C9800F85D03089C6C0020906C0020326E0020A8
:104CA800DC6D0020A06C002008B5FFF7D3FF1CF0D6
:104CB800C7FFFDF7BFFEBDE808401CF0A9BF00BF55
:104CC800F0B50C292BD8DFE801F06F2A2A2A4C2AE4
:104CD8002A2A2B2A2A2A0700046AB2F80CE09788A5
:104CE8001668674D24F480540462036A4468C169F5
:104CF80023F4005343EA0E3321F4E641A84243EA81
:104D0800073341EA062100F0B58005F50065A842A1
:104D180000F0B08092684460C16102640362F0BD33
:104D2800046A96899588D2F800E0554F24F4807477
:104D38000462036A4468C16923F4007343EA0623E2
:104D480021F07301B84243EA052341EA0E017ED0FF
:104D58004C4DA8427BD092684460C161C263036233
:104D6800F0BD046A96899588D2F800E0444F24F093
:104D780010040462036A4468816923F0200321F067
:104D8800807143EA061321F4E641B84243EA051369
:104D980041EA0E2148D03B4DA84245D09268446074
:104DA800816182630362F0BD046A9389B2F804E00A
:104DB8001768334E24F001040462056A4468816967
:104DC80043EA0E0321F4803125F002059BB221F05D
:104DD8007301B04243EA050341EA070114D0294DA3
:104DE800A84211D005F54065A8420DD005F58065AB
:104DF800A84209D005F58065A84205D092684460AC
:104E0800816142630362F0BDD689158A578A23F00F
:104E1800080333433D43D68824F4407423F0040345
:104E2800ADB233432C43E9E7D589178AD68823F0F6
:104E3800800343EA051324F44064558A23F04003B1
:104E480044EA870443EA061344EA8504A6E7D589B9
:104E5800178AD68823F4006343EA052324F44054D0
:104E6800558A23F4806344EA071443EA062344EA94
:104E7800051470E7158A24F4804444EA851449E748
:104E8800002C0140003401402DE9F04FC8220021D8
:104E980083B07848784CDFF80492784D784E794F93
:104EA800DFF8FC812AF0B9FE77487849DFF8F4E1A9
:104EB800DFF8F4C100221359834200F0C180B3F136
:104EC800804F00F0C980AB4200F0C880B34200F0C8
:104ED800C780BB4200F0C680734500F0C5806345BB
:104EE80000F0C480434500F0C380DFF8C0A15345FB
:104EF8007ED00AF5806A534508BF092379D0143259
:104F0800DC2AD8D15C4C624D624E604F04F1DC085B
:104F180002E01434A04568D0A379002BF9D0237996
:104F28004FEA131909F1FF39B9F1050F03F00F031F
:104F3800EFD835F8190040FA03F2D207E9D54FF057
:104F4800010A0AFA03F3013B184028F0BBFA16F8E5
:104F580009305149184411EBC002DAD051F8300039
:104F6800DFF84CE1217A00F138439B0A1EF8033040
:104F780003F01F0E5B09022B0AFA0EFA62D0032B0C
:104F880065D0012B03D17B694AEA03037B619388CF
:104F98000093B3FA83F3C3F11F039BB2DA0800EB63
:104FA800820203F00703D2F820E09B004FF00F0CB9
:104FB8000CFA03FC2EEA0C0EC2F820E0D2F820E02E
:104FC80001FA03F343EA0E0313626946002302223F
:104FD80014348DF804208DF805308DF806308DF8DE
:104FE800073023F087FFA04596D103B0BDE8F08FC6
:104FF800082309EBC3034FF0010B93F85CA00AF0F8
:105008001F034FEA5A1ABAF1020F0BFA03F30BD037
:10501800BAF1030F0ED0DA457FF471AFD1F814A0BE
:1050280043EA0A034B616AE7D1F818A043EA0A0386
:105038008B6164E7D1F81CA043EA0A03CB615EE701
:105048000023D6E7BB694AEA0303BB619FE7FB6914
:105058004AEA0303FB619AE70123CAE70223C8E788
:105068000323C6E70423C4E70523C2E70623C0E7F2
:105078000723BEE75C5E00206821030800040040A7
:105088000008004000100040002C014000100240C1
:1050980048210308542103082C60002098FE0208C8
:1050A8000040014000140040003401400044014029
:1050B8006021030801490248FEF7E4BCFC5E0020B9
:1050C8000048014001490248FEF7DCBCD45E0020DC
:1050D8000040014001490248FEF7D4BCAC5E002004
:1050E8000004004002494FF08040FEF7CBBC00BFEF
:1050F800845E002001490248FEF7C4BC5C5E0020C3
:10510800002C014001490248FEF7BCBC5C5E00204F
:10511800002C01402DE9F04104684A4DA30AAB4236
:1051280072D009D8B3F5801F6AD04A3DAB425AD134
:105138004FF0700E022608E0434DAB4268D00235AE
:10514800AB4252D14FF0C00E042647794FEA970C74
:10515800002961D0B000634685190227D4F80C8075
:105168009F400CEB4503BFB2384D03F1040C47EAEE
:10517800080745F8231045F82C20E760EFF3118164
:10518800502282F31288821905EBC202136973B3A5
:1051980013620433821905EBC202576917B11F6005
:1051A80053690433821905EBC202976917B11F606E
:1051B80093690433821905EBC202D76917B11F60DE
:1051C800D36904330027CAB21F6082F311883044C0
:1051D80005EBC000036A6BB9E3684FF6FE72134033
:1051E800E360BDE8F081BDE8F081BDE8F08105EB42
:1051F8000E03CFE7E36843F00103E360BDE8F08105
:105208004FF0480E0126A0E74FF0200E00269CE73D
:105218004FF0980E032698E7BF08022306FA03F01A
:10522800BB40DB43E768094D9BB23B4087190CEB59
:10523800470CE3600CF1040345F82C1045F82320D3
:105248009CE700BF4B001000500010005C5E00207F
:1052580030B503685C4D18885C4CB4FBF2F2013938
:10526800013AAB4294B283B089B282B266D0584850
:10527800834263D0B3F1804F60D0A0F59830834269
:105288005CD000F58060834258D0524883425BD09E
:1052980000F5806083427DD022F4407200F58C30A6
:1052A80092B283421A80D9621C850ED0484A934232
:1052B8000BD002F54062934207D002F58062934218
:1052C80003D002F58062934201D100221A8601229E
:1052D8005A611A883C4992B242F001028B421A8004
:1052E80062D0B3F1804F61D03B4A934260D002F55F
:1052F800806293425ED002F5006293425CD002F570
:10530800806293425AD002F59032934258D002F507
:105318004062934256D002F5806293421ED002F555
:105328008062934208BF092219D002A84FF00123D6
:1053380040F8043D23F0B0FA03B030BD254822F010
:105348007002834292B2A3D101201A80D9621C85CF
:1053580058611A8892B202431A80C5E708221F4B87
:1053680003EBC20301A893F85D408DF804400123C4
:1053780000228DF805308DF807308DF8062023F0CF
:105388008BFA1B2CD8D1164B019301A823F084FA71
:1053980003B030BD01201A80D9621C8558611A8873
:1053A80092B202431A809CE70022D8E70122D6E78E
:1053B8000222D4E70322D2E70422D0E70522CEE76F
:1053C8000622CCE70722CAE7002C014000A24A04C3
:1053D80000340140001000400004004098FE02081C
:1053E80019010001204B98422DD0B0F1804F2CD0EC
:1053F800A3F5943398422AD003F58063984228D0C5
:1054080003F50063984226D003F58063984224D0C0
:1054180003F59033984222D003F54063984220D098
:1054280003F58063984207D003F58063984208BF6C
:10543800092202D00020704708220C4B03EBC2035C
:1054480093F85C0070470022F7E70122F5E7022293
:10545800F3E70322F1E70422EFE70522EDE706224E
:10546800EBE70722E9E700BF002C014098FE02089D
:105478002DE9F04F013085B0C3B203938E4D8F4FA5
:105488008F4C904E0A230293DFF840921EF056FA92
:105498004FF4FA7A4FF0100C4FF47A70D9F80430C0
:1054A800C3F30803002B40F0C880EFF31183002BEF
:1054B80040F0C3802968A26800BF2B689942F9D1DF
:1054C800D7F800E000FB0EF39B1AB3FBFEF300FBDA
:1054D80001314FF0010E0191D9F80430C3F30803EC
:1054E800002B40F08E80EFF31183002B40F0898071
:1054F8002B68A16800BF2A689342F9D1D7F800B099
:1055080000FB0BF2521AB2FBFBF200FB0323019AD9
:105518009B1AB3F57A7FDFD3BAF1010ABED1039B98
:10552800002B40F0C4804FF47A7ADFF8A0915046FF
:105538004FF0100CD9F80430C3F30803002B40F0E7
:105548009980EFF31183002B40F094802968A268BA
:1055580000BF2B689942F9D1D7F800E000FB0EF3A1
:105568009B1AB3FBFEF300FB01314FF0010E0191D2
:10557800D9F80430C3F308033BBBEFF3118323BB13
:105588002B68A16800BF2A689342F9D1D7F800B008
:1055980000FB0BF2521AB2FBFBF200FB0323019A49
:1055A8009B1AB3F57A7FE3D3BAF1010AC2D1029B01
:1055B800013B02937FF468AF4349444B4448454A52
:1055C8000860DA6005B0BDE8F08FEFF311888CF35E
:1055D8001288A1682368DB0344BFC6F800E0A1680D
:1055E8002B6832685FFA88F888F31188D7F800804A
:1055F8001A4400FB08F35B1AB3FBF8F300FB023311
:10560800CDE7EFF311888CF31288A1682368DB03D8
:1056180044BFC6F800E0A1682B6832685FFA88F8D2
:1056280088F31188D7F800801A4400FB08F35B1A46
:10563800B3FBF8F300FB023369E7EFF311828CF355
:105648001288D4F808E02368D90303D5012333600E
:10565800D4F808E02B683168D2B282F311883A682E
:10566800194400FB02F3A3EB0E03B3FBF2F300FBB8
:1056780001312EE7EFF311828CF31288D4F808E099
:105688002368D90303D501233360D4F808E02B68D5
:105698003168D2B282F311883A68194400FB02F3E8
:1056A800A3EB0E03B3FBF2F300FB01315DE71846F1
:1056B8001FF030FE37E700BFA4610020A86100207A
:1056C80010E000E0A0610020FC9F002000ED00E059
:1056D800EFBEADDE0400FA052DE9F047B14FB24E3A
:1056E8001CF0AEFABE421ED2DFF84483DFF84493C2
:1056F8004446258862197DB14A450DD2052D0BD93E
:1057080033886188C3F30B03994200F0FA8014468A
:1057180025886219002DEFD1716830461436FDF7DF
:1057280015F9BE42E4D3A14A1378A3F1170102295F
:105738000FD99F4911F83300002840F00481D800A0
:105748000144497829B19B4911F83330002B00F006
:105758002281994C6378022B84BF002363702378DD
:10576800022B84BF00232370944B9A78042A00F0FC
:10577800098132B91A88B2F5F07F84BF4FF4F0720C
:105788001A808F4D8F4A2B681A40002A00F0068134
:10579800D80700F1F280590400F1EA801A0700F1F5
:1057A800E2809B0400F1D880874D2B685A8C998C35
:1057B800914224BF00225A84FFF7AEF920F03EFF41
:1057C80010B982481DF0FEF88020FDF7F5F84FF477
:1057D8000070FDF7F1F84FF48020FDF7EDF84FF475
:1057E8000010FDF7E9F84FF00070FDF7E5F84FF00D
:1057F8008060FDF7E1F84FF00060FDF7DDF86378B1
:10580800022B06D8724A734903EB430302EB830366
:105818000B602378022B07D803EB83016E4AC3EB96
:10582800C10302EB43032B6025F038FF002130222F
:105838006A482AF0F2F928680FF0CAFE684B2E6809
:1058480003F1500102E0043399427AD01A78002A11
:10585800F9D19C78D8788442F5D26249624B91F8A4
:1058680004E06248624D5C6B624B2860C827642183
:1058780011FB0E71DFF8C0E159605F4F30F8061C6C
:105888005E4DAEF8001000219960D9601961596128
:105898009961D96183F8201083F821103A702E603D
:1058A8000CB113F0A5FD564B9FED565A1B88564A6E
:1058B8009FED566A5579564C56495748086006EE8A
:1058C800903AF8EEE66A1388C5EE265A07EE103AC3
:1058D80053881279C4ED005A07EE903AB8EEC77AA9
:1058E8004E4BF8EEE77A1D725A7227EE067A67EE8B
:1058F800867ABDE8F04783ED017AC3ED007A1CF0A3
:1059080087B963799B077FF402AF716894F804A0A4
:105918003046FDF71BF83388BAEB133F04D0143632
:10592800BE42FFF4E5AEFEE673887068AA1FC3F3B3
:105938000B039A4204F10601A8BF1A4627F0ECFEB1
:10594800EDE7012289E7D8000C186468002C7FF481
:10595800F7AE17241470F3E63148FDF72DF8402010
:10596800FDF72AF820E72F48FDF726F82B6818E7F7
:105978002D48FDF721F82B6810E72C48FDF71CF897
:105988002B6808E79A8AB2F57A7FBFF4FAAE4FF42B
:105998007A729A82F5E618231370DAE643F0080360
:1059A8002B60F5E6F85D0308C05903082C3E00207B
:1059B8000C1D0308FC030308906C0020B065002050
:1059C800806F0020096000029C6C0020285F002086
:1059D800A06C0020DC6D0020326E002028240020FE
:1059E800303E002034340020C86C0020F63D0020F2
:1059F800286B0020506D0020DE1500205C2400205C
:105A080070220020C0C9FB48841E002017B7D13877
:105A180074220020A03100203661023D7C31002034
:105A2800094000020160000209200002086000022B
:105A380002F0030800000408583B002008B51CF0D9
:105A4800FFF8FCF7F7FF1CF0E3F8FFF745FE01202D
:105A5800BDE808401DF056BE2DE9F04F013085B075
:105A6800C3B203930B4602918B4C8C4E002B00F073
:105A780099808B4D8B4FDFF830921DF05FFF4FF40C
:105A8800FA7A4FF0100C4FF47A70D9F80430C3F357
:105A98000803002B40F0DE80EFF31183002B40F069
:105AA800D9802968A26800BF2B689942F9D1D7F834
:105AB80000E000FB0EF39B1AB3FBFEF300FB013181
:105AC8004FF0010E0191D9F80430C3F30803002BFD
:105AD80040F08780EFF31183002B40F082802B6821
:105AE800A16800BF2A689342F9D1D7F800B000FB3B
:105AF8000BF2521AB2FBFBF200FB0323019A9B1A2A
:105B0800B3F57A7FDFD3BAF1010ABED1039B002B2C
:105B180040F0BD804FF47A7ADFF88C9150464FF010
:105B2800100CD9F80430C3F30803002B75D1EFF338
:105B38001183002B71D12968A26800BF2B68994294
:105B4800F9D1D7F800E000FB0EF39B1AB3FBFEF384
:105B580000FB01314FF0010E0191D9F80430C3F375
:105B6800080313BBEFF31183FBB92B68A16800BFCF
:105B78002A689342F9D1D7F800B000FB0BF2521A09
:105B8800B2FBFBF200FB0323019A9B1AB3F57A7F61
:105B9800E3D3BAF1010AC4D1029B013B0293002B63
:105BA8007FF467AF05B0BDE8F08FEFF311888CF391
:105BB8001288A1682368DB0344BFC6F800E0A16827
:105BC8002B6832685FFA88F888F31188D7F8008064
:105BD8001A4400FB08F35B1AB3FBF8F300FB02332B
:105BE800D2E7EFF311888CF31288A1682368DB03EE
:105BF80044BFC6F800E0A1682B6832685FFA88F8ED
:105C080088F31188D7F800801A4400FB08F35B1A60
:105C1800B3FBF8F300FB023370E7EFF311828CF368
:105C28001288D4F808E02368D90303D50123336028
:105C3800D4F808E02B683168D2B282F311883A6848
:105C4800194400FB02F3A3EB0E03B3FBF2F300FBD2
:105C580001317FE7EFF311828CF31288D4F808E062
:105C68002368D90303D501233360D4F808E02B68EF
:105C78003168D2B282F311883A68194400FB02F302
:105C8800A3EB0E03B3FBF2F300FB013118E7184650
:105C98001FF040FB3EE700BF10E000E0A0610020DD
:105CA800A4610020A861002000ED00E02DE9F04F7C
:105CB8002DED028B93B0834619F0AAFFB54B1D78E2
:105CC80025B113B0BDEC028BBDE8F08FB24B1B6859
:105CD8005C05F6D5B14FB24E3B68002B56D0B14C9F
:105CE8003168D4F810218A1A7C2A4FD994F81421E3
:105CF800DFF8FC829FEDAC8AC4F81011013284F8F9
:105D080014214FF0240A5E20984750463B68984774
:105D1800A64BF8EC016A9B8A07EE103AF8EEE66AA1
:105D2800B8EEC77A0AF1010AC6EE877A5FFA8AFAEC
:105D380067EE887AFDEEE77ACDED027ABDF9089034
:105D48005FFA89F018F0D8F8C9F3072018F0D4F8EA
:105D5800BAF1270F3B68D6D15E2098473B683020C0
:105D68009847002018F0C8F8002018F0C5F83B68DC
:105D78005E20984794F8143113F0030800F08481EA
:105D8800580701F03682282B01F03283884B1B78A4
:105D9800002B72D0834C874AD4F81831ABEB03033D
:105DA800934200F27B8794F82091B9F1000F35D126
:105DB800DFF84082D8F80000FBF7DCFAC0B201280F
:105DC8000FD902287C4F41F0A5833B78002B41F086
:105DD8002A86D4F82431ABEB0303B3F57A6F81F04C
:105DE8009D87D4F82831002B47D094F82031C3B9C7
:105DF800724B1B689B7801211E3B00228B4284F862
:105E0800201184F8342141F22E87D8F800000221AD
:105E1800043017F0E7FF94F82C3111E0D4F828315A
:105E28005BB3D4F8303140F6B732ABEB030393429F
:105E380023D994F82C31002B01F0C382DFF8B48108
:105E4800013BDBB284F82C31002B00F08287D4F8B8
:105E5800287194F8342117F8011B94F83531D8F8D3
:105E68000000C4F828710A44013384F8342184F806
:105E78003531FBF783FAC4F830B1514BD6F80080BE
:105E88001B7843B14F4F386828B14F4B1B78013B03
:105E9800012B40F26E874D4B1B7863B14C4F3B682A
:105EA8004BB1404CD6F80090D4F84C31A9EB030321
:105EB800632B00F21C81DFF8408198F80030022B38
:105EC80001F05E823C4F97F87430032B00F02B876B
:105ED800404B1B7873B1404D2B685BB1314CFBF7DD
:105EE8004BF8D4F85831029044F61F62C31A934213
:105EF80000F25881394B1B78002B7FD1384B1B7827
:105F080043B1284CD4F8A83203F5C333A0339B45DA
:105F180080F07286334B1B78002B3FF4D2AE214EB3
:105F2800314C324D06F2C9272068FBF723FA0028C6
:105F38003FF4C7AE2068FBF715FA2B7880465A1E47
:105F480033B120682A70FBF715FA0028F2D1B8E6B9
:105F580003223946781E29F046FE96F8C83296F88C
:105F6800C92286F8CB8283F47F4383F0FF039B1A10
:105F78001FFA88F89BB2B8EB132FD5D196F8CA222E
:105F8800DBB29A42D0D1781E17F0AAFC2B781844BD
:105F98002870C9E7756C002004690020D4450020EA
:105FA800A4610020941E002000007A44C86C0020E0
:105FB800825500203F0D030024000020D04500201A
:105FC80084550020504300208C5500209455002013
:105FD800244F00209C550020A0550020E0550020AB
:105FE800F1550020A6550020AC550020B0550020E2
:105FF800006D0020CC4500203E5800205B4C2278E4
:10600800A2B15B4B9B7A53B1FAF7B6FF594B1B68A9
:10601800C31AA3F57A73B3F5FA6F07D82278564BEB
:1060280056491868FBF776F900232370544CD4F8C6
:10603800A03203F5C333A0339B45FFF45FAF514D46
:10604800C4F8A0B22B78002B41F030834E4D2B784A
:10605800002B41F01D824D4994F8A4228D5CE9077C
:1060680001F1E784AA0701F1A1846B0701F1998383
:10607800474A94F8A4321178013393FBF1F201FBFB
:10608800123384F8A43239E7D4F8102141F2883366
:106098009A4201F216823B685E2098473B681420BA
:1060A80098473C4B3C4AB3F9043082FB03124FEA51
:1060B800E378C8EBA2080FFA88F85FFA88F017F0BF
:1060C8001BFFC8F3072017F017FF3B685E209847AF
:1060D8003B681C209847002017F00EFF002017F09F
:1060E8000BFF3B685E20984794F8143148E6DFF8C8
:1060F800A4A0DFF8A480412017F024FEBAF90230EA
:1061080088FB0320DB17C3EBA00080B217F000FE6A
:10611800BAF9003088FB0320DB17C3EBA00080B27C
:1061280017F0F6FDBAF9043088FB0320DB17C3EB40
:10613800A00080B217F0ECFD184B38681978FBF70F
:106148001DF994F8503113F0010801F0F481144A54
:10615800C4F84C910133DBB2A2FB0312D20802EB64
:106168008202A3EB420384F85031A4E67455002060
:10617800446A0020B8370020E45500203455002038
:10618800941E0020E8550020E9550020EC55002019
:10619800F0550020206D002067666666A453002035
:1061A800CDCCCCCC94F85E31002B41F06C81DB4B2C
:1061B8001A6802F00803002B48F603414AF60B4020
:1061C8004BF60F4349F6074704BF03460F4612F044
:1061D800040F4FF0190118BF1F46920684F85E118C
:1061E80003D547F4804747F02007CD4B5A79C7F3CA
:1061F8000909002A41F0BF859B79002B41F0AA8646
:10620800984664204FF0FF3A4FF0000C0A970B971E
:10621800ADF834C0CDF83AC0CDF83EC0CDF842C094
:10622800CDF83090ADF83680ADF838A08DF846003E
:106238000AAF0FCFDFF800E384F805C0AEE80F001F
:1062480097E80F00AEE807002EF8023B71464FF0C2
:10625800010C1B0CFE271F20C82201F81E39A7704D
:10626800A27184F807C0E07094F86E01207180F084
:10627800F10383EA0313DAB2130983F0E70343EA6D
:10628800022383EAC2031BB283EA0312D2B2C3F326
:10629800072383EA121343EA022383EAC2031BB2E9
:1062A80083F0C80282EA0212D2B2C3F3072383EA58
:1062B800121343EA022383EAC2031BB283EA0C07E0
:1062C80087EA0717FFB2C3F3072282EA171242EAE6
:1062D800072200EB0C0382EAC7070EEB0C0084F8D8
:1062E8006E31278011F8013B7B4083EA0313DBB250
:1062F8001A0982EA172242EA032282EAC3031BB27E
:106308009FB281422780EDD183F07C0383EA031397
:10631800DBB24FEA131E8EEA172E8EEA032E8EEAA0
:10632800C30E0FFA8EFE1FFA8EFADFF810C2A4F819
:1063380000A05FFA8EFE4FEA1A2A84F828A084F893
:1063480027E00CF5CB7804F12209DCF80000DCF832
:106358000410DCF80820DCF80C3047460FC70CF1B5
:10636800100CCC45B846F0D1DCF8000038606D4F11
:106378009CF8043088F8043007F1270884F8BDE158
:1063880084F8BEA117F8011F2868FAF7F7FFB84587
:10639800F8D194F85F31002B41F07080624932687F
:1063A80009780A2084F85F01002901F0F0815F4F25
:1063B80001293888069041F2C1850229B7F802E020
:1063C80001F0F484B8880590032901F0CE85F88897
:1063D8000490042901F0DC850529388901F0D3856A
:1063E8000629B7F80A9001F0CA850729B7F80C8082
:1063F80001F0C285FB89039394F86E110A920B464B
:1064080083F0300282EA0212D2B217094849079390
:1064180087F07A0747EA02270988237187EAC202C8
:10642800444FC1EB012187FB013A069B4FF0000C5A
:1064380063F30F0C059B6EF31F4C4FF0000E63F3D4
:106448000F0E049BCDF82CC012B28A440027C9173E
:1064580063F31F4EC1EB6A2A039BCDF830E082EA52
:10646800021160F30F070020C9B268F30F00C2F3EE
:10647800072269F31F4782EA111263F31F404FF0A6
:1064880000090D978DF83DA00E908DF83C9042EADA
:1064980001220DF1280C82EAC107BCE80F003FB2C7
:1064A80087F0C80888EA0818DFF88CE084F80590B7
:1064B8005FFA88F8C7F30727AEE80F0087EA1817CE
:1064C80047EA08239CE8030083EAC8031BB283F069
:1064D80023024EF8040B82EA0212D2B2C3F3072356
:1064E800079F83EA1213704643EA022383EAC20233
:1064F80007F1010C20F814194FF023081621FE2784
:10650800C82384F86EC1228084F807800EF1020E39
:10651800A770E170A371114612E000BFC46C00209F
:10652800406D00202B200020286D0020D85200202C
:10653800EC540020030820809C1E0020961E00209A
:1065480010F8013B4B4083EA0313DBB21A0982EAD5
:10655800112242EA032282EAC3031BB299B27045B0
:106568002180EDD183F0F40383EA0313DBB24FEA11
:10657800131E8EEA112E8EEA032E8EEAC30E0FFA30
:106588008EFE1FFA8EF8E64FA4F800804FEA182C0A
:106598005FFA8EFE84F81EE084F81FC07968BA6836
:1065A8003868FB6807F5CB78A8E80F00386979697F
:1065B800BA6904F29717A8E8070004F2B51884F836
:1065C800B5C184F8B4E117F8011F2868FAF7D6FEB8
:1065D800B845F8D194F866C1BCF1000F40F048877F
:1065E800D04B94F86E71B3F90010B3F90220B3F9E7
:1065F80004309FEDCD6ADFF840E384F805C007EE6C
:10660800103A33680A9387F06A0383EA031306EEA5
:10661800901AD9B20B0983F0D50343EA012383EA20
:10662800C1031BB283EA03115242C9B207EE902A92
:10663800C3F3072383EA111343EA0123F8EEE77A49
:10664800F8EEE66AB8EEC77A83EAC1031BB267EED2
:10665800867A66EE866A27EE067A002083F0C808F6
:10666800CDED0C7ACDED0B6A8DED0D7A0E900F9075
:10667800109088EA08160DF12809F6B2C3F3072826
:10668800B9E80F0088EA161848EA062888EAC60812
:106698000FFA88F8AEE80F0088F01E0699E80700A0
:1066A80086EA0616F6B2C8F3072383EA161343EA06
:1066B80006238EE8070083EAC6061C20C8214FF08F
:1066C80005084FF01E0CFE237A1CE070A17184F8B7
:1066D800668184F807C0A370AEF1100127710EF12E
:1066E8000C00268084F86E2111F8013B734083EA80
:1066F8000313DBB21A0982EA162242EA032282EA6B
:10670800C3031BB29EB281422680EDD183F02703DA
:1067180083EA0313DBB24FEA131E8EEA162E8EEAC3
:10672800032E8EEAC30E0FFA8EFE1FFA8EFC7C4FE4
:10673800A4F800C05FFA8EFE4FEA1C2C84F825C02E
:1067480084F824E007F5CB7804F1220938687968E1
:10675800BA68FB6846460FC610374F45B046F5D1B4
:10676800724E3B88A8F8003006F1240784F8BAE195
:1067780084F8BBC116F8011F2868FAF7FFFDB74275
:10678800F8D194F867A1BAF1000F40F06B8694F83D
:106798006E81644B664AB3F90410B2F90620654E5F
:1067A800DFF898E1644F84F805A088F0220080EAB9
:1067B8000010C0B2030983F0590343EA002383EAB7
:1067C800C0031BB2B2F5FA6F83EA0310C0B2A8BFC8
:1067D8004FF4FA62C3F30723B2F57A7F83EA101302
:1067E80043EA0023B8BF4FF47A7283EAC000A2F5E7
:1067F8007A72642303FB02F28EFB023ED31786FBF8
:106808000162C9174FF0000CC3EBAE13C1EBA20134
:10681800CDF828C006B2CDF82CC0CDF830C0CDF8E0
:1068280034C0ADF83A30ADF838100DF1280CBCE89A
:106838000F0086F0C80E8EEA0E1E5FFA8EFEC6F3B3
:10684800072686EA1E1646EA0E260FC786EACE06F1
:1068580036B286F04A0383EA0313DBB2C6F3072194
:1068680081EA13113A46DCF800E042F810E941EAFF
:10687800032108F1010681EAC30305204A214FF0EC
:10688800FE0C84F86E614FF0C80E142684F8670178
:1068980084F8048023800437E17184F802C0E6702C
:1068A80084F806E0184612F8011B414081EA0111FC
:1068B800C9B20B0983EA102343EA012383EAC10121
:1068C80009B288B2BA422080EDD181F0140181EA80
:1068D8000111C9B24FEA111E8EEA102E8EEA012E5E
:1068E8008EEAC10E0FFA8EFE1FFA8EF60C4F268026
:1068F8004FEA16295FFA8EFE84F81D9084F81CE092
:1069080079683868BA68FB68B7F8188007F5CB7CEF
:10691800ACE80F0038697969ACE8030010E000BF03
:10692800961E0020206D002088C3E43A2B2000200A
:10693800D8520020676666669C1E0020D34D621000
:1069480004F29716ACF8008084F8B391B04684F846
:10695800B2E104F2B31918F8011F2868FAF70EFD1E
:10696800C145F8D1C44BC54A1B781278013B12F0D7
:106978000100DBB214BFC0214021172B03D8C04A45
:10698800134493F830A0BF4B1A8893071ABF00230B
:1069980041F01001012312F4027F18BF022312F004
:1069A800100F18BF062312F0200F18BF102300285D
:1069B80041F08C814FF0030C94F86E910A9389F0A2
:1069C800460383EA0313DAB2130983F0920343EA16
:1069D800022383EAC2031BB283EA0310C0B2C3F3E3
:1069E800072282EA101242EA002282EAC00212B2A8
:1069F80082F0C80E8EEA0E1E5FFA8EFEC2F30722E0
:106A0800002382EA1E1203208DF82CA08DF82FC0D7
:106A18008DF82D3042EA0E2C8DF82E108DF83000AE
:106A28000AAA07CA8CEACE0E0FFA8EFEDFF868A211
:106A3800E3718EEA0E1CAAE803005FFA8CFCCEF321
:106A4800072E8EEA1C1E4EEA0C2181EACC0C94F823
:106A580008E08AF800200FFA8CFC8EEA0C0E8EEA09
:106A68000E1E5FFA8EFECCF3072282EA1E1242EA5D
:106A78000E22607AA17A94F80BC0637182EACE0282
:106A880012B2504080EA001E5FFA8EFEC2F3072061
:106A980080EA1E1040EA0E2080EACE0000B2414093
:106AA80081EA0111C9B2C0F3072282EA111242EA4F
:106AB800012282EAC10212B28CEA020C8CEA0C1C96
:106AC8005FFA8CFCC2F3072282EA1C1242EA0C220B
:106AD80094F80CE0607BA17B94F8108084F8049013
:106AE80082EACC0212B28EEA020E8EEA0E1E5FFA1B
:106AF8008EFEC2F3072282EA1E1242EA0E2282EAC0
:106B0800CE0212B2504080EA0010C0B2C2F307228F
:106B180082EA101242EA002282EAC00212B251400E
:106B280081EA0111C9B2C2F3072282EA111242EACC
:106B3800012282EAC102E17B13B281EA030282EAFE
:106B48000212D2B2C3F3072383EA121343EA0223E1
:106B580083EAC2031BB288EA030282EA0212D2B2B3
:106B6800C3F3072383EA121343EA022383EAC20327
:106B78001BB283F0320282EA0212D2B2C3F30723B5
:106B880083EA121343EA022383EAC2031BB29AB2CE
:106B98004FF0FE0C4FF0090EC82009F10101DBB2DD
:106BA80084F802C084F803E04FEA122CA07184F83C
:106BB8006E11228084F812C0637438687968BA68E4
:106BC800B7F80C900AF5C47EAEE807000AF5CC7A4F
:106BD8008EF80280AEF8009084F8A8C184F8A73136
:106BE80016F8011F2868FAF7C9FBB245F8D1029BCD
:106BF800C4F85831FFF77EB994F8AC32204AC4F88B
:106C0800A8B202EB8302926C42B312AD04F2B32332
:106C18001D4E45F8203D002104F2C52331800B9319
:106C280080211523A52784F8B232284684F8B112AA
:106C380084F8B072904728463188FCF745F90A9DD8
:106C4800124804F52C716D1A152DA8BF15252A4672
:106C580026F062FD0E4A94F8AC3215700D4A0133E5
:106C680082FB0312A2EBE37202EB42029B1A84F846
:106C7800AC32FFF74FB900BF2C3E0020FC6B002060
:106C880040FF0208EE540020A85300207836002068
:106C98008D360020565555559C1E0020D34AD44B9E
:106CA80092F80BE03168D4F81C211B88D148891A66
:106CB8004FF47A72DFB202FB0EF21B0A8777077570
:106CC80091424FF00007C37743758770077180F0D2
:106CD8001284C94BC9491A689B68C4F818B181FB6A
:106CE80002E7D21781FB03E1C2EBA702DB17C3EB74
:106CF800A10311124FEA232C4FF0F40E027701275B
:106D0800417780F8203030217522782380F821C01F
:106D180080F81AE0C77680F8221080F8232080F8DF
:106D28002430FFF740B8DFF8F492D9F80000FAF7FA
:106D380015FB00283FF4CCA8D9F800000121FAF788
:106D480009FB0222002387F8742088F80030FFF737
:106D5800BFB894F8341194F83531D8F800004A1CBB
:106D6800013384F8342184F83531FAF707FBFFF74B
:106D780082B8A34CDFF8A8924FF0000A0AE01B2B58
:106D880000F014830D2B00F012824FF0010389F8F4
:106D980001303868FAF7EEFA002838D03868FAF780
:106DA800E1FA83B27E2B32682AD099F801100029C3
:106DB800EFD194F83621002AE1D07D2B00F00C8227
:106DC80094F844E1BEF1000F04D080F02003DBB258
:106DD80084F84411511CC9B22244092984F8361197
:106DE80082F8383100F0EC810829D2D8B4F8422171
:106DF800134403EB132303F0FF03A4F84231C8E75D
:106E080084F836A184F837A189F801A0C1E794F87D
:106E1800453133B194F8393184F84501302B00F00D
:106E2800498794F83721774BDFF8F8C1DFF8F8E1A4
:106E3800DFF8F8A10127104600283FF42CA8326893
:106E4800A2EB0802012A00F2AD8194F84691B9F14B
:106E5800000F40F0C28294F8471133F8112012B99C
:106E680084F84771E8E70131B2F5826F84F8471179
:106E780000F002811FD9B2F5E26F00F09A8034D990
:106E8800B2F5046F00F0A480B2F5116F00F04781ED
:106E9800B2F5E46FD0D110465B4A176C918A64232F
:106EA80003FB07F393FBF1F116F082FF002384F84C
:106EB8003731FEF7F0BFB2F5007F00F0B9802CD86B
:106EC800B2F5807F00F04581B2F5887FB4D1DCF857
:106ED80000205207B0D500214FF4887016F068FFE3
:106EE800002384F83731FEF7D6BFB2F5C06F00F043
:106EF800B380B2F5E06F9FD1434A906B918A6423C7
:106F080003FB00F34FF4E06093FBF1F116F050FF40
:106F1800002384F83731FEF7BEBFB2F5047F00F0D6
:106F28002781B2F5806F87D194F848310133DBB2FD
:106F3800032B00F2588142F2107184F8483101FBAA
:106F480003F1324B1B88002B40F04B810131304B51
:106F58001B78DF072F4B1B8848BF0431D80748BF71
:106F68000A319A0748BF14311F0648BF2831D8058F
:106F780048BF28315A0748BF64311F0748BFC83186
:106F8800980548BF01F5C8719A0648BF01F57A719E
:106F9800DF0648BF01F5FA61580648BF01F57A6176
:106FA8004FF4806016F004FF002384F83731FEF7B1
:106FB80072BF1046144AD76B918A642303FB07F308
:106FC80093FBF1F116F0F4FE84F83791FEF763BFF6
:106FD800114BB3F9041001EB81011046490016F07A
:106FE800E7FE84F83791FEF756BF00BF0044002043
:106FF800F8430020B4550020AC530020676666664D
:10700800941E002040FF0208C86C0020746D002008
:10701800FC6B0020EE540020206D0020CC5800208E
:1070280024000020C46C0020406D00200E44002085
:107038009EF8061000293FF4FFAEC44BC4491B68F4
:10704800104681FB0321DB17C3EBA10116F0B0FE4C
:1070580084F83791FEF71FBF9EF80620002A3FF4F8
:10706800EBAEBA4B4FF4C060996816F0A1FE00234E
:1070780084F83731FEF70FBFDCF8002012F0200942
:107088007FF4DAAEB34A1168090600F1F585B24A11
:10709800127B002A3FF4D0AE94F84911032900F27C
:1070A8009486DFE801F032281902AC4B1B68597945
:1070B8009A79DB7901F1407101EB022101EB03417F
:1070C800002384F849314FF4826016F071FE0023E2
:1070D80084F83731FEF7DFBEA14B1A68137A50796E
:1070E80092781B0403EB002313444A1C84F84921BB
:1070F80003EB0161E7E79A4B1A68D3791079527864
:107108001B0403EB00231344EFE7954B1A689379AC
:10711800D07812781B0403EB00231344E5E79EF8AC
:107128000520002A3FF488AE9AF8001000293FF4A1
:1071380083AE8C4B1B8803EB83035B004FF4116019
:1071480093FBF1F116F034FE002384F83731FEF793
:10715800A2BEDCF8002051077FF56EAE00214FF487
:10716800807016F025FE002384F83731FEF793BEB1
:107178009EF80520002A3FF45FAE9AF80010002917
:107188003FF45AAE744B5B7B002B00F09B85754B2C
:107198001B8893FBF1F101EB810149004FF4047066
:1071A80016F006FE002384F83731FEF774BE4FF060
:1071B800010184F8361184F83831A4F84221E8E551
:1071C800B4F84221C2F1FF0293427FF4DEAD4FF0E2
:1071D800010384F84531D8E54FF0010384F84431C0
:1071E800D7E50231B3E6012384F8483142F2107141
:1071F800A7E63B685E2098473B68022098475A4BB1
:10720800534AB3F9503082FB03124FEAE378C8EBD4
:10721800A2080FFA88F85FFA88F016F06DFEC8F336
:10722800072016F069FE3B685E2098473B680320FC
:1072380098474E4B1B78D90740F1318124F0E2F989
:107248004B4B9FED4C7AD3ED037A67EE877AFCEED1
:10725800E77ACDED027ABDF80830002800F02285E3
:10726800D8B24FEA132816F047FE404616F044FEFF
:10727800DFF8088198F80530002B40F0C4820AA98D
:107288003D4816F0FDFD3B685E2098473B6813209B
:107298009847BDF928805FFA88F016F02DFEC8F3EC
:1072A800072016F029FE3B685E2098473B681B20A4
:1072B8009847BDF92A805FFA88F016F01DFEC8F3DA
:1072C800072016F019FE3B685E2098473B6823208C
:1072D80098474E2016F010FE002016F00DFE0AA961
:1072E800254816F0CDFD3B685E2098473B68122084
:1072F8009847BDF928805FFA88F016F0FDFDC8F3BD
:10730800072016F0F9FD3B685E2098473B681A2075
:107318009847BDF92A805FFA88F016F0EDFDC8F3AA
:10732800072016F0E9FD3B685E2098473B6822205D
:107338009847452016F0E0FD002016F0DDFD3B687B
:107348005E20984794F81431FEF71DBDAC53002019
:10735800676666660469002000440020DC6D002032
:107368009C6C0020F843002000620020FC6B002089
:1073780010440020CDCC4C3E80969800406D0020F3
:10738800F9F7FAFDB54B1B68C01A40F6B8339842B6
:1073980000F2C680DFF804A39AF804303A2B00F014
:1073A8009283002388F80030FEF792BD3868F9F719
:1073B800E1FF00287FF4E9AC4FF0010384F837318E
:1073C800E7E4C4F8283184F82031DFF8D48216F0D5
:1073D8003DFD94F82C31FEF733BDA149062016F087
:1073E80009FB002384F8460184F83731FEF753BDC2
:1073F8004FF000093B6884F814915E203468DFF888
:10740800A48298473B6817209847484616F074FDB1
:10741800944BA3FB04239B0BA8FB03125209C2EB5A
:107428000212A3EB8203D8B216F066FD3B685E2019
:1074380098473B68182098478B4BA3FB04239B096C
:10744800A8FB03125209C2EB0212A3EB8203D8B2C3
:1074580016F052FD484616F04FFD3B685E209847EF
:10746800FEF794BC0AF1FF3A84F867A1FFF7BFBBA7
:107478000CF1FF3C84F866C1FFF783B9013B84F83F
:107488005F31FFF7A7B8013B84F85E31FEF781BF93
:1074980076493A2016F0AEFA2870FEF72FBDDFF8CD
:1074A8000882734BB8F80890A3FB09394FEA990989
:1074B8005FFA89F016F020FD4FEA192016F01CFD3E
:1074C800D8E63B685E2098473B68102098474046BE
:1074D80016F012FD404616F00FFD3B685E209847F7
:1074E8003B6821209847404616F006FD404616F0B6
:1074F80003FDFEF7D0BD5F4B32681B78C4F81C2132
:10750800013B012B3FF6E5AB102202238270037189
:10751800FFF7DFBB16F08AFC01233B70FEF761BC66
:10752800554AB2F8523100210133A2F8523188F895
:107538000010FEF7CDBC514B1B88DA0515D4D806D0
:1075480000F13084990600F13C845A0600F1488421
:10755800180700F15284D90700F1EC8413F0020FE8
:107568000CBF4FF004084FF00C08454B454A1B78F8
:10757800D27803F001030AB143F0020353200293C7
:1075880016F0E0FB404A128802EB820202EB82020C
:10759800900080B216F0BCFB002016F0B9FB3B4A05
:1075A8003B4912883868C2EBC212520081FB023193
:1075B80011444FEAE27ACAEB612A5FFA8AFA514625
:1075C800F9F7DCFE334B38681A78029B48EA03085F
:1075D800304B8AEA020A002183F800A0F9F7CEFEB0
:1075E80041463868F9F7CAFE2A4B2A4A1B78386898
:1075F80088EA0303DBB219461370F9F7BFFE94F863
:107608005031002B7EF4A3AD4F2016F09BFB17F0F2
:1076180035FB17F033FB17F031FB01213868F9F718
:10762800ADFE1D4A1B4B92F800801B78194A38683A
:1076380008F0010883F0010341461370F9F79EFE34
:10764800144B144A1B78386888EA030319461370E8
:10765800F9F794FE94F85031FEF779BD44580020AC
:10766800B3DD010873B2E745D34D621099FB0108F9
:10767800CDCCCCCCF2540020941E0020EE54002037
:10768800FC6B0020506D0020F8430020EC540020D3
:1076980003082080A4530020403C00202C580020E0
:1076A800CC45002089888888406D0020AE4EAF4BBD
:1076B80000930024A6F13F01AD4BAE4A089106F8AD
:1076C800404CAD4909960AA8FBF7D6FC089E731CE6
:1076D80008933470089B2922591C08911A70089B3A
:1076E800EA22591C08911A70089BC822591C089153
:1076F8000AA81A7025F03CFA471C0AA93A460898C5
:1077080026F00AF8089AD31901330893D455089B30
:107718005A1C08921C70089B5A1C08921C70089BE3
:107728005A1C08921C70089B5A1C08921C70089BD3
:107738005A1C08921C70089B5A1C08921C70089BC3
:107748005A1C08921C70089B5A1C08921C70089BB3
:107758005A1C08921C70089B5A1C08921C70089BA3
:107768005A1C08921C70089BFF22591C08911A7019
:10777800089B0122991812A808911A7050F8283D00
:107788009B1B337018F0D4F92C70FEF7B7BB8846F2
:1077980089460846049105918E4606910391FEF7A5
:1077A8002BBE764A704B12680B93A3F1400500205C
:1077B8002121D70003F8400CA97040F1D08270490C
:1077C8000326704B1B88580500F1C682DA0700F1C2
:1077D800F58203F002036C4A002B1CBF03261146F6
:1077E8006A4F3246384625F097FFF31912A801333D
:1077F800B91E40F8203D00225B1AF2556B7018F054
:1078080097F9FEF735BC624B93F800A0BAF1000F68
:107818003FF435AD5F4AB4F816E111883B6802922F
:107828004FEA0E1E64201FFA8EFE00FB01A14FEAEC
:107838004A00B1FBF0F14EEA012E1FFA8EFEC1F3A9
:1078480003215E204EEA010998473B6806209847C5
:107858005FFA89F016F050FB4FEA192016F04CFB3E
:10786800B4F81631029A4C49B2F800904A7A0133BA
:107878009BB2012A93FBFAF00AFB1033A4F81631E5
:1078880000F049836E2345484A7B03FB09F380FBDC
:1078980003014FEAE379C9EBA1092AB13C4B1FFA6E
:1078A80089F91B7899FBF3F93B68DFF8FCA05E20A7
:1078B80098471FFA89F93B683A209847AAFB093A82
:1078C8004FEA5A1A1FFA8AF3D8B2029316F014FB39
:1078D800029B180A16F010FB3B685E2098473B682D
:1078E8003B209847642303FB1A939BB22C4805332B
:1078F80080FB0320DB17C3EBA000C0B216F0FCFA34
:10790800002016F0F9FA3B68DFF898A0DFF89090AD
:107918005E2098473B6828209847DAF8003089FBB2
:107928000329DB17C3EBA9095FFA89F016F0E4FA1B
:10793800C9F3072016F0E0FA3B685E2098473B68D9
:1079480004209847B8F80830002B40F04D82DAF848
:10795800083083F310085FFA88F016F0CDFAC8F300
:10796800072016F0C9FA8AE434550020956C0020E7
:10797800002703080827030814270308383C0020B9
:10798800E4260308EE540020FC260308F7540020E0
:107998000E440020F843002000440020310CC3307E
:1079A80067666666AC5300201F85EB51CC4ACD4B09
:1079B8000B9212AEA2F13D0046F8200D1988CA4F6D
:1079C800A2F1400300204FF00A0E02F8400C0822F2
:1079D80083F801E030469A70FBF750FA3B68C349D8
:1079E800DA1781FB0313C2EBA30399B23046FBF706
:1079F80045FA09F005F9BF680A9B3A0C591C0A9127
:107A08001A700A9B3A0A591C0A911A700A9B5A1C46
:107A18000A921F700A9B5A1C0A921870304618F076
:107A280087F8FEF722BBC4F824B187F80090FEF768
:107A3800D8B9AF4F9FEDAF8AB7F90220A8480B908D
:107A480007EE902AF8EEE77A12AE67EE887AA0F190
:107A58003D01FDEEE77A46F8201D00F8403C08237A
:107A6800CDED027A00F83F3C1E23BDF8081000F85F
:107A78003E3C3046FBF702FAB7F9003007EE903A81
:107A8800F8EEE77A304667EE887AFDEEE77ACDEDD4
:107A9800027ABDF80810FBF7F1F9B7F9043007EEE0
:107AA800903AF8EEE77A304667EE887AFDEEE77AA4
:107AB800CDED027ABDF80810FBF7E0F9304618F072
:107AC80037F8FEF7CFBA9AF80240C4B1013CE4B2E5
:107AD800013454445146002211F8013B534083EAD3
:107AE8000313DBB2120ADF0042EA03228C4287EA60
:107AF800131382EA0302EFD1002A7FF452AC794AC9
:107B08007D4F794B12887D4CFA61DFF808921A682C
:107B1800FA629B68B4F85221F8660021FB64D9F830
:107B28000000F963FA65F8F7E7FB029000287EF495
:107B3800CAA90221D9F80000F9F70CFC94F85431CD
:107B48009AF803200392642B4FF0040287F87420FC
:107B580040F0578194F85531072B04BF9DF8083041
:107B680084F8553194F85531069307EB031ADAF87F
:107B780004100291084624F0FBFFDAF8081005917A
:107B88005FFA80FA084624F0F3FFC0B204900AEBCB
:107B98000002069B5A48029902900832C27123F0EB
:107BA8000F0286468272049803F00F0300EBCA00A6
:107BB8008EF80D3052468EF80E000EF10F0025F0AB
:107BC800ABFD504B049A05990AF10900184425F0B9
:107BD800A3FD0298C37903F1010ACBB1013B5FFA17
:107BE80083FC0CF1080CDFF830E1844400230730F3
:107BF80010F8011B59408B00CA0883EA410302F0C0
:107C080018024B404EFA02F253408445DBB2EFD1E2
:107C18003C4A03980AF8023016F0FEFF94F85531F2
:107C28000022013384F8553184F85421029BDDF891
:107C380008A09B785BB11AF80510D9F80000F9F78D
:107C48009DFB01359AF80230EDB2AB42F3D894F8B7
:107C580054310322013384F8543187F8742088F8AA
:107C68000020FFF762B80221D8F80000F9F772FB8C
:107C780094F82C31FEF7E4B81023042218460AA918
:107C88008DF82A908DF82B908DF82C908DF82D90EA
:107C98008DF828308DF8292016F06CF884F8379183
:107CA800FEF7F9B8184A1268D2067FF5D9AA8046B5
:107CB800FFF7D9BA1549881F15F040FF84F8460127
:107CC800FFF7AFB8074B1988FFF765BA104AD278A3
:107CD800002A0CBF4FF0040C4FF0050CFEF76CBEE9
:107CE80034550020F8430020AC53002067666666D0
:107CF800206D002058A08B4124000020941E0020F5
:107D0800FC4E0020024F002004690020D41F0020F0
:107D1800506D0020CC5800200007090E0123D8F828
:107D280000003B70F9F71EFB0746D8F80000F9F78A
:107D380019FB7F067EF455A88E287EF452A894F885
:107D48002031002B7EF46AA8944BC4F828312D23E7
:107D580084F82C31FEF74CB80326914940E5914B45
:107D6800914A1B68914903F4800383420ABF114674
:107D78000326042625E58E499A790B8803EB8303AD
:107D880003EB83034FEA83081FFA88F8002A00F000
:107D9800DE80884B1B680FFA83FA08F031FF40B287
:107DA800FEF732BA4FF03408FFF7DFBB9846994622
:107DB8001846049305930393FEF71EBB7E490426D9
:107DC8000EE54FF02408FFF7D0BB4B1CDBB2042BA9
:107DD80084F849314FEA01617FF475A9FFF770B95A
:107DE8004FF01008FFF7C1BB08F00AFF16F084F83F
:107DF800002016F081F8FFF742BA4FF02008FFF78D
:107E0800B4BB97F875A06D4904951AF00F0F04BF1D
:107E18000AF1010A5FFA8AFABAF1070F28BF4FF090
:107E2800010A4FEA0A1C07EB0C03187C644B029307
:107E38000A18002392F82410614A93725FFA8CF3AF
:107E48001A46604B964607EB0C024EEA00000129E1
:107E58001870D26803F101000CD90239C9B28D1C1F
:107E68001D44034603F8012BAB424FEA1222F9D115
:107E780001310844BC4422F060030AF1010A9CF86D
:107E880011205FFA8AFA1343BAF1080F037000F160
:107E9800010366D04FEA0A1C07EB0C01494A087C2B
:107EA800464901449A1A91F8241055180EF1100EFB
:107EB800132D5FFA8EFEC6DD049D0298DFF80CE1F3
:107EC800D1B28B1DDBB243F04002C27103F1010C49
:107ED800CBB14B1DDBB20833C31804930EF101007C
:107EE800002310F8011B59408B0083EA4103CA089C
:107EF8004B40354902F0180241FA02F25340049A05
:107F08008242DBB2EDD103980CF80E3087F875A0E9
:107F180016F082FE8AE63B685E2098473B68392067
:107F280098475FFA89F015F0E7FF4FEA192015F036
:107F3800E3FFE8E44FF00808FFF717BB98469946B7
:107F48001846049305939E460393FEF755BA4FF0DF
:107F5800FF3320E7174B9046B3F900A06420FEF7E3
:107F680053B9184A049D9A1AA7E79846994618469D
:107F780004930393FEF740BA0393FEF73DBA98467D
:107F88000393FEF739BA984699460393FEF734BA35
:107F98009846994618460393FEF72EBAB455002022
:107FA800F026030804690020E8260308E4260308ED
:107FB800F8430020AC530020F426030840FF0208D1
:107FC800FC4E0020094F00200007090E024F002038
:107FD8002DE9F04F2DED0C8B3C4B1B7895B0012B08
:107FE800099001F073863A4C94F80021002A41F078
:107FF800C180072B374D01F06486002305936B6819
:1080080034489847002800F06981B5F8B470002218
:1080180085F85520002F40F04387B5F93E00AA6A3D
:10802800B5F93C60696AB5F94030DFF8B4B0821A36
:10803800E86A6A63711A1B1A2963274895F856106B
:10804800AB6311F057F9DBF80030990040F1F0808C
:10805800D5ED0D5AD5ED0C7A204A94ED656AD4ED2C
:10806800666A94ED677AD4F8A0311268B8EEE58AAA
:10807800D5ED0E5AF8EEE77AF8EEE58A013377EE99
:10808800867A38EE268A78EE878A9342C4ED657A36
:1080980084ED668AC4ED678AC4F8A03101F0D683FE
:1080A8000A4B1F78142F02F07B870023D4F8A861AD
:1080B8000693062E00F2AF80DFE816F02E16F316B0
:1080C800D314071714009E15371500BFE843002086
:1080D8006021002000620020306200200438002067
:1080E80004690020D84B1A78D4F8ACE1DFF8D0C383
:1080F8009FEDD67A4FEACE000CEB000383ED007AB1
:10810800002A7DD0D249B0EE476AF0EE476A0023D4
:10811800F1EC017A013367EEA77A05EE903AB4EEF6
:10812800E77AF1EE10FAF8EEE55AB8BFB0EE677AE2
:10813800934276EEA76AA7EEA56AE9D1F5EEC06A82
:108148000CEB0003F1EE10FA83ED007A58DDC6EE71
:10815800265AC04BC04A1288F7EE007A75EEE75AE5
:10816800D3ED007A65EEA77AFDEEE77A17EE903A3E
:10817800812B43F365859342A8BF134607EE903AD7
:10818800F8EEE77AB54B00EB0E0103EB810393EDB4
:10819800057AD3ED003A93ED066A93ED014AD3EDE3
:1081A800046AD3ED034A93ED025AA3EEA77AA4EE2C
:1081B800276A66EEC76AA7EE646ABDEEC77AE5EE7F
:1081C800276A17EE101A812983ED056AC3ED066A3E
:1081D80043F333858A42A8BF0A4607EE902AF8EE91
:1081E800E77AFCEEE77ACDED077ABDF81C300CEBA8
:1081F80000029380BEF1000F02D1132F04F080819A
:10820800152F42F083846044DFF8B882838828F809
:108218001E30D4F8A861924B013683FB06239A19C5
:10822800F317C3EBA203C3EBC303F61AC4F8A861A0
:108238008C4B1B78002B01F0A8808B4EDFF88892BE
:10824800DFF880A206F5BC780027884BD5ED087AC0
:108258001B78172B01F08E8396ED007AB8EEC78A4B
:10826800082B28EE278A07D1B0EE480A069325F096
:10827800C7FB069B2AF81700DBF8002092000BD5F5
:10828800002F04F06384B0EE480AD5F8143208F1E0
:1082980070009847B0EE408AB0EE480AD5F83431FD
:1082A800A8F170009847D5F8A431404698476F4B1D
:1082B8001B78032BB0EE408A01F06983D6F8F800EA
:1082C800D5F8B830B0EE480A98470137032F08F1BF
:1082D8002408A9EC010A06F10406B6D1634B93F809
:1082E8000090B9F1070F00F0988694F8B831002B88
:1082F80040F0A0865E4B5B79002B40F0CB850123D4
:108308005A4A84F8B8311278072A02F08380002389
:108318000B93584B94ED709A93ED007A564BD4ED2D
:108328006FCAD3F800A0554B0693F7EE007A37EEE4
:10833800C9CA534B08932CEE07CA524B0A93B4EEA2
:10834800E7CA514B07930025F1EE10FA4F4BDFF8BF
:108358007C91DFF87CB1DFED4E8A9FED4EAADFED10
:108368003BBADFED4D9A9FED4DBADFED4DAADFF830
:1083780064814C4F059388BFB0EE67CA2E464A4BBE
:1083880099ED008A2B44D3ED007AF5EE407AF1EEB0
:1083980010FA17D0454B2B44D3ED006A38EE667AB5
:1083A800B0EEC76AF4EEC67AF1EE10FA08D5B5EE6B
:1083B800C07AF1EE10FACCBF37EEA68A36EEE78A1D
:1083C80083ED008A069B1A88930700F08580022EA9
:1083D80000F082809AF82E10354B07EE901A2B4445
:1083E80093ED007A4B42F8EEE76A07EE903A26EEF4
:1083F800877AF8EEE77AB4EEE77AF1EE10FA0AD463
:1084080007EE901AF8EE677AF4EEC77AF1EE10FAF2
:1084180088BFF0EE477A274B274903EB460331F92B
:108428001600B3F90C30C01A07EE100AB8EEC77A76
:10843800D007E7EE687A40F10586204B93ED008A75
:1084480027EE888A48E000BF0A38002000000000B4
:10845800602100200C38002008380020403A002015
:10846800932449920138002030620020E84300201C
:10847800E0680020403300209C6C0020EE5400206F
:108488009C000020FC6B0020F4680020D43B0020F6
:10849800CDCCCC3DAE47813F0000C84200003443FC
:1084A800610BB63BE03B002034330020242300203E
:1084B800CC220020F03D0020206D00201C3300203D
:1084C800283A0020EC430020F868002064220020AD
:1084D800AC2F0020EC3B0020079B94F8D0212B44C4
:1084E800D3ED01DA38EE6DDA002A3DD0D24BD4F85C
:1084F800D42109991B688A1A9A4235DD9AF84830BE
:10850800022B01F0FD87022E04F07F82CB4B1B6803
:10851800990740F12187CA4BCA49DFF890E331F93E
:1085280016C09EED008ADFF888E3C7ED00BA03EBBA
:10853800460028EE288AB0F90C00A0EB0C0007EEE4
:10854800900AF8EEE77ADEF8000027EE888A904273
:1085580038EE6DDAC1F22C81F7EE007AB4EEE79AC4
:10856800F1EE10FA01F1FB80B74B2B4493ED000AB2
:10857800059B2CEE800A022E20EE0D0AA3EC010AC0
:10858800059304F00982089BDBED007A93ED007AED
:10859800AE4BD7ED006A93ED006AAD4B67EE277AD4
:1085A8002B4427EE8C7AD3ED007A67EE277AF0EE2B
:1085B800665AE7EE8D5AB1EE467AB4EEE57AF1EEF8
:1085C80010FA08DCB4EEE56AF1EE10FA8CBFB0EEF2
:1085D800657AB0EE467A94ED706AF7EE007AB4EEFA
:1085E800E76AF1EE10FAACBF0123002343B1F0EEC5
:1085F800E66AF0EEC77AF4EEE67AF1EE10FA01D503
:1086080087ED007A022E04F09281924A924B52F83A
:1086180026001B68B0EE6D0A9847904A904B52F8B6
:1086280026001B6898479AF8373023B1069B1B88A9
:10863800002B00F06B85B0EE6B8A8A4B9BED007ABD
:1086480038EE400A2B4493ED008A83ED000A9AF82D
:10865800483030EE480AC0EE077A2BB30A9B1B78E5
:10866800DB0721D5B7EE007AB4EEC79AF1EE10FA1F
:1086780004DB94F8D031002B00F05B87D4F8D431B8
:10868800099AD31A6C4A12689A420DDD764B93ED1B
:10869800007AB0EECDDAB4EEC7DAF1EE10FA41F1B5
:1086A800A380002384F8D031704B94F8E0212B4448
:1086B80093ED007A2CEE877A67EE277AC8ED007A78
:1086C80032B9059BC7ED00BA43ED01BAC8ED00BA4F
:1086D8000136032E09F1040908F1040807F104071B
:1086E80005F104057FF44BAE614B1B78072B01F0B5
:1086F8000B83012B01F07B86002794F8E831002BCF
:1087080040F0F4855B4A5C4B10681B6810F4805A93
:1087180093F82C3040F06386584A594992ED006A24
:10872800498B584A84ED7E6A92ED007A564A84ED68
:108738007F7A07EE901AF8EEE76AD2ED037A534A89
:1087480084ED7C6A37EE467A77EEE67AD2ED006AF7
:1087580084ED7B7A012284F80022C7EEA65A4C49A0
:108768004C4A91ED005A4C499FED4C6A91ED004AF4
:108778004B49DFED4C6AD1ED004A92ED007A35EEB7
:10878800045AF7EE007AF4EEE75A35EE245AF1EE81
:1087980010FA88BFF0EE675A25EE065AF4EEE65A4C
:1087A800B1EE476AF1EE10FAB4EEC65AB8BFF0EE71
:1087B800665AF1EE10FAC4ED815A01F1D480B4EE94
:1087C800C75AF1EE10FA88BFB0EE475A304ADFEDCB
:1087D800336AD2ED017A304A92ED014A304A77EE97
:1087E800847AD2ED014A77EEA47A67EEA67AB4EEDF
:1087F800E76AF1EE10FA08DCB4EEE77AF1EE10FA67
:108808008CBFB0EE676AB0EE476A214ADFED236A93
:10881800D2ED027A204AD2ED024A234A77EEA47AB0
:1088280092ED007A67EEA67AB1EE473AF4EEC37A93
:10883800F1EE10FA47D43DE048330020C46C002024
:10884800F03D0020206D0020F0320020643300202D
:10885800FC320020B42F0020B02F00200830002068
:10886800043000203823002054330020083300202F
:10887800E8430020046900209C6C00205C3C002038
:10888800446A0020C03D0020104400202434002009
:10889800D43B002068330020E03B00206F12833A6D
:1088A800EC3B0020000000006C3300201C3300204B
:1088B80044330020F4EEC77AF1EE10FA8CBFB0EE24
:1088C800473AB0EE673AF04A52780AB9B1EE433AFD
:1088D800002B41F06883F7EE003AEC4D2A78002A25
:1088E80002F0A486EA4BDFEDEB7AD3ED024AD3ED32
:1088F800016A93ED037A66EE244AE5EE264AE3EE32
:10890800074A63EEA44AF4EEE74AF1EE10FAB4BF60
:10891800B0EE674AB0EE644A98BFF0EE647A012A76
:10892800CDED0C4A02F0A78693ED067AD3ED052A21
:10893800D3ED076A26EE077AA5EE227AA3EE267A09
:1089480023EE877AB4EEE77AF1EE10FAB4EEC47A41
:108958008CBFF0EE676AF0EE476AF1EE10FA88BF56
:10896800F0EE676AB4BFF0EE447AF0EE477A022A76
:108978008DED0D7A00F0DE8093ED0A7AD3ED092AA9
:1089880093ED0B4A26EE077AA5EE227AA3EE047A37
:1089980023EE877AB4EEE67AF1EE10FAB4EEE77ACF
:1089A8008CBFB0EE664AB0EE474AF1EE10FA98BFB7
:1089B800F0EE446AA8BFF0EE477A032A8DED0E7AEE
:1089C80000F0B88093ED0E7AD3ED0D2A93ED0F4A9F
:1089D80026EE077AA5EE227AA3EE047A23EE877AAA
:1089E800B4EEE67AF1EE10FAB4EEE77A8CBFB0EEA8
:1089F800664AB0EE474AF1EE10FA98BFF0EE446AC4
:108A0800A8BFF0EE477A042A8DED0F7A00F0928025
:108A180093ED124AD3ED112A93ED137A26EE044A08
:108A2800A5EE224AA3EE074A23EE844AB4EEE64AAC
:108A3800F1EE10FAB4EEE74A8CBFB0EE667AB0EE0B
:108A4800447AF1EE10FA98BFF0EE476AA8BFF0EE4C
:108A5800447A052A8DED104A6CD093ED164AD3ED71
:108A6800152A93ED177A26EE044AA5EE224AA3EEBC
:108A7800074A23EE844AB4EEE64AF1EE10FAB4EE61
:108A8800E74A8CBFB0EE667AB0EE447AF1EE10FA9F
:108A980098BFF0EE476AA8BFF0EE447A062A8DED3B
:108AA800114A47D093ED1A4AD3ED192A93ED1B7A50
:108AB80026EE044AA5EE224AA3EE074A23EE844A8C
:108AC800B4EEE64AF1EE10FAB4EEE74A8CBFB0EE27
:108AD800667AB0EE447AF1EE10FA98BFF0EE476A83
:108AE800A8BFF0EE447A072A8DED124A22D093ED02
:108AF8001E7AD3ED1D2A93ED1F4A26EE077AA5EEBE
:108B0800227AA4EE037A27EE237AB4EEE67AF1EE1F
:108B180010FAB4EEE77A8CBFB0EE666AB0EE476A38
:108B2800F1EE10FA8DED137A98BFF0EE466AA8BF01
:108B3800F0EE477A77EEE67AF7EE006AF4EEE67A38
:108B4800F1EE10FAC4ED707A43F3BF8486EEA77A8B
:108B5800022ADDED0D7A67EE244A67EE877ACDEDBD
:108B68000C4ACDED0D7A2DD0DDED0E7A67EE877AC1
:108B7800032ACDED0E7A25D0DDED0F7A67EE877AE0
:108B8800042ACDED0F7A1DD0DDED107A67EE877AD5
:108B9800052ACDED107A15D0DDED117A67EE877ACA
:108BA800062ACDED117A0DD0DDED127A67EE877ABF
:108BB800072ACDED127A05D0DDED137A27EE877AF4
:108BC8008DED137A344B1E6816F0805601F09780AD
:108BD800F6EE005AC4ED815A002A02F01C852F4B8C
:108BE800D4ED7F4A93F8038094F900320A99D4EDC2
:108BF8007E6A91F800E0DFF8B0C02949DFF8AC9050
:108C0800B1F906109CED007A059106EE103AFDEEDA
:108C1800E44A244B99F80090B3F81AB094ED7B5AC3
:108C2800D4ED7C7A14EE903AFDEEE64A00F0100C92
:108C380000F480000EF0010EB8EEC66A14EE901A29
:108C48000690B8F1000F41F0EF81DFF84480BCF1E5
:108C5800000F41F09C8098ED007ADDED0C6ADFF89A
:108C680050C025EE877AA6EE867AF0EE676AE7EEC0
:108C7800056ABDEEE67A17EE106A17EE100A9E42F4
:108C8800A8BF184616E000BF2C3E002096430020DF
:108C98009433002000000000383C0020506D002074
:108CA800D8520020446A002070330020D465002088
:108CB800083C0020B142C8BF084607EE100AB8EECB
:108CC800C77A012A8CED007A00F0DC8098ED047AEE
:108CD800DDED0D6A25EE877AA6EE867AF0EE676AF4
:108CE800E7EE056ABDEEE67A17EE106A17EE100A8F
:108CF8009E42A8BF1846B142C8BF084607EE100AF0
:108D0800B8EEC77A022A8CED017A00F0BB8098EDA4
:108D1800087ADDED0E6A25EE877AA6EE867AF0EE01
:108D2800676AE7EE056ABDEEE67A17EE106A17EE97
:108D3800100A9E42A8BF1846B142C8BF084607EEAF
:108D4800100AB8EEC77A032A8CED027A00F09A80EE
:108D580098ED0C7ADDED0F6A25EE877AA6EE867A15
:108D6800F0EE676AE7EE056ABDEEE67A17EE106A7E
:108D780017EE100A9E42A8BF1846B142C8BF08465F
:108D880007EE100AB8EEC77A042A8CED037A79D078
:108D980098ED107ADDED106A25EE877AA6EE867AD0
:108DA800F0EE676AE7EE056ABDEEE67A17EE106A3E
:108DB80017EE100A9E42A8BF1846B142C8BF08461F
:108DC80007EE100AB8EEC77A052A8CED047A59D056
:108DD80098ED147ADDED116A25EE877AA6EE867A8B
:108DE800F0EE676AE7EE056ABDEEE67A17EE106AFE
:108DF80017EE100A9E42A8BF1846B142C8BF0846DF
:108E080007EE100AB8EEC77A062A8CED057A39D033
:108E180098ED187ADDED126A25EE877AA6EE867A45
:108E2800F0EE676AE7EE056ABDEEE67A17EE106ABD
:108E380017EE100A9E42A8BF1846B142C8BF08469E
:108E480007EE100AB8EEC77A072A8CED067A19D011
:108E580098ED1C7ADDED136A65EE875AE6EE265A20
:108E6800E5EE257AFDEEE77A17EE900A8342A8BF71
:108E780003468142C8BF0B4607EE903AF8EEE77A00
:108E8800CCED077ABEF1000F40F03D82002A40F099
:108E9800358238E2AB4B1B78013BDBB2FFF730BAC7
:108EA800A94B07934FF47A761B68B6FBF3F3C3EB31
:108EB8004316A649DFF8B88291F801A0A449B8F989
:108EC800060091F8009003EB8603DE00B6B2B742C5
:108ED80002F04981D5F88810B5F93CE0EB6E4A1CE0
:108EE80007EE90EA7344012AC5F88820EB66F8EE8D
:108EF800E77A02F04381D5ED1E5AD5ED206A07EED8
:108F0800102A37EEE56AB8EEC75A012F86EE057AC1
:108F180037EE257A77EEC77A85ED1F7AE7EE866A0F
:108F280085ED1E7AF0EE667AC5ED216AC5ED206AF8
:108F380002F0DE84D5F89C10B5F93EE02B6F4A1C90
:108F480007EE90EA7344012AC5F89C202B67F8EED7
:108F5800E77A02F02C81D5ED235AD5ED256A07EE84
:108F6800102A37EEE56AB8EEC75A012F86EE057A61
:108F780037EE257A77EEC77A85ED247AE7EE866AAA
:108F880085ED237AF0EE667AC5ED266AC5ED256A89
:108F980002F0D684D5F8B010B5F940E06B6F4A1CE2
:108FA80007EE90EA7344012AC5F8B0206B67F8EE23
:108FB800E77A02F01581D5ED285AD5ED2A6A07EE31
:108FC800102A37EEE56AB8EEC75A012F86EE057A01
:108FD80037EE257A77EEC77A85ED297AE6EE276AA5
:108FE80085ED287AF0EE667AC5ED2B6AC5ED2A6A1A
:108FF80002F0CE84A8F80600B5F8B430544A013B14
:1090080092F80090A5F8B43007990023B9F1070F3A
:109018004B608B60CB607FF468A9F7F7ADFF059BC9
:10902800DFF84C81C01A94F8B831A8F80000002B7A
:109038003FF460A9013B84F8B83115B0BDEC0C8B46
:10904800BDE8F08F94ED5E7AB1F90000D4ED5F6A67
:10905800B1F902E03F4AF4EEC76A80EAE0738EEAAB
:10906800EE71A3EBE073F1EE10FAA1EBEE71B8BF6D
:10907800F0EE476A8B42B8BF0B4607EE103A1378FA
:10908800B8EEC77A27EE287A002B40F02382324BBD
:1090980093ED006AB4EECA6AF1EE10FA41F1E0808D
:1090A800F7EE005A75EEC65A3BEE477A65EEAA5AB5
:1090B8002A4BA7EE256A93ED007A26EE076AB5EEED
:1090C800C06AF1EE10FA40F21686C9EE865AB7EE7B
:1090D800007AB0EE476AA6EEE56AF0EE466AF4EE6C
:1090E800C76AF1EE10FA88BFF0EE476AF5EEC06A7B
:1090F800F1EE10FAB8BFF0EE6B6A194B93ED007AF7
:1091080067EE877AA7EEA68AFFF7E6B9154B164AE7
:109118002B4493ED007AD2ED007A144B67EE277A50
:10912800F7EE006AF4EEE67AF1EE10FA93ED007AC3
:1091380088BFF0EE667A67EE877A27EE888AFFF7AF
:109148007CBA00BFE43D0020F4680020E0680020FD
:10915800E843002028330020303300202433002047
:1091680020330020D8220020183300201433002098
:10917800EC430020072B02F079820026DFF848B381
:10918800B84DDBF800305A0501F16F80B64B1B680B
:109198001B0701F1D280B54B1B78002B40F0F481FE
:1091A800B34F94F8123123B1B24A1288920742F0B1
:1091B800898094F81821002A41F06180BB7F002B38
:1091C80000F0F483022B02F07680032B01F01A835F
:1091D800A94B5B88F97F0231C9B2002A02F05C8092
:1091E800002B02F05980A5480068B3FBF0F30FFA92
:1091F80083F9A4F84891002903F06F8107EE909A4B
:10920800F8EEE77AF7EE006A86EEA77A9C4B01291A
:10921800D4ED576AD3ED007A77EEE67A67EE877A6F
:10922800C4ED537A21D0D3ED017AD4ED586A77EEA4
:10923800E67A022967EE877AC4ED547A15D0D3ED21
:10924800027AD4ED596A77EEE67A032967EE877ACF
:10925800C4ED557A09D0D3ED037AD4ED5A6A77EE86
:10926800E67A67EE877AC4ED567A86480078092848
:1092780003F0F581B9F1000F40F39F8391B394EDAA
:10928800577AD4ED537A77EE877A0129C4ED577A65
:10929800C3ED007A21D094ED587AD4ED547A77EE64
:1092A800877A0229C4ED587AC3ED017A15D094ED76
:1092B800597AD4ED557A77EE877A0329C4ED597A2D
:1092C800C3ED027A09D0D4ED5A7A94ED567A77EE46
:1092D800877AC4ED5A7AC3ED037A01390229B8BFF7
:1092E8000221C9B2002A18BF022167E30A9B664D12
:1092F8001B78DE0700F164812A7822B19200634965
:10930800634824F009FA634B1B68002B40F02F8355
:10931800614B1B789BB1287870B1DFF87481DFF856
:10932800AC910026F0B2D9F80030B8EC010A9847A1
:10933800287801368642F5DB584B1B689847514B15
:109348001B78072B00F01C85012384F8003115B029
:10935800BDEC0C8BBDE8F08F514BC7ED00BA1B6814
:109368009342BFF6F9A84F4B1A88002384F8D031EE
:10937800002A41F0EE864C4A4C4B1178186881F06F
:109388000101F8F7F7FFFFF7EFB8494EDFF8409112
:1093980006F5F47806F51577F6EC017A95ED080AE6
:1093A800D5F81432F8EEE77A404627EE800A984757
:1093B800A8F1E000D5F834319847A8F17000D5F845
:1093C800A4319847D6F8F400D5F8B830984708F192
:1093D80024084745A9EC010ADED1FEF77FBF0A9AA7
:1093E8001278D50703D4224A128BA4F8F421314A03
:1093F8002349128891ED037A07EE902AF8EEE77A6E
:10940800B4EEE77AF1EE10FA41F214812A4909889C
:1094180007EE901AF8EEE77AB4EEE77AF1EE10FA72
:10942800C1F243802549264AD1ED006A92ED006ACF
:109438002449C4ED7E6ABCEEC75A76EE665A15EE2C
:10944800102AC4ED7C6AC4ED7B5A84ED7F6AA4F8C7
:10945800F4210122D1ED006A84F8002277EE677AC0
:10946800FFF77BB900620020C46C0020DE150020E5
:10947800446A0020EE540020286D0020143E00208D
:1094880010440020E8430020964300207433002055
:10949800083C0020A82F0020DC680020D0650020B0
:1094A80044330020C4640020C6640020C86400203F
:1094B80030620020283400202A3400201434002090
:1094C800C03D00203034002004690020C865002019
:1094D800F8680020CC4B93ED005AB5EEC05AF1EE77
:1094E80010FA40F30884C94BD3ED004AF5EEC04AA0
:1094F800F1EE10FA40F3FF8334EEC77A66EEE95ACC
:1095080087EE246AC5EE856AB7EE007AB4EEC76ABC
:10951800F1EE10FA88BFB0EE476AB5EEC06AF1EE18
:1095280010FA76EE876AB8BFB0EE6B6A66EE266A06
:10953800D5E5B74A92ED007AF0EEE76AF4EEC76A2D
:10954800F1EE10FA7FF79AA8B24A92ED007AF0EE9F
:10955800CD6AF4EEC76AF1EE10FA7FF78FA8AE4A2B
:1095680099ED007AD2ED006AB0EEC77AB4EEE67AE9
:10957800F1EE10FA7FF582A801220999C4F8D411F6
:1095880084F8D021FFF77EB8A44BA54FB3F9062085
:109598007B8B9A423FF705AEA24B1B78012B01F05B
:1095A8006686192B01F063860E2B3FF4FAAD082B63
:1095B8003FF4F7AD9C4B00229A60C4F80C21F0E50B
:1095C8002B78002B3FF49FAED4ED5F3A94ED5E6AA2
:1095D800D4ED7C7A954A94ED7B7AD2ED005A94EDDD
:1095E8005C4AD4ED5B4ADFF85C82DFF85CC2F4EEDB
:1095F800C63AF3EE046AF1EE10FA37EEA65A01F114
:10960800528098ED026A26EE446AF0EE674AE6EE6A
:10961800074AF4EEC54A34EEE66AF1EE10FA48BF9E
:10962800B0EE656A012B8CED006A3FF46CAE98EDE4
:10963800066A26EE446AF0EE674AE6EE074AB4EE9A
:10964800E45A34EEE66AF1EE10FA88BFB0EE656AC5
:10965800022B8CED016A3FF456AE98ED0A6A26EEAD
:10966800446AF0EE674AE6EE074AF4EEC54A34EE7D
:10967800E66AF1EE10FA48BFB0EE656A032B8CED8E
:10968800026A3FF440AE98ED0E6A26EE446AF0EEA8
:10969800674AE6EE074AB4EEE45A34EEE66AF1EEBB
:1096A80010FAC8BFB0EE656A042B8CED036A3FF46C
:1096B8002AAE98ED126A26EE446AF0EE674AE6EEA4
:1096C800074AB4EEE45A34EEE66AF1EE10FAC8BF7F
:1096D800B0EE656A052B8CED046A3FF414AE98ED84
:1096E800166A26EE446AF0EE674AE6EE074AF4EE9A
:1096F800C54A74EEE66AF1EE10FAB8BFF0EE656A94
:10970800062BCCED056A3FF4FEADD8ED1A6A66EE7D
:10971800C46AF0EE674AE6EE874AB3EE046AB4EE2E
:10972800E45A74EEC66AF1EE10FAC8BFF0EE656A44
:10973800072BCCED066A3FF4E6ADD8ED1E6A26EE9F
:10974800C44AE4EE077AF4EEC57A77EEC67AF1EE0B
:1097580010FA48BFF0EE657ACCED077AD3E50799A1
:10976800334BD1ED017A93ED007AF0EEE77AF4EE1F
:10977800C77AF1EE10FA7EF5F7AED1ED027AF0EE87
:10978800E77AB4EEE77AF1EE10FA7EF7EDAED1EDB6
:10979800037AF0EEE77AB4EEE77AF1EE10FA7EF7A4
:1097A800E3AE244B1B689A077FF5DDAD2249234BB6
:1097B800B3F90C20B1F900E02148AEEB020E0068C5
:1097C8008EEAEE72A2EBEE728242BEF6CDAEB3F92D
:1097D8000E30B1F90220D21A82EAE273A3EBE273E7
:1097E80098427EF7C1AEBEE50B4B99ED007AD3EDFA
:1097F800006AB0EEC77AB4EEE67AF1EE10FA7EF7B8
:1098080053AFFEF74EBF00BF243300202C33002097
:1098180058330020543300205C330020D8520020F5
:10982800446A00202C3E00201044002070330020A1
:1098380050330020C46C0020206D0020F03D002033
:109848004C33002094330020083C002007EE103AE7
:10985800524BDFF854811B78C4F8A071B8EEC77A70
:10986800F7EE006A132B86EE879AB8F90400B4F86D
:10987800A47195ED080A01F0F783494B494A93ED25
:10988800001A93ED053A93ED122A93ED176AD3ED7A
:10989800091A93ED0E4AD3ED015AD3ED063A93ED2A
:1098A8000A7A93ED0F5AD3ED132AD3ED186AD3ED44
:1098B800044AD3ED030A67EE897A69EE288A29EE0D
:1098C800088AA1EE273A02EB87060021A2EE286A51
:1098D800C4F89411C4F89811A1EE884AE5EEA73AA5
:1098E800A7EE085A93ED167AD3ED0D5A93ED021AA6
:1098F800D3ED0C1A86ED003AE2EEA86A64EEC34A8C
:1099080027EE467A93ED0B2AD3ED152A86ED204AE9
:10991800E0EEC33A65EEC45A93ED143AC3ED053A46
:10992800E1EE274AF0EE477AA1EEC45AE2EE085A71
:10993800E2EEC66AE3EE287AC3ED064A83ED0E5AD4
:10994800C3ED0F5A86ED406AC3ED176AC3ED187A66
:10995800C4F89C117B1C03F01F03A4F8A431A8F8D9
:109968000400FEF79DBBB0EE465AFEF72FBF0AF083
:1099780071F9CDE496ED007A05EB4702B8EEC78A97
:10998800928F2AF8172028EE278AFEF775BC24F054
:1099980037F82AF81700FEF791BC00BFE84300200B
:1099A800AC3A002028380020EC430020A4F84831C5
:1099B8009946002A00F07281DE4B0221DE4ADFED73
:1099C800DF6A1068DE4A90F802C092F800E0027878
:1099D80007EE902AF8EEE77AB0EE007A67EEA67AFC
:1099E800F4EEC77AF1EE10FA40F30E8337EEC77A39
:1099F800DFEDD46AB0EE676AA7EE266AB0EE467A63
:109A08009FEDD16AD3ED006A66EE866AB0EEE66A2B
:109A1800C4ED5B6A84ED5E6ABCF1000F13D005EEFD
:109A280090CAB8EEE55ADFEDC55A66EEA64A25EEAD
:109A3800255AF7EE005A75EEC55A64EE864AE4EEEA
:109A4800855A66EEA56ADFEDC15A427927EE257A76
:109A580027EE267ACAB1DFEDB96ADFEDBD5A26EEE8
:109A6800266A06EE902AF8EEE66A26EE266AB4EE34
:109A7800E56AF1EE10FA00F30486F7EE005A35EEC7
:109A8800C66AC5EE866A27EE267ABEF10C0F9FEDF0
:109A9800B18ADFEDB16A00F06F85B4EEC87AF1EEF5
:109AA80010FA98BFB0EE478AB4EEE68AF1EE10FAE3
:109AB800B8BFB0EE668A84ED418A002900F0E280E2
:109AC800B0EE007AF4EEC77AF1EE10FA05DD37EE63
:109AD800C77ADFED9C6AE7EE267A93ED017ADFED2F
:109AE8009A6A27EE267AB0EEC76A84ED5C7A84ED2E
:109AF8005F6ABCF1000F13D006EE90CADFED8F5AF3
:109B0800F8EEE66A27EE075A66EEA56AF7EE005AFF
:109B180075EEE65A25EE065AE5EE265A27EE257A20
:109B2800DFED8A6A827967EEA67A67EE877AAAB14C
:109B380007EE102AB8EEC77ADFED805ADFED846AA7
:109B480027EE067A27EE257AB4EEE67AF1EE10FAD9
:109B580040F39B85DFED816A67EEA67ABEF10C0FB4
:109B680000F0E984DFED7B6A9FED7B7AF4EEE67A1C
:109B7800F1EE10FA88BFF0EE667AF4EEC77AF1EEED
:109B880010FAB8BFF0EE477A0129C4ED427A79DDC0
:109B98004278DFED6A6A07EE902AF8EEE77AB0EECF
:109BA800007A67EEA67A427AF4EEC77AF1EE10FAF6
:109BB80005DD37EEC77ADFED636AE7EE267A93EDC7
:109BC800027ADFED616A27EE267AB0EEC76A84ED85
:109BD8005D7A84ED606A9AB106EE902ADFED575AF5
:109BE800F8EEE66A27EE075A66EEA56AF7EE005A1F
:109BF80075EEE65A25EE065AE6EE855A27EE257AE0
:109C0800DFED526AC37967EEA67A67EE877A0BB3FF
:109C180007EE103AB8EEC77ADFED485ADFED4C6A26
:109C280027EE067A27EE257AB4EEE67AF1EE10FAF8
:109C38000CDCB5EEC07AF1EE10FA01F12383B7EE31
:109C4800006A36EE477AC6EE076A01E0DFED436A3E
:109C580067EEA67ABEF10C0F00F06384DFED3D6A73
:109C68009FED3D7AF4EEE67AF1EE10FA88BFF0EE59
:109C7800667AF4EEC77AF1EE10FAB8BFF0EE477ADA
:109C8800C4ED437ABEF1090F00F02E8497F82170D5
:109C9800002F40F0C483002384F81831304B1B7820
:109CA80023B9304FBB78002B41F04B83244B1B78F2
:109CB800072B00F07E840022072B84F800217EF415
:109CC8009CA9F7F759F90590FEF799B9264B274C47
:109CD8001A68274BDFF8A48094F80001D2691B8822
:109CE800A8F80020A8F8023000287FF446AA0590BA
:109CF800204DFEF784B9DFED206AFFF7FEB9410277
:109D08003EF566AFFEF768BFF7F736F90C4B0B9ACE
:109D18001B78DFF86880801A012BA8F8020000F091
:109D28006883072B7EF4E8ACF7F726F90746FEF7B9
:109D3800E4BC00BF10440020DC6D00200AD7233C9F
:109D4800E8430020D7A368416F12033B0000484353
:109D5800A4707D3F00C0F94400C0F9C40000C842A7
:109D6800756C00204E6F00201057002060210020E5
:109D7800923400200062002000000000EC43002024
:109D8800F7F7FAF8A24BC01BD880FFF7DDBABEF18F
:109D9800000F41F09F8498ED007ADDED0C6ADFF842
:109DA80084C225EE877AA6EE867AF0EE676AE7EE39
:109DB800056ABDEEE67A17EE106A17EE100A9E42A3
:109DC800A8BF1846B142C8BF084607EE100AB8EE49
:109DD800C77A012A8CED007A3FF490AA98ED047AAC
:109DE800DDED0D6A25EE877AA6EE867AF0EE676AD3
:109DF800E7EE056ABDEEE67A17EE106A17EE100A6E
:109E08009E42A8BF1846B142C8BF084607EE100ACE
:109E1800B8EEC77A022A8CED017A3FF46FAA98ED62
:109E2800087ADDED0E6A25EE877AA6EE867AF0EEE0
:109E3800676AE7EE056ABDEEE67A17EE106A17EE76
:109E4800100A9E42A8BF1846B142C8BF084607EE8E
:109E5800100AB8EEC77A032A8CED027A3FF44EAAAC
:109E680098ED0C7ADDED0F6A25EE877AA6EE867AF4
:109E7800F0EE676AE7EE056ABDEEE67A17EE106A5D
:109E880017EE100A9E42A8BF1846B142C8BF08463E
:109E980007EE100AB8EEC77A042A8CED037A3FF46D
:109EA8002DAA98ED107ADDED106A25EE877AA6EED8
:109EB800867AF0EE676AE7EE056ABDEEE67A17EE97
:109EC800106A17EE100A9E42A8BF1846B142C8BFD2
:109ED800084607EE100AB8EEC77A052A8CED047A10
:109EE8003FF40CAA98ED147ADDED116A25EE877A15
:109EF800A6EE867AF0EE676AE7EE056ABDEEE67AC8
:109F080017EE106A17EE100A9E42A8BF1846B14213
:109F1800C8BF084607EE100AB8EEC77A062A8CEDC5
:109F2800057A3FF4EBA998ED187ADDED126A25EE73
:109F3800877AA6EE867AF0EE676AE7EE056ABDEEE6
:109F4800E67A17EE106A17EE100A9E42A8BF184666
:109F5800B142C8BF084607EE100AB8EEC77A072A0A
:109F68008CED067A3FF4CAA998ED1C7ADDED136AE8
:109F780065EE875AE6EE265AE5EE257AFDEEE77A93
:109F880017EE900A8342A8BF03468142C8BF0B461A
:109F980007EE903AF8EEE77ACCED077A002A7FF4DC
:109FA800ADA9FFF7B0B91B4B5A79002A3EF493AC20
:109FB800194A1278002A3EF48EAC1B78DFED174A56
:109FC80007EE903A164BB8EE677A1B8807EE902A90
:109FD80006EE903AF8EEE77AF8EE666A67EE277AC8
:109FE800B7EE007AC7EEA63AF4EEE43AF1EE10FACC
:109FF80088BFF0EE643AF4EEC73AF1EE10FAB8BF53
:10A00800F0EE473AFEF769BCB0EE677AF8E400BFB5
:10A01800EC430020406D00200E440020713DAA3F13
:10A02800F8430020083C0020BCF1000F00F0FE833C
:10A03800BEF1000F41F0CE87DFF8EC85B9F1000FD3
:10A0480041F02686D8ED006ADDED0C4ADFF8DCC564
:10A0580065EEA66ABDEEC77A17EE101AB0EE667AFC
:10A06800A4EE867AF0EE676AE7EE056ABDEEE67A58
:10A0780017EE106A17EE100A9E42A8BF1846B142A2
:10A08800C8BF084607EE100AB8EEC77A012A8CED59
:10A09800007A3FF433A998ED047ADDED0D6A25EED8
:10A0A800877AA6EE867AF0EE676AE7EE056ABDEE75
:10A0B800E67A17EE106A17EE100A9E42A8BF1846F5
:10A0C8008E42B8BF084607EE100AB8EEC77A022AD1
:10A0D8008CED017A3FF412A998ED087ADDED0E6A4D
:10A0E80025EE877AA6EE867AF0EE676AE7EE056ACD
:10A0F800BDEEE67A17EE106A17EE100A9E42A8BF68
:10A1080018468E42B8BF084607EE100AB8EEC77A5E
:10A11800032A8CED027A3FF4F1A898ED0C7ADDED74
:10A128000F6A25EE877AA6EE867AF0EE676AE7EE82
:10A13800056ABDEEE67A17EE106A17EE100A9E421F
:10A14800A8BF18468E42B8BF084607EE100AB8EEF8
:10A15800C77A042A8CED037A3FF4D0A898ED107AD8
:10A16800DDED106A25EE877AA6EE867AF0EE676A4C
:10A17800E7EE056ABDEEE67A17EE106A17EE100AEA
:10A188009E42A8BF18468E42B8BF084607EE100A7E
:10A19800B8EEC77A052A8CED047A3FF4AFA898ED9B
:10A1A800147ADDED116A25EE877AA6EE867AF0EE4E
:10A1B800676AE7EE056ABDEEE67A17EE106A17EEF3
:10A1C800100A9E42A8BF18468E42B8BF084607EE3E
:10A1D800100AB8EEC77A062A8CED057A3FF48EA8E5
:10A1E80098ED187ADDED126A25EE877AA6EE867A62
:10A1F800F0EE676AE7EE056ABDEEE67A17EE106ADA
:10A2080017EE100A9E42A8BF18468E42B8BF0846ED
:10A2180007EE100AB8EEC77A072A8CED067A3FF4E3
:10A228006DA898ED1C7ADDED136A65EE875AE6EEA7
:10A23800265AE5EE257AFDEEE77A17EE900A834274
:10A24800A8BF03468142D8BF194607EE901AF8EE18
:10A25800E77ACCED077A002A7FF450A8FFF753B8C5
:10A26800D94B93ED006AFEF72ABFAB68002B3EF48A
:10A278008DAF05F1500128469847FEF787BFD34BAD
:10A28800D349D3F8EC30086844F620618B42A8BF64
:10A298000B46B3F57A7FB8BF4FF47A7399B2C0060C
:10A2A800A4F81A11DBF8003041F11D83DB0440F1FA
:10A2B800D283C84BD3F800C0BCF832E04FEA5E0E38
:10A2C800C54BC648D3ED037AD4F81C31A0FB010175
:10A2D8008809642191FBF0F11429BDEEE77A04EBBB
:10A2E8004308A8BF142101338B42C4F81C3117EE70
:10A2F800109AA4BF0023C4F81C3104EB4303A8F848
:10A308002091B3F9203107EE103AB8EEC77A77EE0C
:10A31800C77AFDEEE77ACDED057ABDF9141081EA2A
:10A32800E173A3EBE173734502F3C080AC4B1946AC
:10A338004FF07E530B60FEF741BFA74BA949D3ED01
:10A34800027AB2EE0E7AF0EEE76AF4EEC76AF1EE40
:10A3580010FA40D5A44A128857073CD5A348B1F94A
:10A368000420B4F8027180FB0201D217C2EBA102EB
:10A37800D21B92B211B211F1B30FBCBF02F5B47285
:10A3880011B2B329C4BFA1F5B47211B2984A994861
:10A3980012790078002A4FF6FF7218BF01220007D1
:10A3A8007EF5F9AE8B48006811FB02F2017E9248F7
:10A3B80092B211FB02F280FB02011144D217C2EBE8
:10A3C800211207EE102AB8EEC77A77EEC77AC3EDE6
:10A3D800027AFEF7E0BEB1F90430844A82FB031228
:10A3E800DB17C3EBA203A4F80231FEF7D4BEDFF8F3
:10A3F8004082F6F7C1FD814AD4F8E4311268C4F806
:10A40800E401C31A9A1A0746A8F80430A8F80620E7
:10A41800FEF773B9F6F7B0FD0B90FDF77ABF1E2172
:10A428006B48F8F737FF00283FF435AC6E4B1B88B4
:10A438005A063FF530AC94F88431BB4242F0718043
:10A44800674BD4ED627A93ED010AD4ED435A9FED40
:10A458006C6ADFED6C6A27EEE57A68EE277AA8EE7B
:10A46800007AE5EE807AB4EEC67AF1EE10FA88BF8B
:10A47800B0EE467AB4EEE67AF1EE10FAF4EEC67A69
:10A48800B8BFB0EE667AF1EE10FA88BFF0EE467A01
:10A49800F4EEE67AF1EE10FAB8BFF0EE667A84EDE3
:10A4A800417AC4ED437AFFF7F6BBB4F8F411914250
:10A4B80040F28B855449554AD1ED007A92ED007AE5
:10A4C8005349C4ED7E7A77EE676AC4ED7C7A01223F
:10A4D800C4ED7B6A84ED7F7AD1ED006ADFED4D7AB9
:10A4E80084F80022FEF739B9FDEEC87ADFF840811A
:10A4F80017EE903AA8F80490A8F80630FFF7C6BB04
:10A50800454B1B88002B40F07F85444A444B11780B
:10A518001868F7F72FFFD4F8D421099B9A1AFDF78A
:10A52800F2BFBDEEE77ADFF8088117EE103AA8F817
:10A538000430FFF793BB9FED327ADFED326ADFF824
:10A54800F080F4EEC77AF1EE10FA98BFB0EE677AB1
:10A55800FDEEE77AB4EEE67AF1EE10FA17EE902AFD
:10A56800B8BFB0EE667A012984ED427AA8F80220D5
:10A578003FF70EABFFF78ABBB4EEC87AF1EE10FADC
:10A5880098BFB0EE478ABDEEC77AB4EEE68ADFF828
:10A59800A080F1EE10FA17EE102AB8BFB0EE668A66
:10A5A80084ED418AA8F8002000297FF489AAFFF7E2
:10A5B8006DBBF6F7E1FCDFF878801A4B801B1B783F
:10A5C800A8F80400FFF777BB24330020C40100205B
:10A5D800383C00209C6C002010440020D34D6210B1
:10A5E8009C000020206D0020EE54002067666666FF
:10A5F800E83D0020403C002089888888143E0020DF
:10A6080000C0F94400C0F9C414340020C03D002043
:10A618003034002000000000C4640020C66400201C
:10A62800C8640020E843002094330020083C002040
:10A63800EC430020784A7949D2ED006A784A91EDD6
:10A64800006A1278C4ED7E6A84ED7F6A002A40F0C1
:10A65800B88476EEC65AF0EE466ABCEEC76A71490F
:10A66800C4ED7B5A16EE102AC4ED7C6AA4F8F421D6
:10A67800FF22D1ED006A84F8002277EEC77AFEF750
:10A688006CB8DFED696AFFF7FEB9B5EEC07AF1EE96
:10A6980010FA00F1F385B7EE006A36EE477AC6EE97
:10A6A800076AFFF759BA98ED016A26EE646AB0EEB8
:10A6B800674AA6EE074AB4EEC45A34EE666AF1EE6B
:10A6C80010FAC8BFB0EE656A012B8CED006A3EF443
:10A6D8001AAE98ED056A26EE646AB0EE674AA6EEF1
:10A6E800074AB4EEC45A34EE666AF1EE10FAC8BFEF
:10A6F800B0EE656A022B8CED016A3EF404AE98ED6B
:10A70800096A26EE646AB0EE674AA6EE074AB4EE16
:10A71800C45A34EE666AF1EE10FAC8BFB0EE656A44
:10A72800032B8CED026A3EF4EEAD98ED0D6A26EE31
:10A73800646AB0EE674AA6EE074AB4EEC45A34EE2D
:10A74800666AF1EE10FAC8BFB0EE656A042B8CEDAC
:10A75800036A3EF4D8AD98ED116A26EE646AB0EE4D
:10A76800674AA6EE074AB4EEC45A34EE666AF1EEBA
:10A7780010FAC8BFB0EE656A052B8CED046A3EF48A
:10A78800C2AD98ED156A26EE646AB0EE674AA6EE89
:10A79800074AB4EEC45A74EE666AF1EE10FAC8BFFE
:10A7A800F0EE656A062BCCED056A3EF4ACADD8ED4B
:10A7B800196A66EEE46AB0EE674AA6EE874AB3EE17
:10A7C800046AB4EEC54A74EE466AF1EE10FA48BF60
:10A7D800F0EE656A072BCCED066A3EF494ADD8ED31
:10A7E8001D6A66EEE44AE4EE877AF4EEC57A77EEFF
:10A7F800C67AF1EE10FAB8BFF0EE657ACCED077ABA
:10A80800FEF781BD97F82030C3EB431103EB8103BA
:10A81800DB009BB2FEF7DEBC5C3C00201834002055
:10A82800D46500202C3400200000C842DFF8D8840A
:10A83800B9F1000F41F0C280D8ED006ADDED0C4A95
:10A84800DFF8C8C465EEA66ABDEEC77A17EE101A1F
:10A85800B0EE667AA4EE867AF0EE676AE7EE056AED
:10A86800BDEEE67A17EE106A17EE100A9E42A8BFF0
:10A878001846B142C8BF084607EE100AB8EEC77AB4
:10A88800012A8CED007A3EF4FDAA98ED047ADDEDFC
:10A898000D6A25EE877AA6EE867AF0EE676AE7EE0D
:10A8A800056ABDEEE67A17EE106A17EE100A9E42A8
:10A8B800A8BF18468E42B8BF084607EE100AB8EE81
:10A8C800C77A022A8CED017A3EF4DCAA98ED087A60
:10A8D800DDED0E6A25EE877AA6EE867AF0EE676AD7
:10A8E800E7EE056ABDEEE67A17EE106A17EE100A73
:10A8F8009E42A8BF18468E42B8BF084607EE100A07
:10A90800B8EEC77A032A8CED027A3EF4BBAA98ED1A
:10A918000C7ADDED0F6A25EE877AA6EE867AF0EEE0
:10A92800676AE7EE056ABDEEE67A17EE106A17EE7B
:10A93800100A9E42A8BF18468E42B8BF084607EEC6
:10A94800100AB8EEC77A042A8CED037A3EF49AAA64
:10A9580098ED107ADDED106A25EE877AA6EE867AF4
:10A96800F0EE676AE7EE056ABDEEE67A17EE106A62
:10A9780017EE100A9E42A8BF18468E42B8BF084676
:10A9880007EE100AB8EEC77A052A8CED047A3EF471
:10A9980079AA98ED147ADDED116A25EE877AA6EE8C
:10A9A800867AF0EE676AE7EE056ABDEEE67A17EE9C
:10A9B800106A17EE100A9E42A8BF18468E42B8BF0A
:10A9C800084607EE100AB8EEC77A062A8CED057A13
:10A9D8003EF458AA98ED187ADDED126A25EE877ACA
:10A9E800A6EE867AF0EE676AE7EE056ABDEEE67ACD
:10A9F80017EE106A17EE100A9E42A8BF18468E423C
:10AA0800B8BF084607EE100AB8EEC77A072A8CEDD9
:10AA1800067A3EF437AA98ED1C7ADDED136A65EEE6
:10AA2800875AE6EE265AE5EE257AFDEEE77A17EE26
:10AA3800900A8342A8BF03468142D8BF194607EE51
:10AA4800901AF8EEE77ACCED077ABEF1000F7EF4A3
:10AA58005AACFEF71BBAA04BD3F800C0BCF932E0E1
:10AA68002EE4DFF8AC92D4ED017A94ED006AB9F8DF
:10AA78000000D9F8143077EEA77AF0EE006AB0EE4D
:10AA8800677AA6EE267A013804EBC002D6EE267A5B
:10AA9800083A1033F6EE003A27EE237A67EEA37AE7
:10AAA80084ED207AC4ED217A8C4CA64604F180010D
:10AAB80092ED027A92ED036ADEED036ADEED027A28
:10AAC80053ED014A13ED025A37EE674A76EEC65A3D
:10AAD80077EE277AE4EE845A0138A2F10802E5EE0F
:10AAE800047A0EF1080E03F1080336EE267A01F116
:10AAF8000801E4EE877AE5EE475A67EEA37A25EE79
:10AB0800A37AC1ED007A81ED017AD1D1142F7DF4B9
:10AB180082ABF6F731FA069BDFF8F881C01AA8F87D
:10AB28000200D4F8A861FDF776BBD4F8AC81B4F87C
:10AB3800A4A16B4BCAF120095FFA89F90AEB481EF8
:10AB480003EB8E0E5FEA990301F084850133180147
:10AB58006449654A0EEB000C0EF1100313ED024A2E
:10AB680013ED035A13ED016A13ED047A51ED024A0D
:10AB780051ED035A51ED016A51ED047A64EE244A0D
:10AB880065EE255A66EE266A67EE277A10339C45ED
:10AB980042ED024A42ED035A42ED016A42ED047A5F
:10ABA80001F1100102F11002D8D15049A0F11002B0
:10ABB800964401EB020C224419F0030309D0BEECC1
:10ABC800017AFCEC017A67EE277A013BE2EC017A24
:10ABD800F5D1BAF1000F41F09E81142F7DF41BAB23
:10ABE800F6F7CAF9069BDFF82C81D4F8A861C01AD9
:10ABF800A8F80200FDF70FBBD4F8AC913C4B3D4AD6
:10AC0800DFED3D7AD2ED008A3C4A4FEAC9010B4498
:10AC1800F8EE688A9B8809EE103A643BC82BA8BFF7
:10AC2800C82368EEA78AF8EE497A782BB8BF78234C
:10AC380068EEA78A07EE903A4944B0EE680A02EB3C
:10AC48008108B8EEE78A22F027FFB8EEC99AF0EE3D
:10AC5800409AB0EE680A22F081FE38EE097A79EE61
:10AC6800487A28EE098A67EE877AB7EE006A88EE96
:10AC7800277A142FF8EE007A77EE076A60EE277AC3
:10AC880089EEA67A77EE065A36EE477AC6EE256A38
:10AC980067EEA67A27EE267AC8ED006A88ED047A70
:10ACA800C8ED026AC8ED017AC8ED037A01F0718532
:10ACB800134B144A09F1010983FB0938A8EBE97819
:10ACC80008EB48080136A9EB08081778C4F8A8610A
:10ACD800C4F8AC812BE700BF9C6C002060210020E9
:10ACE80028380020B839002070210020A839002019
:10ACF800283A0020F468002027D4D23618640020AF
:10AD080056555555E843002094330020083C002050
:10AD180010380020EC430020DFF83C93B9F800E03D
:10AD2800D9F804C04FEA5E084FEA880204EB8E06A1
:10AD38005FEADE0E04EB020300F0A08010320EF191
:10AD4800010EBA4803EB0E1E324410330CF1100703
:10AD580006F1100151ED032A51ED043A10ED043AC1
:10AD680010ED032A51ED026A11ED016A10ED020A95
:10AD780010ED018A12ED044A12ED035A53ED044A0C
:10AD880053ED035A13ED027A53ED017A52ED020A9C
:10AD980012ED011A73EE238A72EE221A40ED048A2C
:10ADA80040ED031A70EE268A78EE061A40ED028A04
:10ADB80040ED011A74EE848A75EE851A43ED048A13
:10ADC80043ED031A77EE208A77EE811A43ED028A63
:10ADD80043ED011A73EE633A75EE655A17ED035A9F
:10ADE80032EE623A74EE644A65EE631A17ED044A6D
:10ADF80023EE052A64EE652AE3EE041A10339E4515
:10AE080024EE843AA3EE842A00F1100007F110071B
:10AE1800A5EE853A01F1100102F11002E4EE852A4F
:10AE280041ED071A01ED082A02ED073A42ED082A1A
:10AE380057ED055A17ED065A70EE666A38EE466AFF
:10AE480030EEC77A71EE677A26EE253A65EEE63A75
:10AE580025EE674A67EE054AE6EE053AA6EE853A1C
:10AE6800A7EE254AE7EEA54A01ED063A41ED053A77
:10AE780002ED064A42ED054A7FF46CAF1FFA88F8E6
:10AE8800624641466A4818F0A9FF4146D9F80420AD
:10AE9800304618F0A3FF674B1B78142B7FF441AEA4
:10AEA80037E6DFF8B4916248D9F80820B9F80C10F1
:10AEB80021F0FEFD5F4B1F78142F01F01884D4F8A1
:10AEC800A8610136C4F8A861CDE5DFF8909199F83A
:10AED8000020900801F0B484DFF884C100F1010873
:10AEE8004FEA48180CEB080E0CF12003ACF1700186
:10AEF80013ED076A53ED056A13ED037A53ED017AF2
:10AF080053ED025A13ED084A53ED064A13ED045A5D
:10AF180026EE066A66EEA66A27EE077A67EEA77A35
:10AF2800A4EE046A20339E45E4EEA46A01F1100100
:10AF3800A5EE057AE5EEA57AF1EEC65AB1EEE66A17
:10AF4800F1EEC76AB1EEE77A41ED085A01ED076AFA
:10AF580041ED066A01ED057ACAD1A8F12008C4447A
:10AF680004EB001012F0030318BF0CF1080C0FD00B
:10AF78005CED017A1CED027A67EEA77A013BE7EEF9
:10AF8800077A0CF1080CB1EEE77AA0EC017AEFD160
:10AF9800142F01F09C830136C4F8A861FDF7A4B80A
:10AFA800F5F7EAFF234B06901F78142F05BFDFF84B
:10AFB800B480D4F8A861D4F8A861A8F80060FDF7B7
:10AFC80078B876EE665AFFF748BB1B4A1B49D2EDA4
:10AFD800007A1B4A91ED007A1278C4ED7E7A84EDEE
:10AFE8007F7A002A01F05C8277EE676A1549C4ED22
:10AFF8007C7AC4ED7B6AFF22D1ED006ADFED127A1C
:10B0080084F80022FDF7A9BB10494B69002B3DF4D9
:10B018007AAA0F480F4B008893FBF0F00B684FF0AB
:10B02800010E186081F811E0FDF76DBA702100205B
:10B0380060210020E84300205C3C002018340020F8
:10B04800D46500202C34002000000000CC640020CF
:10B05800E464002020A10700103800200A380020EE
:10B06800E0210020EC430020C04EDFF8309396ED3D
:10B07800004A96ED057AD6ED014A96ED066AD6EDB8
:10B08800046A96ED035AD6ED025A67EE897A09EBFF
:10B098008703A4EE277AA4EEA76A66EEC76AA5EE30
:10B0A800476AE5EEA76A20EE070A86ED056AC6ED4F
:10B0B800066A83ED007A29EE088A22F0A1FC69EE7F
:10B0C800288AD6ED0E5AD6ED176A96ED091AD6EDEE
:10B0D800121A96ED0F5A96ED187A96ED0A2AD6EDC1
:10B0E800132A96ED0D6AD6ED167A96ED0C3AD6ED42
:10B0F8000B3A96ED154AD6ED144AE1EE085A0022AD
:10B1080009EB8703E8EEA16A00B2C4F89421A2EE25
:10B11800085AC4F89821C4F89C21A8EEA27A26EE11
:10B12800656A67EEE67AA3EE655AA3EE886AA6EE2C
:10B13800C47AE8EEA47A86ED0E5AC3ED205A86ED5D
:10B148000F6AC3ED406A86ED177AC6ED187AFEF7E6
:10B1580001BC87494A69002A3DF406AA0A681360B7
:10B168004B74FDF701BAB5F93C306A6207EE903AC4
:10B178000122F8EEE77AEB66C5F888200023012F54
:10B18800C5ED1F7AC5ED1E7AC5F8803001F0B4818F
:10B19800B7427DF4CFAEB5F93E302B6707EE903A53
:10B1A80000220123F8EEE77AAA62C5F89C30002352
:10B1B800012FC5ED247AC5ED237AC5F8943001F046
:10B1C8009781B7427DF4E6AEB5F940306B6707EE7C
:10B1D800903A00220123F8EEE77AEA62C5F8B03027
:10B1E8000023012FC5ED297AC5ED287AC5F8A830C6
:10B1F8007DF400AF9FED5F8AB9F1030F46D0BAF135
:10B20800000F09D007EE90AAF8EEE77AF4EEC87AB4
:10B21800F1EE10FA01F15E83574A6B6F126894F8E9
:10B22800B011A8F8060003EB560393FBF6F60023CB
:10B23800EE6293621363D36231B1504B1B8823F4DF
:10B248000063002B7DF4D8AE4D4B1B6813F400331C
:10B2580041F046814B491A46C85C012803F10C03AA
:10B2680000F0F2840132152AF6D1FDF7C5BE464B2F
:10B278009B7B002B3EF49EA9FDF793BFF7EE006A77
:10B28800FEF76ABCF7EE006AFEF7E2BCB0EE480AC9
:10B2980022F0B6FB00B2B2E7B4F8489109F1FF39E1
:10B2A8000FFA89F9B9F1000FA4F848917EF781AB3C
:10B2B800364BFDF7E3BFB4F81A3103F57A739BB246
:10B2C800FDF788BF324ADFED337A92ED080A05931D
:10B2D800B4EEE70AF1EE10FA40F2198622F026FCE5
:10B2E800D4ED457A20EE270A22F08AFBB0F5617F7B
:10B2F800059B00F3A68707EE900AF8EEE76ADFEDF4
:10B30800267A66EEA76A07EE903AB8EEE77AFDEE7F
:10B31800E67A17EE903A2033402B41F24D829FEDAA
:10B32800150A22F06DFB00B207EE900AB8EEE77A34
:10B33800164BD3ED037A77EE877AC3ED037AFDF7E0
:10B3480038BFDFF85C8098F80020013A0A2A3AD81A
:10B35800DFE812F0E5005501AC0039013900390089
:10B368000F01250187007100280000BFAC3A0020BA
:10B37800CC6400200000000010570020746D0020ED
:10B38800C8310020C40703085C5F00201044002077
:10B39800543100208FC2753CD06D393A28380020CE
:10B3A8004B6F0020BD4ABE4952680968C8328A42BC
:10B3B80003D31DF047F830B1BB78032B01F04D8360
:10B3C800012388F80030FB78002B3EF46FACB54BB6
:10B3D8001B78D80740F1AC80DFF8C492D4F89021EC
:10B3E800D9F800309A4200F2AF8098F80030012B6B
:10B3F8003EF45CAC94F88C21002A3EF457AC0B2B3D
:10B408000DD801229A4040F6030112EA01070DD136
:10B4180012F4C06F03D0093B012B41F247839F4BC5
:10B42800D9F800205A600B2388F80030002384F8EC
:10B438008C31FEF73BBC9C4B1B78002B01F0B7818D
:10B448001A2020F0B3F8002841F0B18194F88C312B
:10B45800002B41F0AC81092388F800300EF016FE6D
:10B46800B1E71A2020F0A2F80028F7D08F4B1B88EC
:10B47800002BF3D18E4B4520D3F800901DF006F831
:10B488000E201DF003F848460EF066FADDF8249009
:10B4980048460EF061FA874A874B12681A60484698
:10B4A8000A2388F800300EF021FBD7E7DFF8EC918B
:10B4B8001CF0A8FF7A4AD9F8043012686433934222
:10B4C80081D240201CF082FF00287FF47CAFD9F89D
:10B4D8000030DFF8FCB179494FF0400A0FE00591E0
:10B4E8001CF0D4FF0599D9F800300A680133013AF5
:10B4F800BAF1010A0A60C9F8003001F025821BF888
:10B5080003301846002BEAD100234FF0FF32C9F868
:10B5180000300423C9F8042088F8003053E7614B51
:10B528001B78DB0701F1F981FB78002B3EF4BEABF9
:10B538000AF0A0FF00283FF44FAF594B1B6803F5F2
:10B548009C530833C4F8903198F80030012B7EF4EE
:10B55800ADAB94F88C31002B7EF4A8ABBB78032BF1
:10B5680001F0BF820FF084FB012384F88C31FEF7D1
:10B578009DBB1CF047FF524B002105208DE80300BE
:10B58800A3F10802029153200FF0A8FA00287FF4D3
:10B598001AAF424A0823106088F8003013E71CF0FD
:10B5A80031FF0EF0A5FD00283FF40DAF1CF04AFF57
:10B5B80000283FF408AF3F4A3F4B12681A600A233D
:10B5C80088F80030FFE61CF01DFF3E4A0292A2F107
:10B5D8000C03282101930091A2F10A035021163A85
:10B5E80049200FF07BFA00287FF4EDAE2B4B4FF08B
:10B5F800FF3107221860596088F80020E3E6284BDD
:10B60800264A1B6853602D490023136003220B60F0
:10B6180088F80020D7E60A9B93F800E00EF0010EA8
:10B62800BEF1000F7DF46FAEFDF730BC264BDFEDA9
:10B63800277A1E68C4ED707A16F0805640F01C8395
:10B6480010F4800600F0B0810026B6EE007A67EEAE
:10B65800877AF4EEE75AF1EE10FA48BFF0EE675A2F
:10B6680040F10A83C4ED815AFDF7B6BAF5F784FCB8
:10B678000646FDF783BD74EE677AB7EE007AF4EEFE
:10B68800C77AF1EE10FAC4ED707A40F31E8784EEA3
:10B69800A77A8DED0C7AFDF795BA00BFC43D00205E
:10B6A800A4610020FC6B0020803E0020483C002064
:10B6B800443C00202C3C0020283C0020DC6B00206F
:10B6C800D0010308FEFF0208383C0020000000807B
:10B6D80098FF0208BAF1000F00F0CD8598ED007AC6
:10B6E800DDED0C6ADFF8E8C825EE877AA6EE867AE3
:10B6F800F0EE676AE7EE056ABDEEE67A17EE106AC5
:10B7080017EE100A9E42A8BF1846B142C8BF0846A5
:10B7180007EE100AB8EEC77A012A8CED007A3DF4DC
:10B72800F2AD98ED047ADDED0D6A25EE877AA6EE86
:10B73800867AF0EE676AE7EE056ABDEEE67A17EEFE
:10B74800106A17EE100A9E42A8BF1846B142C8BF39
:10B75800084607EE100AB8EEC77A022A8CED017A7D
:10B768003DF4D1AD98ED087ADDED0E6A25EE877AC5
:10B77800A6EE867AF0EE676AE7EE056ABDEEE67A2F
:10B7880017EE106A17EE100A9E42A8BF1846B1427B
:10B79800C8BF084607EE100AB8EEC77A032A8CED30
:10B7A800027A3DF4B0AD98ED0C7ADDED0F6A25EE26
:10B7B800877AA6EE867AF0EE676AE7EE056ABDEE4E
:10B7C800E67A17EE106A17EE100A9E42A8BF1846CE
:10B7D800B142C8BF084607EE100AB8EEC77A042A75
:10B7E8008CED037A3DF48FAD98ED107ADDED106A9B
:10B7F80025EE877AA6EE867AF0EE676AE7EE056AA6
:10B80800BDEEE67A17EE106A17EE100A9E42A8BF40
:10B818001846B142C8BF084607EE100AB8EEC77A04
:10B82800052A8CED047A3DF46EAD98ED147ADDEDC1
:10B83800116A25EE877AA6EE867AF0EE676AE7EE59
:10B84800056ABDEEE67A17EE106A17EE100A9E42F8
:10B85800A8BF1846B142C8BF084607EE100AB8EE9E
:10B86800C77A062A8CED057A3DF44DAD98ED187A25
:10B87800DDED126A25EE877AA6EE867AF0EE676A23
:10B88800E7EE056ABDEEE67A17EE106A17EE100AC3
:10B898009E42A8BF1846B142C8BF084607EE100A24
:10B8A800B8EEC77A072A8CED067A3DF42CAD98EDF0
:10B8B8001C7ADDED136A65EE875AE6EE265AE5EE48
:10B8C800257AFDEEE77A17EE902A9342A8BF134631
:10B8D8008A42A8BF194607EE901AF8EEE77ACCED2F
:10B8E800077AFDF710BDD8003EF5E0ACFDF766BC61
:10B8F800012A40F3018607EE101AB8EEC77AC7EEA0
:10B90800876AB1EEE68AB9F1030F13D0BAF1000FD6
:10B9180009D007EE90AAF8EEE77AF4EEC87AF1EECD
:10B9280010FA00F1D787EB6E03EB560393FBF6F39F
:10B938006B622DE4B0EE480A22F062F800B2E5E747
:10B94800012A40F3D58507EE101AB8EEC77AC7EE7C
:10B95800876AB1EEE68AB9F1030F13D0BAF1000F86
:10B9680009D007EE90AAF8EEE77AF4EEC87AF1EE7D
:10B9780010FA00F1AF872B6F03EB560393FBF6F336
:10B98800AB621EE4B0EE480A22F03AF800B2E5E7EE
:10B99800012A7FF72FAC07EE101AB8EEC77AC7EE68
:10B9A800876AB1EEE68A27E4B6EE007AF4EEC75A63
:10B9B800F1EE10FA3FF749AEFDF70EB9D8ED004A9F
:10B9C8009DED0C4ADFF808C665EEA44AFDEEC73ABD
:10B9D800E4EE064AB0EE674AA4EE854A13EE901AE2
:10B9E800F4EEC46AF1EE10FAF0EE444A88BFF0EEC5
:10B9F800474AFDEEE44A14EE900A14EE906A984223
:10BA0800A8BF1E468142C8BF0E4604EE906AF8EEF3
:10BA1800E44A012ACCED004A3DF434AAD8ED044AA0
:10BA28009DED0D4A65EEA44AE4EE064AB0EE674A7B
:10BA3800A4EE854AF4EEC46AF1EE10FAF0EE444A38
:10BA480088BFF0EE474AFDEEE44A14EE900A14EE81
:10BA5800906A9842A8BF1E468842B8BF0E4604EEB8
:10BA6800906AF8EEE44A022ACCED014A3DF40AAAAB
:10BA7800D8ED084A9DED0E4A65EEA44AE4EE064A62
:10BA8800B0EE674AA4EE854AF4EEC46AF1EE10FA05
:10BA9800F0EE444A88BFF0EE474AFDEEE44A14EE61
:10BAA800900A14EE906A9842A8BF1E468842B8BF12
:10BAB8000E4604EE906AF8EEE44A032ACCED024AF8
:10BAC8003DF4E0A9D8ED0C4A9DED0F4A65EEA44A75
:10BAD800E4EE064AB0EE674AA4EE854AF4EEC46A7C
:10BAE800F1EE10FAF0EE444A88BFF0EE474AFDEE58
:10BAF800E44A14EE900A14EE906A9842A8BF1E46D3
:10BB08008842B8BF0E4604EE906AF8EEE44A042A6A
:10BB1800CCED034A3DF4B6A9D8ED104A9DED104A84
:10BB280065EEA44AE4EE064AB0EE674AA4EE854AFA
:10BB3800F4EEC46AF1EE10FAF0EE444A88BFF0EE73
:10BB4800474AFDEEE44A14EE900A14EE906A9842D1
:10BB5800A8BF1E468842B8BF0E4604EE906AF8EEAB
:10BB6800E44A052ACCED044A3DF48CA9D8ED144AE0
:10BB78009DED114A65EEA44AE4EE064AB0EE674A26
:10BB8800A4EE854AF4EEC46AF1EE10FAF0EE444AE7
:10BB980088BFF0EE474AFDEEE44A14EE900A14EE30
:10BBA800906A9842A8BF1E468842B8BF0E4604EE67
:10BBB800906AF8EEE44A062ACCED054A3DF462A9FB
:10BBC800D8ED184A9DED124A65EEA44AE4EE064AFD
:10BBD800B0EE674AA4EE854AF4EEC46AF1EE10FAB4
:10BBE800F0EE444A88BFF0EE474AFDEEE44A14EE10
:10BBF800900A14EE906A9842A8BF1E468842B8BFC1
:10BC08000E4604EE906AF8EEE44A072ACCED064A9E
:10BC18003DF438A9D8ED1C4A9DED134A65EEA45AA7
:10BC2800E6EE045AE5EE257AF4EEE76AF1EE10FA4C
:10BC3800C8BFF0EE477AFEF7F8BE8223FCF7D7BA02
:10BC4800DFEDE07AFCF79EBAD4F8B46153003EB158
:10BC5800981801EB800076784078B042BDF4CCA902
:10BC6800134401EB83010023C4F8B411A4F808328B
:10BC7800C4F80C32FDF7C0B9B7EE007A77EE677AF0
:10BC8800F4EEE75AF1EE10FA88BFF0EE675AE9E4ED
:10BC9800D8ED004A9DED0C4ADFF834C365EEA44A9E
:10BCA800FDEEC73AE4EE064AB0EE674AA4EE854ACE
:10BCB80013EE901AF4EEC46AF1EE10FAF0EE444A6C
:10BCC80088BFF0EE474AFDEEE44A14EE900A14EEFF
:10BCD800906A9842A8BF1E468142C8BF0E4604EE2D
:10BCE800906AF8EEE44A012ACCED004A3DF406AB2E
:10BCF800D8ED044A9DED0D4A65EEA44AE4EE064AE5
:10BD0800B0EE674AA4EE854AF4EEC46AF1EE10FA82
:10BD1800F0EE444A88BFF0EE474AFDEEE44A14EEDE
:10BD2800900A14EE906A9842A8BF1E468842B8BF8F
:10BD38000E4604EE906AF8EEE44A022ACCED014A77
:10BD48003DF4DCAAD8ED084A9DED0E4A65EEA44AFA
:10BD5800E4EE064AB0EE674AA4EE854AF4EEC46AF9
:10BD6800F1EE10FAF0EE444A88BFF0EE474AFDEED5
:10BD7800E44A14EE900A14EE906A9842A8BF1E4650
:10BD88008842B8BF0E4604EE906AF8EEE44A032AE9
:10BD9800CCED024A3DF4B2AAD8ED0C4A9DED0F4A0B
:10BDA80065EEA44AE4EE064AB0EE674AA4EE854A78
:10BDB800F4EEC46AF1EE10FAF0EE444A88BFF0EEF1
:10BDC800474AFDEEE44A14EE900A14EE906A98424F
:10BDD800A8BF1E468842B8BF0E4604EE906AF8EE29
:10BDE800E44A042ACCED034A3DF488AAD8ED104A67
:10BDF8009DED104A65EEA44AE4EE064AB0EE674AA5
:10BE0800A4EE854AF4EEC46AF1EE10FAF0EE444A64
:10BE180088BFF0EE474AFDEEE44A14EE900A14EEAD
:10BE2800906A9842A8BF1E468842B8BF0E4604EEE4
:10BE3800906AF8EEE44A052ACCED044A3DF45EAA7D
:10BE4800D8ED144A9DED114A65EEA44AE4EE064A7F
:10BE5800B0EE674AA4EE854AF4EEC46AF1EE10FA31
:10BE6800F0EE444A88BFF0EE474AFDEEE44A14EE8D
:10BE7800900A14EE906A9842A8BF1E468842B8BF3E
:10BE88000E4604EE906AF8EEE44A062ACCED054A1E
:10BE98003DF434AAD8ED184A9DED124A65EEA44A3D
:10BEA800E4EE064AB0EE674AA4EE854AF4EEC46AA8
:10BEB800F1EE10FAF0EE444A88BFF0EE474AFDEE84
:10BEC800E44A14EE900A14EE906A9842A8BF1E46FF
:10BED8008842B8BF0E4604EE906AF8EEE44A072A94
:10BEE800CCED064A3DF40AAAD8ED1C4A9DED134A4A
:10BEF80065EEA45AE6EE045AE5EE257AF4EEE76A12
:10BF0800F1EE10FAC8BFF0EE477AFEF794B99FED4C
:10BF18002E7AFFF70DBA2D4B4FEA890E5FEA9A0980
:10BF280001EB0E0C03EBC818A64400F0F38409F1EA
:10BF380001094FEA091908EB090008F110030CF18F
:10BF480010010EF1100213ED024A13ED035A13ED1E
:10BF5800016A13ED047A51ED024A51ED035A51ED8D
:10BF6800016A51ED047A64EE244A65EE255A66EEBC
:10BF7800266A67EE277A1033984242ED024A42ED6C
:10BF8800035A42ED016A42ED047A01F1100102F10F
:10BF98001002D8D1A9F11009C8440CEB0901CE440C
:10BFA8001AF0030A3EF419AEB8EC017AF1EC017A02
:10BFB80067EE277ABAF1010AEEEC017AF4D1FEF7BE
:10BFC8000CBE00BF0000024300000000283800201B
:10BFD800083C0020BAF1000F00F09583DFF868866E
:10BFE8009DED0C4AD8ED004A65EEA44AE4EE064AF7
:10BFF800B0EE674AA4EE854AF0EE444AB9F1000F64
:10C0080006D0F4EE446AF1EE10FAC8BFF0EE474AE3
:10C01800BDEEC77A17EE101ABDEEE47A04EE901A58
:10C0280017EE100A814200F361849842A8BF1846AF
:10C0380007EE100AB8EEC77ADFF810C6012A8CEDB1
:10C04800007A3DF460A998ED047A9DED0D4A25EE3D
:10C05800877AA4EE067AB0EE674AA7EE054AB0EEF4
:10C06800447AB9F1000F00F02A84F4EEC46AF1EEC4
:10C0780010FA40F3248408469842A8BF184607EEF1
:10C08800100AB8EEC77A022A8CED017A3DF43BA972
:10C0980098ED087A9DED0E4A25EE877AA4EE067A89
:10C0A800B0EE674AA7EE054AB0EE447AB9F1000F40
:10C0B80000F0FB83F4EEC46AF1EE10FA40F3F58366
:10C0C80008469842A8BF184607EE100AB8EEC77A85
:10C0D800032A8CED027A3DF416A998ED0C7A9DEDB1
:10C0E8000F4A25EE877AA4EE067AB0EE674AA7EEE5
:10C0F800054AB0EE447AB9F1000F00F0CC83F4EEB3
:10C10800C46AF1EE10FA40F3C68308469842A8BF05
:10C11800184607EE100AB8EEC77A042A8CED037A9F
:10C128003DF4F1A898ED107A9DED104A25EE877A36
:10C13800A4EE067AB0EE674AA7EE054AB0EE447A56
:10C14800B9F1000F00F09D83F4EEC46AF1EE10FA25
:10C1580040F3978308469842A8BF184607EE100A8E
:10C16800B8EEC77A052A8CED047A3DF4CCA898ED90
:10C17800147A9DED114A25EE877AA4EE067AB0EE80
:10C18800674AA7EE054AB0EE447AB9F1000F00F00D
:10C198006E83F4EEC46AF1EE10FA40F36883084641
:10C1A8009842A8BF184607EE100AB8EEC77A062AC2
:10C1B8008CED057A3DF4A7A898ED187A9DED124A02
:10C1C80025EE877AA4EE067AB0EE674AA7EE054A0E
:10C1D800B0EE447AB9F1000F00F03F83F4EEC46A80
:10C1E800F1EE10FA40F3398308469842A8BF184682
:10C1F80007EE100AB8EEC77A072A8CED067A3DF4E6
:10C2080082A898ED1C7A9DED134A65EE875AE4EEF4
:10C21800065AE5EE857AB9F1000F00F01683F4EEC0
:10C22800E67AF1EE10FA40F110830A469A42A8BF66
:10C238001A4604EE902AF8EEE44ACCED074AFDF7D8
:10C2480062B807EE903ADFEDEE6AB8EEE77A66EE8E
:10C25800A65A9FEDEC5A9FEDEC6ADFEDEC7AA5EE5D
:10C26800856A26EEA55AE5EE867AE5EE276A26EE79
:10C27800870AFFF756B8D8ED006ADDED0C4A65EE7F
:10C28800A66AE4EE866AF0EE674AE6EE854AFDEEB7
:10C29800E46A16EE90EA714500F316829E45A8BF3F
:10C2A8009E4606EE90EAF8EEE66A002E00F0398423
:10C2B800DFF898C3012ACCED006A3DF424A8D8ED34
:10C2C800046ADDED0D4A65EEA66AE4EE866AF0EED4
:10C2D800674AE6EE854AFDEEE46A16EE90EA714595
:10C2E80000F3EF819E45A8BF9E4606EE90EAF8EE61
:10C2F800E66A002E00F00A84022ACCED016A3DF4B9
:10C3080002A8D8ED086ADDED0E4A65EEA66AE4EEED
:10C31800866AF0EE674AE6EE854AFDEEE46A16EEB6
:10C3280090EA714500F3CA819E45A8BF9E4606EE75
:10C3380090EAF8EEE66A002E00F0AE83032ACCED10
:10C34800026A3CF4E0AFD8ED0C6ADDED0F4A65EE09
:10C35800A66AE4EE866AF0EE674AE6EE854AFDEEE6
:10C36800E46A16EE90EA714500F3A5819E45A8BFE0
:10C378009E4606EE90EAF8EEE66A002E00F082830A
:10C38800042ACCED036A3CF4BEAFD8ED106ADDEDAB
:10C39800104A65EEA66AE4EE866AF0EE674AE6EEB3
:10C3A800854AFDEEE46A16EE90EA714500F3808155
:10C3B8009E45A8BF9E4606EE90EAF8EEE66A002E75
:10C3C80000F0BA83052ACCED046A3CF49CAFD8EDA2
:10C3D800146ADDED114A65EEA66AE4EE866AF0EEAF
:10C3E800674AE6EE854AFDEEE46A16EE90EA714584
:10C3F80000F35B819E45A8BF9E4606EE90EAF8EEE4
:10C40800E66A002E00F07883062ACCED056A3CF433
:10C418007AAFD8ED186ADDED124A65EEA66AE4EE49
:10C42800866AF0EE674AE6EE854AFDEEE46A16EEA5
:10C4380090EA714572DC9E45A8BF9E4606EE90EADA
:10C44800F8EEE66A002E00F09F83072ACCED066A14
:10C458003CF459AFD8ED1C6ADDED134A65EEA65AD7
:10C46800E4EE865AE5EE857AFDEEE77A17EE902A35
:10C47800914203DC9A42A8BF1A46114607EE901A69
:10C48800F8EEE77A002E7FF42AAA069B002B7FF4A9
:10C4980026AA059B5B45B8BFF0EE477AFFF71FBA9F
:10C4A80077EEC76AF0EE477AFEF7A0BDBCF83430E5
:10C4B8009FED577A07EE903AF8EEE77A554B67EE1C
:10C4C800877AC3ED007AFCF779BE534B1E6816F0E5
:10C4D80080567FF4BAA8FFF7B3B8504BFCF7C5BE37
:10C4E8004F4B1B78032B00F011820023FEF7B2BEDE
:10C4F8009FED4C8AFFF72FBA9FED4A8AFFF703BAE0
:10C508009FED490ADFF8488125EE800A21F078FA84
:10C51800D4F8A861A8F80600FBF77DBE06EE901ACD
:10C528008EE707EE907AF8EEE78ADFED407A9FED26
:10C53800400A84F8847168EEA78A38EE800AFDEE16
:10C54800C07A17EE903A2033402B40F2CC819FED11
:10C55800350A304BFDEEE87A83ED010A17EE903A82
:10C568002033402B00F2BC81DFED327AF4EEE78A0B
:10C57800F1EE10FA40F3E581DFED2F6ADFED2F7A57
:10C5880001E0F0EE478AF4EEE78AF1EE10FA38EEB1
:10C59800E67AF6DCDFED2A7AB4EEE77AF1EE10FA05
:10C5A80040F1CC819FED246ADFED266A01E0B0EE10
:10C5B800677AB4EEE67AF1EE10FA77EE067AF6D4F8
:10C5C8009FED1B7AF4EEC77AF1EE10FA40F39281F0
:10C5D8009FED187A77EE677A27EEA76ADFED095A9A
:10C5E800DFED096A9FED097AE6EE256A67EE865A5D
:10C5F800A6EE267AE5EE877AC4ED627AFDF725BFC6
:10C6080084F9223F92E741B99730083C15A82ABE21
:10C618006F12833A9C000020383C00201044002010
:10C62800F2540020000000000000C84235FA8E3C99
:10C63800DB0FC93FDB0F4940DB0FC940E4CB164194
:10C64800DB0F49C0E4CB16C194330020083C00201E
:10C65800EC430020C049C14A8C46FEF7ADBA93EDC1
:10C66800000A05930791069221F0CAF9DFF814E34E
:10C67800DFF814C3DEF8ECE0DFF81083069AA8F8B8
:10C6880000008CFB0E3C4FEAEE7ECEEBAC1E07EEB4
:10C6980090EAF8EEE77A059B0799FDEEE77A17EE40
:10C6A800900AA8F80200FCF7E5BD06EE901AA6E687
:10C6B80006EE901A81E606EE901A5CE606EE901AEF
:10C6C80037E606EE901A12E606EE901AEBE5F4F756
:10C6D80053FCA34BDFF8B4821F78069B99F800201F
:10C6E800D4F8A861C01AA8F80400FEF754BCF4F7FF
:10C6F80043FC9B4BDFF894821F78069BC01AA8F86E
:10C708000200FEF7DCBBFDEEC74A0DF1300E9A467B
:10C71800DFF87CC2DFF87C8214EE901A0EEB8202FE
:10C728004B4606E07245E8EC014A0CF1100C3CF46B
:10C73800EAADDCED004ABEEC014A65EEA44AE6EE3D
:10C74800044AB0EE674AA5EE244AF0EE444A33B1F3
:10C75800F4EE446AF1EE10FAC8BFF0EE474AFDEE77
:10C76800E44A14EE909A494504EE901A04DCD14547
:10C77800A8BFD14604EE909AF8EEE44A002ED1D133
:10C7880006980028CED105985845B8BFF0EE474A1C
:10C79800C8E7F4F7F1FB069BDFF8F081D4F8AC9119
:10C7A800D4F8A861C01AA8F80200FEF781BA09985F
:10C7B8000DF09CF9FEF752BEDFED6A7AF4EEE76AF7
:10C7C800F1EE10FA40F39581DFED675A9FED676A45
:10C7D80001E0F0EE676AF4EEC66AF1EE10FA76EE62
:10C7E800E57AF6DCDFED626AF4EEE67AF1EE10FA4D
:10C7F80040F1C781DFED5C5A9FED5E6A01E0F0EE23
:10C80800667AF4EEC67AF1EE10FA77EEA56AF6D4F7
:10C81800DFED597AF4EEE76AF1EE10FA04DDDFEDA8
:10C82800517A77EEE66A12E5DFED547AF4EEE76ABC
:10C83800F1EE10FA44BFDFED4E7A77EEE66A06E5D0
:10C84800464800F1800CFEF78DBBFDEEE77A17EE47
:10C85800902A8A42FFF6EFACE8E4BDEEC77A17EEFD
:10C86800100A8842BFF6C1AC07EE101AC2E4BDEE4A
:10C87800C77A17EE100A8842BFF692AC07EE101A74
:10C8880093E4BDEEC77A17EE100A8842BFF663AC90
:10C8980007EE101A64E4BDEEC77A17EE100A884254
:10C8A800BFF634AC07EE101A35E4BDEEC77A17EEC2
:10C8B800100A8842BFF605AC07EE101A06E4BDEE72
:10C8C800C77A17EE100A8842BFF6D6AB07EE101AE1
:10C8D800FFF7D7BBA8F80600A5F8B460FCF794BB2F
:10C8E800DFED277A88E6F6F7FDFB32E607EE101A49
:10C8F800FFF7A0BB9FED217AF4EEC77AF1EE10FAAC
:10C9080044BF9FED1B7A77EE677A65E616F0FEFD69
:10C91800FCF772BB6146FFF743BB802011F0DAFFDA
:10C9280008B105F009FA0EF0A3F9FEF74CBD94F82A
:10C93800E031002B7BF4D8AEFBF7C3BEF0EE477AAC
:10C948003EE6B0EE687A25E61BF80330002B7EF44D
:10C958003AADFEF7D9BD00BFA839002060210020FC
:10C96800E8430020DB0F4940DB0FC940E4CB164108
:10C97800DB0F49C0E4CB16C1DB0FC93FDB0FC9BFD2
:10C9880000000000C4010020D34D6210EC430020D9
:10C9980094330020083C0020804A814B10681B68B3
:10C9A8009847089B9BED007AD3ED007A7D4BD7ED35
:10C9B800006A83ED020A7C4B67EE277A2B4427EE48
:10C9C8008C7AD3ED007A794B67EE277AF0EE665AC7
:10C9D800EDEE275A93ED006AB1EE467AB4EEE57AA9
:10C9E800F1EE10FA73DD724B1B78012B02D0192B74
:10C9F8007BF4F1ADDFED6F7AB4EEE7DAF1EE10FA21
:10CA0800CCBF01230023FBF7F1BDDFED6B7AF4EE19
:10CA1800E7DAF1EE10FA32DCDFED687AF4EEE7DA05
:10CA2800F1EE10FA2BD4664BD3ED007AB1EE677AAB
:10CA3800B4EEC7DAF1EE10FA46D4B4EEE7DAF1EE66
:10CA480010FA88BFB0EE67DA5E4BC7ED00BA1B6814
:10CA58009342BBF681ADFCF7A4BEDFF88091D9F80C
:10CA6800000005F03DF9584B1B780022022BC9F84D
:10CA780000207EF4A5AC04F063FBFEF7A1BC9FED9B
:10CA880053DAE1E7069800287FF47AAC0598584510
:10CA9800B8BFF0EE476A73E4069800287FF44EACFE
:10CAA80005985845B8BFF0EE476A47E445201BF0A3
:10CAB800EDFCFF201BF0EAFC45481BF0D3FC384690
:10CAC8001BF0E4FCFEF7ABBCB0EE47DABCE7B4EE13
:10CAD800E56AF1EE10FA8CBFB0EE657AB0EE467AF0
:10CAE80081E7802011F0F6FE00287DF4DFA8FEF72C
:10CAF80039BDF0EE667A75E6069800287FF484ACB6
:10CB080005985845B8BFF0EE476A7DE406980028B6
:10CB18007FF4F2AB05985845B8BFF0EE476AFFF7C7
:10CB2800EBBB069800287FF4C3AB05985845B8BFFF
:10CB3800F0EE476AFFF7BCBB069800287FF442ACCA
:10CB480005985845B8BFF0EE476A3BE4132B05D16A
:10CB5800B0EE480A20F054FFAAF80000B0EE480AE8
:10CB6800D5F814321B4898471B4B1B78132BB0EE93
:10CB7800408A7BF491AB20F043FFAAF80200FBF750
:10CB88008BBBF0EE676A43E6069800287FF45DAC3D
:10CB980005985845B8BFF0EE476A56E4583000206B
:10CBA8006C300020D43B0020FC320020643300208D
:10CBB800402E00200000964200C0F84400C0F8C48F
:10CBC8006033002044330020103E002000000000A5
:10CBD8008027030818640020E8430020E06B002049
:10CBE8002DE9F047B0F908400C81E4B2442C8AB032
:10CBF8000D46164600F0098407462FD9812C00F00F
:10CC0800538300F28280542C00F0AF8040F2B98048
:10CC18006E2C00F0C883802C40F0B580664B1C78E1
:10CC28000B3C14F0FF0412D0644F00220A26296836
:10CC38003B88481C28600E702968FF2B02F101020E
:10CC4800A8BFFF23481CA24228600B70EFDB012419
:10CC5800234620466B810AB0BDE8F087052C00F01A
:10CC6800C2831FD8022C78D040F2FE82032C00F039
:10CC78009083042C40F08780514928462246F6F7D5
:10CC8800F3F8504B28461978F6F71EF92A68002160
:10CC9800531C01242B602046234611706B810AB077
:10CCA800BDE8F087242C56D040F29482282C00F05E
:10CCB8003583382C67D10A68434B0124511C2960FD
:10CCC80014702A6805211019286011702A680A2131
:10CCD8001019286011702A68002110192860117035
:10CCE8002A6819781019286011702A68597810195B
:10CCF800286011702A68997813192B6023461170DF
:10CD080020466B810AB0BDE8F087A02C11D040F214
:10CD18008082B82C00F03B83FE2C34D12B4C04F1DC
:10CD2800080634F8021B2846F6F7CEF8B442F8D1C4
:10CD38008DE7274B08461968F6F7AEF8254B2846C5
:10CD48001968F6F7A9F8244B196828460124F6F75C
:10CD5800A3F823467DE7214BF6E70422204928461D
:10CD68000124F6F781F82346CAE70B6800215A1C0C
:10CD78002A6019702A68012413192B602346117040
:10CD8800BEE7522C82D029462046F6F7D1FE00286D
:10CD98007FF45DAF742C00F07A82772C24D13B6845
:10CDA8007A689A421BBF5A1C3A60014619780D4AA4
:10CDB80028461AF079FD4AE796430020B42400205B
:10CDC800956C0020023800201D6E0020EC430020E6
:10CDD800ACF7FF1FB0F7FF1FB4F7FF1F806F0020ED
:10CDE800682803087D6B0208F52C00F03B83292C8A
:10CDF8003E6801F07281392C01F05F81212C01F02D
:10CE08003C817A680B3C931BEF2C00F2F78301A15D
:10CE180051F824F029DB000805D6000805D60008DB
:10CE280005D6000805D6000805D6000805D600086E
:10CE380005D6000805D6000805D6000805D600085E
:10CE480005D6000805D6000805D6000805D600084E
:10CE580005D6000805D6000805D6000805D600083E
:10CE680005D6000805D6000805D6000805D600082E
:10CE780005D6000897DA000805D600087DDA00080C
:10CE880005D600085BDA000805D6000805D60008B4
:10CE980005D600082DDC000805D60008B7DB000819
:10CEA80005D6000885DB000805D600085FDB00080A
:10CEB80005D6000849DA000805D60008F5D90008A3
:10CEC80005D60008A9D9000805D6000805D6000827
:10CED80005D6000805D6000857CC000805D6000876
:10CEE8008DD9000805D6000805D6000821E00008FD
:10CEF80005D60008C7DF000805D6000805D60008D3
:10CF080005D6000805D6000805D6000805D600088D
:10CF180005D6000805D600083BE0000805D600083D
:10CF2800AFDE000805D6000805D6000871DE000847
:10CF380005D6000805D6000805D6000805D600085D
:10CF480005D6000805D6000805D60008A5DD0008A6
:10CF580005D60008FFDC000805D6000855DC0008E7
:10CF680005D6000825DF000805D60008FDDE000804
:10CF78006FD9000805D6000805D6000805D60008B0
:10CF880005D6000805D6000805D6000805D600080D
:10CF980005D6000805D6000805D6000805D60008FD
:10CFA80005D6000805D6000805D6000805D60008ED
:10CFB80005D6000805D6000805D6000805D60008DD
:10CFC80005D6000805D6000805D6000805D60008CD
:10CFD80005D6000805D6000805D6000805D60008BD
:10CFE80005D6000805D6000805D6000805D60008AD
:10CFF80005D6000805D6000805D6000805D600089D
:10D0080005D6000805D6000805D6000805D600088C
:10D0180005D6000805D6000805D6000805D600087C
:10D0280005D6000805D6000805D6000805D600086C
:10D0380005D6000805D6000805D6000805D600085C
:10D0480005D6000805D6000805D6000805D600084C
:10D0580005D6000805D6000805D6000805D600083C
:10D0680005D6000805D6000805D6000805D600082C
:10D0780005D6000805D6000805D6000805D600081C
:10D0880005D6000805D6000805D6000805D600080C
:10D0980005D6000805D6000805D6000805D60008FC
:10D0A80005D6000805D6000805D6000805D60008EC
:10D0B80005D6000805D6000805D6000805D60008DC
:10D0C80005D6000845D9000805D600082FD900085C
:10D0D80005D6000805D6000805D6000805D60008BC
:10D0E80005D6000805D6000805D6000805D60008AC
:10D0F80005D6000805D6000805D6000805D600089C
:10D1080005D6000805D60008D3D8000805D60008BB
:10D118009BD8000805D60008FFD7000829D70008C3
:10D128000DD7000805D60008F3D6000805D6000874
:10D13800CBD60008B9D600085FD6000805D6000887
:10D1480031D6000805D6000805D600080FD6000815
:10D15800D1D700086BD7000843D70008E7D50008E7
:10D16800C5D5000805D60008ADD5000805D60008C5
:10D1780005D6000805D6000805D6000805D600081B
:10D1880005D6000805D6000805D6000805D600080B
:10D1980005D6000805D6000805D6000805D60008FB
:10D1A80005D6000893D5000805D6000805D600085E
:10D1B8003BD5000805D6000805D6000805D60008A6
:10D1C80005D6000805D6000805D6000805D60008CB
:10D1D80023D50008202C7FF4D6AD0B688F4C591C42
:10D1E800627829601A702B682278591C29601A7095
:10D1F8002B68A278591C29601A7021892846F5F7EE
:10D2080063FE2B686279591C29601A702A68A17913
:10D218003EE5822C7FF4B7AD0B68814A814C1178CA
:10D228007E4A581C2860197011892846F5F74CFE6B
:10D238007D4B2A681B88FF2B02F10101A8BFFF2341
:10D2480029601370A16881F3100189B22846F5F7A7
:10D258003BFE216801F30F0189B22846F5F734FE39
:10D26800724B2A68197813E5012C7FF48CAD0B6892
:10D278000022591C29601A702B685A1C2A601C70DD
:10D288002A682421531C2B602346117038E53B681B
:10D298007A689A421BBF5A1C3A6001461978644A58
:10D2A80028461AF001FBD2E4624B1E780A3E16F0BB
:10D2B800FF063FF4CCAC604B604F1E4403F10108FD
:10D2C8000A2314E0502B00F0D486002421462A6853
:10D2D800501C286028461370F5F7F6FD21462846AD
:10D2E800F5F7F2FDB0453FF4B2AC18F8013B0A2B54
:10D2F800E8D1534A9468116804EB84044FF6FF722E
:10D3080064009442A8BF14469142A8BF114624EA7B
:10D31800E47421EAE171A4B289B2D8E70B68DFF8B6
:10D328004081484E591C022229601A702B68062732
:10D338005A1C2A601F702B680A22591C29601A700F
:10D348002B6801241A192A601C70B8F800102846A6
:10D35800F5F7BAFDB8F802102846F5F7B5FD2B68C1
:10D368001A192A601F702B685022191929601A701F
:10D378002B680022191929601A7031882846F5F798
:10D38800A3FD71882846F5F79FFD2346B8E42E4B88
:10D39800DAE40B685A1C0A601C700B680222591CDC
:10D3A80029601A7072E4204B0A681B881D4CFF2BF9
:10D3B800A8BFFF23511C29601370A16881F31001D5
:10D3C80089B22846F5F780FD204B28461988F5F7DD
:10D3D8007BFD216801F30F0189B228460124F5F786
:10D3E80073FD23468CE40B2219492846F5F73CFDCA
:10D3F800082218492846F5F737FD0124072216495F
:10D408002846F5F731FD23467AE4002A3FF41FAC9D
:10D41800124B13600124234672E400BF406D0020C4
:10D428000E440020AC530020F8430020F2540020A2
:10D438005D77020896430020F0010308A824002025
:10D4480070240020A4240020C8310020EC540020BF
:10D45800702803087C28030888280308613A000814
:10D46800E03D00203B687A689A4240F07186C24BE2
:10D47800FF221A704FF00009C04C1CF0E1FC49462D
:10D488002022BF4884F8009022F0C7FB8DF8049052
:10D498009DF80430072B00F2B986DFF82083B84FD7
:10D4A8004A469DF8043003EB430308EBC3035B7C57
:10D4B800E3B19DF8043003EB430308EBC3032021D9
:10D4C8005B699BB19DF8043003EB430308EBC3038E
:10D4D800586947F82200F4F785FD237857F82300A8
:10D4E800F4F742FF22780132D2B222709DF804305C
:10D4F8000133DBB28DF804309DF80430072BD0D906
:10D508002B68591C29601A70002E3FF4A0AB9D4B64
:10D51800336001242346FFF7F3BB9B4B1B78DB07E3
:10D528006CD40124F7F7EEFAF8F7D6F82346FFF79C
:10D53800E7BB731C3B6033780F2B5FD8B21C3A6093
:10D54800C3EBC303914A7178D154F11C3960134479
:10D55800B2785A70321D3A60F2789A70721D3A6049
:10D568003279DA70B21D3A6072791A71F21D3A6036
:10D57800B2795A7106F108023A60F2799A71012477
:10D5880006F018FF2346FFF7BBBB3846F5F75AFCF1
:10D598007F4EF0813846F5F755FC0124B0812346CB
:10D5A800FFF7AEBB3846F5F74DFC7A4A00EB800032
:10D5B8004300012413802346FFF7A2BB3846F5F742
:10D5C80041FC754E30823846F5F73CFC708238468F
:10D5D800F5F738FC0124B0822346FFF791BB3346A8
:10D5E800721C3A6013F8020B3B60F31C71783B60C5
:10D5F800B27812F05FFE00287FF429AB4FF0FF34B9
:10D608002346FFF77DBB3846F5F71CFC634E308098
:10D618003846F5F717FC70803846F5F713FC0124F7
:10D62800B0802346FFF76CBBDFF8948198F8003090
:10D63800002B3FF40CAB5A4E00243846F5F702FC99
:10D6480008F072FA98F80030A6EC010A01349C42FE
:10D65800F3DBFFF7FCBA0D2BD0D1731C3B60347899
:10D66800072CCBD8DFF85C8138460C26F5F7EAFBA7
:10D6780006FB04F608EB0604A0803846F5F7E2FB43
:10D68800E0803846F5F7DEFB3B6820811A46591CD6
:10D69800396012F8021BA1723A605B78E37238466F
:10D6A800F5F7B8FB012448F806002346FFF728BB26
:10D6B8003846F5F7C7FB3B4B012418802346FFF794
:10D6C8001FBB731C3B603078060600F1C1852E4BEA
:10D6D8001B78DC073FF5BBAA032828BF00200124DC
:10D6E800F7F7F4F92346FFF70BBB274B1B78D8074E
:10D6F8003FF5ADAA0124F7F7D7FAF7F7EDFF234670
:10D70800FFF7FEBA204B1B78DA073FF5A0AA264A96
:10D718001378012443F0040313702346FFF7F0BA8B
:10D72800194B1B78D9073FF592AA204B4FF4C872C2
:10D7380001241A802346FFF7E3BA3346721C3A6085
:10D748001B4A13F8021B11703B60114A73789370DF
:10D75800F31C3B600F4BB2789A7001242346FFF705
:10D76800CFBA144B144918684E2201241FF0D4FF75
:10D778002346FFF7C5BA00BF742300201F2D0020E1
:10D7880048580020F1350108FC6B0020382F002094
:10D79800F03D0020003E0020B06500201C34002031
:10D7A8007433002062220020403C0020FA6D0020E3
:10D7B800E06800209C6C00206C050308F0640020E1
:10D7C80096430020442E00203246731C3B60C44B15
:10D7D80012F8021B19703A6072785A70F21C3A609B
:10D7E800B2789A703846F5F72DFBBE4B0124D880E5
:10D7F8002346FFF785BA092B7FF700AFDFF81C83B4
:10D808003346721CD8F800403A6013F8022B227095
:10D818003B607378A370F31C3B60B378642BA8BF9C
:10D828006423321D63713A60F378642BA8BF6423C4
:10D83800721DA3713A603379E371B31D3B6073794C
:10D84800642BA8BF6423F21D23723A60B379E37096
:10D8580006F108033B60F37923713846F5F7F2FACD
:10D868007A683B686081D11A00290CDD591CD8F808
:10D8780000003960521A002A1978417203DD9A1C97
:10D888003A605B78437001241DF008FF2346FFF7D8
:10D8980037BA954B1868F31C02462136991E396031
:10D8A80013F8031C1170591E396013F8021C5170CB
:10D8B8003B6013F8011C91700333B34202F1030279
:10D8C800ECD107F0FDFFFFF7C2B9C3F34704122CF0
:10D8D8003FF694AEBCB10AAB0DF1020803EB440964
:10D8E8004646A9F126093846F5F7ACFA26F8020F9C
:10D8F800B145F8D17D4B38F8022F23F8022F464561
:10D90800F9D1112C09D87A4A6300023B134400214B
:10D91800223223F8021F9A42FBD1764A01231C4681
:10D928001370FFF7EDB9744E002338463360F5F7EE
:10D9380071FA012430602346FFF7E2B93346721CBE
:10D948003A6013F8024B3B60F31C70783B60B17887
:10D95800002C00F08884012C7FF479A91CF00AFDC2
:10D968002346FFF7CDB9654B1B7813F001017FF40F
:10D9780045AE731C3B60307801241CF04BFC2346F9
:10D98800FFF7BEB93346721C3A605D4A13F8021BB2
:10D9980091703B607378537001242346FFF7B0B948
:10D9A8000722B3FBF2F2C2EBC2041B1B7FF426AEC4
:10D9B800D2B202F1FF385FFA88F8002A3FF447A98B
:10D9C800DFF8409108F101081C46731C3B604D4B81
:10D9D80096F90010002693F902208A4203F1080301
:10D9E80000F0EF830136062EF5D107E6731C3B6085
:10D9F80033780E2B3FF602AEB21C3A6070780328DB
:10DA08003FF6FCAD4049062202FB03F28B18F41CDA
:10DA180058713C60B0788854321D3A60F2785A7078
:10DA2800721D3A6032799A70B21D3A607279DA7072
:10DA3800F21D3A60B2791A7101242346FFF760B9E2
:10DA4800731C3B60314B32785A7501242346FFF72B
:10DA580057B93846F5F7F6F92D4E30603846F5F7E0
:10DA6800F1F970603846F5F7EDF90124B060234606
:10DA7800FFF746B9274E002333603846F5F7CAF951
:10DA880033680124034333602346FFF739B9731C15
:10DA98003B603478132C3FF6B1ADB31C3B60707813
:10DAA80019F03CFF00283FF4A9AD1B4B027803F89E
:10DAB8002420F21C3A6003EB8403B2785A70321DBA
:10DAC8003A60F2789A70721D3A6007493279DA70D2
:10DAD800086801241DF070FD2346FFF711B900BF47
:10DAE800E83D00201C3400209C6C00204A57002090
:10DAF8004C57002070570020C8310020FC6B0020D4
:10DB08000C3E0020285F0020D4310020446A002009
:10DB1800A42C0020806F0020303E0020DC6D002007
:10DB28009549102B4FF0000228BF10230A604A6065
:10DB38008A60CA600A74002B3FF489A83A680139E0
:10DB4800134401323A6012F8010C01F8010F9A42AD
:10DB5800F7D1FFF77CB8721C3A6034781F2C3FF677
:10DB68004DAD052B7FF44AAD3846F5F753F9834B95
:10DB780043F824001DF0BAF8FFF769B87F4C04F1A8
:10DB880040063846F5F75EF93B68A4F88000591C52
:10DB98001A46396012F8021B84F882103A605B78E2
:10DBA80084F883300434B442EBD1FFF750B8731CC7
:10DBB800734C3B60337823723846F5F743F9A083FA
:10DBC8003846F5F73FF920833846F5F73BF93A68C8
:10DBD8006083531C3B601278E2747A68D31A032B73
:10DBE80000F317833B68D11A05290EDD5A1C3A60E9
:10DBF8001B78E3723846F5F70DF93B68E0605A1C6C
:10DC08003A601B7823743B687A68D21A002A7FF737
:10DC18001EA85A1C3A601B7884F821300124234638
:10DC2800FFF76EB8731C3B60564930780870D31AFA
:10DC3800002B7FF70CA8B31C3B607378003318BF28
:10DC4800012301244B702346FFF75AB8731C3B602D
:10DC58004D4CDFF84481337888F80530384626681B
:10DC6800F5F7F0F8308438462668F5F7EBF87A6867
:10DC78003B68F083D11A072915DD3846F5F7E2F835
:10DC8800A8F80A003846F5F7DDF8A8F80C00384679
:10DC98002668F5F7D7F8708438462668F5F7D2F87D
:10DCA8003B687A68B084D11A03290BDD3846F5F74A
:10DCB800C9F8A8F80E003846F5F7C4F83B687A6842
:10DCC800A8F81000D21A002A05DD591C226839600C
:10DCD8001B7882F82630F6F71FFF18F065F82B4BF3
:10DCE8001B68002B00F0DC822068012406F0F6FB9C
:10DCF8002346FFF705B83346721C3A60DFF8988070
:10DD080013F8022B88F802203B60214A73781370BD
:10DD1800F31C3B601F4CB3782371331D3B60F378D1
:10DD2800092BA8BF09233846A370F5F78BF83B6881
:10DD38007A682080D11A012905DD3846F5F782F87E
:10DD48003B687A68E0819A4207D05A1C3A601B788F
:10DD5800003318BF012388F80730F6F7DDFE3B686B
:10DD68007A689A423EF473AF5A1C3A601B78E370A3
:10DD780001242346FEF7C4BFCC3D0020C053002039
:10DD8800446A00202C3E00209C6C0020143E002099
:10DD9800E43D0020B0650020E06800203846F5F733
:10DDA80051F804460DF0D4FBFF283EF450AF3F2C49
:10DDB80000F25F820DF12808002308F8243DE608E8
:10DDC80041460DF103008DF8033001360DF0A0FB3C
:10DDD8009DF80330F6B204F00704B34204F10104DD
:10DDE80003D19DF80430A34203D0214630460DF0FC
:10DDF8009BFB3B687A68D21A012A7EF728AF5A1C27
:10DE08000AA83A6000221C7800F8252D0DF074FB52
:10DE18009DF80330A3420AD0BC4B1B683BB19A79EA
:10DE2800A24204D31B681B690BB1204698473B6884
:10DE38005A1C3A60404600221C788DF804200DF0E8
:10DE48004FFB9DF80430A3423EF401AFAF4B1B6873
:10DE5800002B3EF4FCAE1B685B69002B3EF4F7AE6A
:10DE680020469847FEF7F3BEA94B1B78012B3EF6D8
:10DE7800EEAE3346711C3960DFF8CC8213F8021B12
:10DE880088F80210F11C3B60531A012B7078396036
:10DE980040F311823846F4F7D5FF0124A8F80000B2
:10DEA8002346FEF72DBF731C3B6096F80080B8F13F
:10DEB800110F3FF6A3ABB31C3B60964C737804F884
:10DEC80018303846F4F7BEFF40F6CA039842A8BF98
:10DED800184640F2EE23984204EB4801B8BF1846B2
:10DEE8000124A0F2EE222346192092FBF0F24A7098
:10DEF800FEF706BF3346721C3A60874A13F8021BC6
:10DF0800D1703B60854A73785371F31C3B60844B36
:10DF1800B278DA7001242346FEF7F2BE3846F4F7E9
:10DF280091FF3846F4F78EFF3846F4F78BFF3846F2
:10DF3800F4F794FF3B687B4C1946581C22683860FC
:10DF480011F8020B82F82C003960597882F83610E3
:10DF5800D91C39609B7882F837303846F4F77EFF51
:10DF68003846F4F77BFF3846F4F778FF38462668DA
:10DF7800F4F768FF708738462668F4F763FF3B6854
:10DF88007A683087D11A01290ADD591C226839605C
:10DF98001B7882F82E303846F4F760FF3B687A68C1
:10DFA800D31A032B09DD38462668F4F74BFF708631
:10DFB80038462668F4F746FFB086206881E4731C6B
:10DFC8003B60594B3278DFF884811A700023C8F817
:10DFD80000303846F4F71EFF3A68D8F80030534945
:10DFE800534C0343501CC8F80030386013780B7248
:10DFF8003846F4F727FF20603846F4F723FF6060BF
:10E008003846F4F71FFFA0603846F4F71BFF384680
:10E01800F4F718FFFEF71BBE464B06F10801013660
:10E028003E6016F8012C03F8012FB142F7D1FEF734
:10E038000EBE3346721C404C3A6013F8022B227114
:10E048003B60737863713846F4F7FCFE3B682080C8
:10E058005A1C3A601B78A3713846F4F7F3FE3B6804
:10E0680060805A1C3A601B78E37101242346FEF74E
:10E0780047BEBC683968FFF73FB93346721C3A603F
:10E088002E4C13F8022B62703B6073782370F31CDC
:10E098003B60B378A3703846F4F7D4FE3B68208120
:10E0A800591C1A46396012F8021B61713A605B7894
:10E0B800A37101242346FEF723BE731C3B6033780B
:10E0C8000A2B6DD03846F4F7C9FE3846F4F7C6FE79
:10E0D8003846F4F7C3FEFEF7BABD731C3B603378CD
:10E0E8000A2B0ED0502B8FD13846F4F7ABFE144EC6
:10E0F80030803846F4F7A6FE012470802346FEF7E8
:10E10800FFBD3846F4F79EFE0E4EF1E7643F00204F
:10E118004B6F00201C590020F03D0020FC560020C9
:10E12800003E00209C6C00202C3E0020446A002009
:10E13800A42C0020436A002034340020406D0020C5
:10E14800A4240020E03D00204E6F0020806F0020B6
:10E158005A1C19463A605E4811F8022B0270396061
:10E168005B784370042A04D9FF2A7EF48FADFFF749
:10E1780081B958490978994205D8022A7EF486ADB2
:10E18800FF2B7EF483AD2B6801241A192A601C70BA
:10E19800002E3EF45CAD504B33602346FEF7B0BD15
:10E1A800B31C3B604D4B72781A70F21C3A60B2781F
:10E1B8005A70321D3A60F2789A7001242346FEF7AD
:10E1C8009FBD09EBC60A38468AF80210F4F73AFEF2
:10E1D8003B6829F836001A46591C396012F8021BA8
:10E1E8008AF803103A605A788AF80420DA1C3A60F0
:10E1F8009A788AF806201E1D3E600134DB788AF87A
:10E208000530A0457FF4E1ABFEF721BD4A46FFF794
:10E2180077B93846F4F716FEA0843846F4F712FEAC
:10E228003B687A68E084D11A03297FF7DCAC1A4688
:10E23800591C396012F8021BA1773A605B7884F8A0
:10E2480020303846F4F7FEFD3B687A686084CAE4FB
:10E2580000F07F00032828BF002001241CF0A6F846
:10E268002346FEF74DBD012407F096F92346FEF735
:10E2780047BD0DF1040840460DF026F9BDF80430FD
:10E28800A3423FF4B6AD164B1B68002B3FF4B1AD6B
:10E298001B689B69002B3FF4ACAD20469847A8E566
:10E2A80010481149114A124B036001240B60136096
:10E2B8002346FEF725BD0F4BB1781A88012412FBBF
:10E2C80000F2234692FBF1F2A8F80020FEF718BDF1
:10E2D8007423002096430020793A00081D6E002020
:10E2E800643F0020B02F0020043000206C30002054
:10E2F800F10600084E3C00202DE9F04F2DED028B71
:10E30800984B994A1C7893B000F59C41203181467E
:10E3180006911160002C00F08686944A126890429B
:10E3280040F28A80924A93491768934DDFF888B281
:10E338000492013C02911C7007F48057002F40F0B2
:10E348008880029B5B7D002B40F03786049B1B680E
:10E358001E0401F10B81894B99459BF8023000F2AC
:10E368000A85002B40F00B85854B0593049B1F689D
:10E3780017F4805940F0C585029BB5F906605B8BA0
:10E388009E42B4BF002601267E4B1B6813F08053C3
:10E3980069D0059A127812F001026AD002987A4977
:10E3A800408C91ED037A039107EE900AF8EEE77A34
:10E3B800B4EEE77AF1EE10FA81F2A081002E60D176
:10E3C800724C94F8A01000295BD17148714900681B
:10E3D80090F82D0000240C604C608C606E49002879
:10E3E80050D10870002A51D0F8064FD56B4A1278E0
:10E3F800D1064BD4B9F1000F48D1002B46D17A028F
:10E4080044D4674B1B78002B01F02187654B9B7820
:10E41800002E41F0E5873BB1634A644B12681B68E4
:10E428009B1A002BC1F296871020584C15F08AF8D9
:10E43800012384F8A13029E04D4B4E4A1F6804930C
:10E4480007F4805702924C4DDFF86CB1002F3FF46F
:10E4580078AF00214B48F4F71DFF00287FF471AF17
:10E4680012F00EFD6DE77C0293D4059A127802F043
:10E478000102464C002184F8A01043490391002E64
:10E48800A3D0454901200870002AADD1484B1A781D
:10E49800002A50D10299B5F900E0488B898BB5F96B
:10E4A80002407045B4BF8027002747F040037145FC
:10E4B800D8BF3B469B0843F08007A042B8BF3B4605
:10E4C80043F04007A142C8BF3B469B08B5F904404A
:10E4D800B5F9067043F0800EA042B8BF734643F00A
:10E4E800400EA142C8BF73469B0843F0800E274CDC
:10E4F8008742C8BF734643F0400E94F8A2C08F42CB
:10E50800B8BF73469C4501F0EF82A4F8A42084F8B4
:10E51800A620234984F8A2300F78002F01F06F82DB
:10E528005F2B01F0BB826F2B01F04481059B1B78A8
:10E53800DE0741F10881049B1B6803F00403002BEC
:10E5480040F07E860DF140081A4C0022C8F80420DD
:10E5580004F15009109240F6330A192740F2833625
:10E568002FE000BF7C580020485700207858002032
:10E5780004690020446A0020D8520020404B4C0017
:10E58800FC6B0020383C0020104400207823002039
:10E598009C6C0020E03B002040230020403C0020F1
:10E5A800DE1500200C3E0020A46100201857002032
:10E5B8005D6B0020303E0020506D002004344C4537
:10E5C80020D0A278E3789A4217FB0260F6D26178ED
:10E5D800043117FB036235F911305345A8BF534680
:10E5E800B3F5617FB8BF4FF461739842E6DA9A4297
:10E5F800E4DB21782429E1D840460434F4F73AFED4
:10E608004C45DED1674A684B177898E8030083E8E1
:10E618000300002F00F07685644B069362480121C1
:10E62800F4F738FE002840F0B3829BF80330002B43
:10E6380040F0AE825E4B07935E4C23881EB226F0F4
:10E6480001061FFA86F84345A4F8008000F0ED871C
:10E65800594E4FF002090E2014274FF0FF0A86F892
:10E668000090777086F802A014F06CFF49464E4877
:10E67800B4F80080F4F70EFE002841F0DB8128F0A2
:10E6880002039BB2434523800BD04B4B1421FF223E
:10E6980002260E201E7059709A7014F053FFB4F8B9
:10E6A8000080464B464A19785068099318F0030FC2
:10E6B80008BF81F00201C1F340010892F3F75AFE46
:10E6C80024213948F4F7E6FD30B9059A137859073B
:10E6D80044BF23F004031370079B1B6813F00A0F51
:10E6E80024D005213048F4F7D5FD002800F0D38761
:10E6F8002688770741F1F4802B480621F4F7CAFDF4
:10E70800002800F0B587700641F1C8800721264827
:10E71800F4F7C0FD50B12B4B2B4AB3F904302B4909
:10E7280082FB0302DB17C3EBA2030B800C211E48FC
:10E73800F4F7B0FD2288002800F04A8242F4807382
:10E748009A42238009D01C4B02201421FF22187002
:10E758000E2059709A7014F0F5FE1D4B1B78082B8B
:10E7680000F042820E2B00F03F82049B1B68590583
:10E7780061D5184B1B79002B00F0258114210A481C
:10E78800F4F788FD002840F0238111F041FA0120B8
:10E7980014F01AFE00284ED0DFF83C9000264FF007
:10E7A800CC0A1EE0756C0020383C0020DC6D00208F
:10E7B800C46C0020EE5400203C340020B4640020D7
:10E7C800B8640020206D0020676666661457002034
:10E7D8002C3E002000440020284F0020DEB2022EEC
:10E7E80029D80AFB06F8731C59F80870002FF5D1D0
:10E7F800C378D04A90F9020052F8233001970322D7
:10E80800009201213A4614F02FF9034606EB460020
:10E8180000EB0010079353B1394609EB8000CC2276
:10E8280021F0FBF9079B49F808300136F6B215F0DC
:10E83800C3FE0028D3D1059B1E7816F0010600F010
:10E848000382BD4B01221A70069BB5F906101B689E
:10E85800BA485A8901279142077080F2DB81B84B88
:10E868004FF07E521A60B74A029BB5F900E01F8B41
:10E8780092F90430107892F801C0002BAEEB070330
:10E8880014BF01224FF0FF32002BB8BF5B42B3F533
:10E89800FA7FA8BF4FF4FA73984280F2B8811B1A26
:10E8A80007EE903AF8EEE77A039BBE45C3ED007A8F
:10E8B80003DAF1EE677AC3ED007AB5F902E0AEEB60
:10E8C8000703002BB8BF5B42B3F5FA7FA8BF4FF42C
:10E8D800FA73984280F24C821B1A07EE903AF8EECF
:10E8E800E77A039B7745C3ED017A03DDF1EE677A9A
:10E8F800C3ED017AB5F90400C31B002BB8BF5B4216
:10E90800B3F5FA7FA8BF4FF4FA736345CCBFA3EB06
:10E918000C03002302FB03F307EE903A039A049BCF
:10E92800F8EEE77AB842C2ED027ABCBFF1EE677A38
:10E93800C2ED027A1A6812F4805200F0F681B1F53D
:10E94800FA6F814BA8BF4FF4FA61B1F57A7F187856
:10E95800B8BF4FF47A71A1F57A71002840F0FE81B2
:10E968007A4D7B4885FB013ECB17C3EB6E1303F151
:10E97800010E6FF0630C30F91EE030F913000CFB48
:10E988000313AEEB000103FB01F385FB0315DB1753
:10E99800C3EB651303441BB207EE903A039BB8EE32
:10E9A800E78A83ED038A002A40F07F8323885B0689
:10E9B80024D4002E40F0B0801DF051F813B0BDEC07
:10E9C800028BBDE8F08F059B1B78DA077FF5DDAE7B
:10E9D8003C200FF07FFF00283FF42DAF03F0ACF987
:10E9E8003C200FF019FF00283FF425AF03F0A4F9ED
:10E9F8003C200FF011FF0028F0D11CE7554B564A78
:10EA0800B3F904305549DFED566A09889FED557A08
:10EA180082FB0302DB17C3EBA2035B1A1BB207EEF0
:10EA2800903AF8EEE77A67EEA67A77EE876ABDEE57
:10EA3800E66A16EE103A2033402B40F26E87BDEEA0
:10EA4800E77ADFED496A17EE103A2033402B00F2DF
:10EA5800B2879FED467AF4EEC77AF1EE10FA41F3E9
:10EA6800F382DFED435A9FED436A01E0F0EE477A07
:10EA7800F4EEC67AF1EE10FA37EEE57AF6DCDFED61
:10EA88003E7AB4EEE77AF1EE10FA41F1D982DFED81
:10EA9800385A9FED3A6A01E0B0EE677AB4EEC67A6A
:10EAA800F1EE10FA77EE257AF6D49FED2E7AF4EE91
:10EAB800C77AF1EE10FA00F339869FED317AF4EE59
:10EAC800C77AF1EE10FA44BF9FED2B7A77EE677A9A
:10EAD80067EEA75A9FED2B5A9FED2B6A9FED2B7A75
:10EAE800A5EE856A27EEA55AA5EE867AE5EE077AA1
:10EAF800039A92ED016AD2ED005A27EEC67A65EEC6
:10EB0800A77AA5EEA67AE6EE267A82ED007AC2ED1D
:10EB1800017A002E3FF450AF099B1978089B01F049
:10EB280001011868F3F726FC13B0BDEC028BBDE8B1
:10EB3800F08F00BFA0200308FD6B00207822002082
:10EB48001C230020E83D0020E42400201F85EB5111
:10EB5800E06D0020206D002067666666145700206F
:10EB680035FA8E3CDB0FC93F00000000DB0F49403F
:10EB7800DB0FC940E4CB1641DB0F49C0E4CB16C11B
:10EB8800DB0FC9BF92E741B99730083C15A82ABEE8
:10EB9800B64B07931B6898077FF54EADB44CB4F895
:10EBA800008018F0010F7FF46AAD48F00103984522
:10EBB80023803FF464ADAF4B022214211A700E205B
:10EBC800FF2259709A7014F0BDFCB4F8008056E525
:10EBD80022F480739BB29A4223807FF4B4ADA64B93
:10EBE8001B78082B7FF4BEAD228822F040039BB22D
:10EBF8009A4223803FF4B9AD9E4B02201421FF2294
:10EC080018700E2059709A7014F09CFCADE5DFED79
:10EC18009B7A49E6B1F5FA6F80F21684187A8B1A56
:10EC280003FB00F3C2F5FA6293FBF2F3C3F164034A
:10EC380007EE903AF8EEE77A9FED917A914B67EEFE
:10EC4800877AC3ED007A0EE68F4B1B780793002B6B
:10EC58007FF4FAADDFF868A2DFF868921AF8030CBF
:10EC680099F800805146AAF103071CF075FC0028AA
:10EC780000F0F383079BB8F1000F53D107F10801A7
:10EC880078791CF069FC002841F028827F49B87A1D
:10EC98001CF062FC002800F0F483B8F1020F41F088
:10ECA80020827B49F87B1CF057FC002841F01C822D
:10ECB8007849387D1CF050FC002800F0F483B8F146
:10ECC800040F41F002827449787E1CF045FC00284C
:10ECD80041F0FE817149B87F1CF03EFC002800F02D
:10ECE800F483B8F1060F41F0F6816D4997F82300D7
:10ECF8001CF032FC002840F0BF876A4997F82800CA
:10ED08001CF02AFC002800F0F483B8F1080F40F04A
:10ED1800C487654997F82D001CF01EFC00283FF4B5
:10ED280093AD09231A4600F0A9BF029B588B814274
:10ED3800C0F29183B1F5FA6FD4BFC0EB0101C0F501
:10ED4800FA614FF47A7303FB01F1584B1D78C0F553
:10ED5800FA60B1FBF0F1002D3FF402AE5B78544845
:10ED680001FB03F380FB0301DB17C3EB6111F7E53C
:10ED7800DFED427AB5E513B901238BF802304D4B2C
:10ED880005931B201F789BF821601CF00FFC012EB7
:10ED980007F00109824600F07D8607F0020303931D
:10EDA8009BF82030DFF82081434C052B00F29C8033
:10EDB800DFE813F08C0050000600DD000101BF0001
:10EDC800012E04BF05238BF82030B9F1000F00F0A5
:10EDD8001581029B394FB3F91810B8F8003000229A
:10EDE80061F30F0263F31F42002361F30F0361F322
:10EDF8001F436A603968DBF814202B608A42C0F030
:10EE08006484012E41F0F88203229BF8203003929B
:10EE1800CBE71CF0F7FB012808D1284FB8F80230DF
:10EE28003A68642101FB0323CBF81030BAF1000FD4
:10EE380004D098F80630002B40F09080012E53D073
:10EE48001E4FDBF810203B689A42C0F093860123DE
:10EE58008BF82030012E6CD098F80730012B00F089
:10EE6800D78007F0F1FB9BF820309EE7C46C0020A8
:10EE7800EE5400203C3400202C3E0020000000000E
:10EE88000AD7233C1C230020FD6B0020C832002039
:10EE9800CD320020D2320020D7320020DC320020D0
:10EEA800E1320020E6320020EB320020E42400208A
:10EEB8001F85EB51FC6B0020746D0020A4610020BD
:10EEC800BE320020A400002034340020B9F1000F25
:10EED8009FD14FF48060BAF1000F00F0C68314F0A0
:10EEE80041FC0023CBF81030039B002B3FF43EAAD3
:10EEF800039814F027FB049B1F6817F480593FF40C
:10EF08003BAA1D21BB48F4F7C5F900287FF434AAB1
:10EF1800B94A029BD2881B8BB5F90660991A8E42B2
:10EF280040F3338613449E42B4BF00260126FFF700
:10EF38002BBAB24F3A68B8F80230642101FB0323B8
:10EF48004FF480600022CBF810308BF820208BF82B
:10EF5800032014F0EFFB9BF8203026E707F074FB42
:10EF680003224FF47A738BF82020CBF81C30A34F80
:10EF7800238843F00203238011F082FF3A68DBF80C
:10EF88001C3013440422CBF818308BF82020012EB3
:10EF980040F0FE853B68DBF818209A42A4D2984BD3
:10EFA800187818B91CF002FB00289DD1238823F09B
:10EFB80002032380BEE7914FE9E7029A013BD27D25
:10EFC80035F91330002A40F07B83A3F57A73B3F543
:10EFD8007A7FA8BF4FF47A7323EAE37307EE903A77
:10EFE8009FED887AF8EEE77A67EE877A864AFCEE34
:10EFF800E77A17EE903A1380FFF7ADB97F4F3B6879
:10F0080047F230520323CBF81C208BF82030AFE7AF
:10F0180007F01AFB032240F6B8338BF82020CBF810
:10F028001C30764FA4E7794F3B78002B01F01C8009
:10F03800774BDFF8F881DFF8F8B1DFF8F8A1029331
:10F0480045465E46039099460EE019F80410984725
:10F05800032C28DC88B93B782AF8020F01349C423B
:10F0680005F1040580F21081072CE1B23046DBF887
:10F078000430EADD984700B2EDE738F824206B88C1
:10F08800801A4FF47A719B1A01FB00F040F6CA020D
:10F0980090FBF3F00844904240F2EE23A8BF1046DC
:10F0A8009842B8BF184600B2D5E71D215148F4F779
:10F0B800F1F800283FF47AAC9BF80330002B7FF47A
:10F0C80075ACDFED547A544938EE678AC7F5FA63B0
:10F0D800FDEEC87A1BB2CDED027ABDF90820120305
:10F0E80081FB0201D217C2EBA11203FB02F343F327
:10F0F8000F333B4407EE903A039BF8EEE77AC3EDF3
:10F10800037A53E4DFF830A1DFF83081434C0AF189
:10F118005A064FF0010951461AF8010C1CF01CFA66
:10F12800F8B19AF804009AF802309AF803E000EB74
:10F13800400104EB8101013BD1F8B42003EB430308
:10F14800434493420DD094F8E02081F8B0E009FAE6
:10F1580000F022EA0000C1F8B430C1F8B87084F8B1
:10F16800E0000AF1060AB245D5D12D4B069319469F
:10F17800224A2C4B2C4C09681B78D2F80090089135
:10F188000793A4F1B00A002663685BB31F784FB3F6
:10F19800A268A9EB0202002A0ADB9AF8E020012102
:10F1A800B14022EA010209F5FA718AF8E020A1606B
:10F1B800079ABAB1227859780432D2B2002940F0BD
:10F1C800A382029935F91220098B01F1C800824205
:10F1D80040F3A2849AF8E0109A7841FA06F3D90726
:10F1E80040F145850136042E04F10C04CCD1FFF71B
:10F1F80015BA00BF383C00201C340020A461002050
:10F20800DE150020AAF1823FEC540020D0580020DF
:10F21800446A002000007A44D34D6210782300200D
:10F22800DC6D0020BD54002028240020E858002070
:10F23800286D002076230020D5310020F401030832
:10F24800B24C94F8AA3053B1059B1B78D80706D561
:10F25800029BB5F906205B8B9A4200F3AE8411211C
:10F26800AB48F4F717F8002800F0368294F8AE306F
:10F278002BB994F8A83013B93223A4F8AC30012381
:10F2880084F8AE30FFF75EB9DDF80C90A14A04921D
:10F298001146A14A096842F2010AA2FB092B11EAA8
:10F2A8000A0A4FEA9B1B00F013829C4D9C489D4C18
:10F2B8009D4A95F800E0007884F800E01070BEF1EF
:10F2C800000F04D0984A92F800E08EF0010E8F4C9F
:10F2D8000F2084F82400002B00F07183934B0B93CC
:10F2E8001B780A931E463B78029F914AB7F824C0C0
:10F2F800DFF8708209903D46FF8C08973746A2FBDD
:10F30800066252082D8B0E9502EB420294F82550A6
:10F318000C95BA1AD2B201F48051079204F128066A
:10F328000BF596726746834DCDF80CE0A44654461B
:10F33800DDF830A00F9100200592CDF834909E465C
:10F34800039B002B00F04F823CF910101FFA81F943
:10F35800B9454FEA400203D3089B994540F285829C
:10F3680058F820108B4580F04782A95E002C40F0A9
:10F378005B8201307045A95206F10606E0DB099868
:10F388006D4ADDF834908CF824000F286446514605
:10F398000CBF01210021734684F825A0117000F0EC
:10F3A8001483DFF8C4B1654E654F34883868DBF8DC
:10F3B8000810DBF80420CBF80C0044F00404401AD1
:10F3C8009042574F3480584C4FF0010188BF0022BB
:10F3D8003970217088BF8BF82120002B00F00A8338
:10F3E800049A02991768574EB1F824C0B1F818E08A
:10F3F800504817F48057344640F02E8339460EE0C3
:10F40800627802EB820202EB820202F2EE2292B2F0
:10F4180001318B4220F8022B04F102040ED016F8B9
:10F428001120002A00F02582022AE9D00131028841
:10F4380020F8022B8B4204F10204F0D10B9A1378C6
:10F4480001331370FEF77ABF1B7AC3F1640307EE2A
:10F45800903AFFF7EFBB114677E40AF10501787996
:10F468001CF07AF800283FF411ACB8F1010F40F015
:10F47800358607F10D01B87A1CF06EF8002840F0C7
:10F4880030863149F87B1CF067F800283FF410AC4F
:10F49800B8F1030F40F028862C49387D1CF05CF841
:10F4A800002840F012862A49787E1CF055F800287A
:10F4B8003FF410ACB8F1050F40F00A862549B87F33
:10F4C8001CF04AF8002840F00686234997F82300E4
:10F4D8001CF042F800283FF410ACB8F1070F40F0D8
:10F4E800CB831E4997F828001CF036F8002840F016
:10F4F800D4831B4997F82D001CF02EF800283FF400
:10F50800A3A9B8F1090F3FF49FA90AE478230020C2
:10F51800383C002004690020D34D62102457002095
:10F52800A0050020BD540020A10500207D58002022
:10F53800ABAAAAAAD8520020926D0020746D0020B0
:10F54800A46100201C590020CD320020D2320020B6
:10F55800D7320020DC320020E1320020E6320020E1
:10F56800EB32002080580020506D0020CF4CD4F89A
:10F578008830A9EB0303002BFEF6EDAECC4A94F8D5
:10F588008C30517C069AC4F888200133C94A029EFF
:10F5980032F81120B17D03F00F0384F88C30234436
:10F5A80092B292FBF1F283F8902094F8901094F8BC
:10F5B800912094F8923094F89C000A4494F893109F
:10F5C800134494F89420194494F895300A4494F814
:10F5D8009610134494F89720194494F898300A44E4
:10F5E80094F89910134494F89A20194494F89B308D
:10F5F8000A44134494F89D1094F89F20184494F8F2
:10F608009E3001440B441A4442F30B12642AF17DE4
:10F61800A8BF642213B209B1C2F1640307EE903A9D
:10F628009FEDA57AF8EEE77ADEE40221A348F3F726
:10F6380031FE00283FF423A8268018F0020F7FF43B
:10F6480030A848F00203434523803FF42AA89C4B86
:10F65800022214211A700E20FF2259709A7013F09A
:10F6680071FFB4F80080FFF71CB814F063F838E4B1
:10F6780026F040039BB2B34223803FF447A8904B47
:10F6880002201421FF2218700E2059709A7013F06E
:10F6980059FFFFF73BB8238823F00406B6B2B342FC
:10F6A80026803FF429A8864B022214211A700E20C6
:10F6B800FF2259709A7013F045FF2688FFF71CB88F
:10F6C800C3F53B6308331BB27FE40323039397E43A
:10F6D8007C4A92F800E0F2E594F8A830002B3EF45A
:10F6E80031AF059B1B7813F001037EF42BAF012289
:10F6F80084F8A83084F8A920FEF724BF6B4C0121B8
:10F7080084F8A010FEF7BDBE012900F05C849AF8C9
:10F71800E0200123B34001361343042E8AF8E03079
:10F7280004F10C047FF430ADFEF778BF9FED667AE4
:10F7380077EE677AFFF7CCB9059B644A1B781060AF
:10F74800DB0700F1778294F8A60000287EF4F3AE78
:10F75800B4F9A430322B7EF7EEAE94F8A220012142
:10F76800572A84F8A61000F0DB84049B1B6813F06A
:10F77800040302D05A2A00F089855D2A00F0258505
:10F788005B2A00F04B855E2A00F05385562A00F06C
:10F798006E85972A00F05185A72A40F0DD844C49F0
:10F7A800049B0A781B6842F004020A7003F0040301
:10F7B800FEF7C5BEB2F5FA7FFEF6BDAE94F8A620F8
:10F7C800002A7EF4B8AE059B1B780121DF0784F878
:10F7D800A61000F1B98410F099FE049B1B6803F091
:10F7E8000403FEF7ACBE002F3DD058F820108B451F
:10F7F8004FEA4002FFF4B9AD364B995C03EB0209BE
:10F80800002900F00981022946D199F8011001EB7D
:10F81800810101EB810101F2EE2189B2032832DD79
:10F8280009B2002C3FF4A5AD079B26F81310BAF1D6
:10F83800000F03D10A9B022B7FF69BADB6F800A000
:10F848007188B6F80490244B514489440FFA89F919
:10F8580083FB0931214BA1EBE97123F8029009B22E
:10F868004FF0010A85E539464200059B48F82030EB
:10F878007CE5CAB2022A04D9032A7FF4D7AD6246CE
:10F88800C6E57246C4E5012303FA00F9099B23EA99
:10F89800090309B2099369E5A95ABFE746F040038D
:10F8A800B34223807FF4EBAEFEF730BF782300200D
:10F8B800AC610020C861002014AE2341383C002010
:10F8C8003C340020BD540020DB0F49401C57002069
:10F8D800403C00201C59002056555555E82300206F
:10F8E80046F004039E4223800AD0BB4B0222142117
:10F8F8001A700E20FF2259709A7013F023FE268882
:10F90800B64BB74AB3F90430B64982FB0302DB179A
:10F91800C3EBA2030B80FEF7EFBEF4EEC77AF1EE5D
:10F9280010FA40F39E83DFEDB05A9FEDB06A01E014
:10F93800F0EE476AF4EEC66AF1EE10FA36EEE57AB2
:10F94800F6DCDFEDAB6AB4EEE67AF1EE10FA40F1E0
:10F95800AB83DFEDA55A9FEDA76A01E0B0EE667AAA
:10F96800B4EEC67AF1EE10FA77EE256AF6D49FED7A
:10F97800A27AF4EEC76AF1EE10FA40F3A9809FED7F
:10F988009F7A77EE666A66EEA65A9FED9D5A9FEDBE
:10F998009D6A9FED9D7AA5EE856A26EEA55AA5EE8D
:10F9A800867AE5EE076ABDEEE77A17EE103A20335D
:10F9B800402B7FF64EA8DFED957AFFF799B894496A
:10F9C800944A0B91944D012111701B219348039384
:10F9D800F3F760FC039B00287FF4E3ACDFF850B238
:10F9E8008F4FDBF80C203B68CBF808309B1AC82BEC
:10F9F80000F25D83049B1F6807F480571EE53946B3
:10FA08008648F3F747FC00283FF496AE84F8A770C1
:10FA180010F07CFDFEF78ABDC1B2022940F2D18206
:10FA280003297FF439AF0E9B19460F9B002B08BFA3
:10FA38003946F3E628F0010292B2424522803FF4AB
:10FA4800FCAD0E2086F80090777086F802A013F0BF
:10FA580079FDB4F80080F0E500210FE0627802EB50
:10FA6800820202EB820202F2EE2292B20131994244
:10FA780020F8022B04F102043FF4E0AC16F8112040
:10FA88001AB1022AEAD00288F0E7CAB2032AFAD8E1
:10FA98007246EBE700230393FFF782B9B2F5FA7FCA
:10FAA800FEF649AD94F8A630002B7EF444AD059BD4
:10FAB8001B78012113EA010084F8A61000F0D8820F
:10FAC80011F0DEF9049B1B6803F00403FEF737BD51
:10FAD8009FED547AF4EEC76AF1EE10FA44BF9FED39
:10FAE800447A77EE666A4EE74F4A50491068B4F98F
:10FAF800A420C76981FB07018911FF17781A00F54F
:10FB0800FF407F3082423EF704ADC91B0A4412B25F
:10FB1800A4F8A420FEF7FDBCC8398A4240DA9AF856
:10FB2800E0109A7841FA06F3DB073FF55BAB5242E7
:10FB38000120099213F0E6FD7B1E099A162B00F2AC
:10FB48002F81DFE813F0B801CE019F01F701E4012E
:10FB580011028A0175015E01470130012D01F7018B
:10FB68001D0111028A0175010701F100DB0026025F
:10FB7800C300AD0006F068FD032240F6B8338BF8E9
:10FB88002020CBF81C30FFF7F3B90126FEF7FCBBA9
:10FB98003A68DBF81C301344CBF81830FFF7A4B9E7
:10FBA8009AF8E0300122B24023EA020309F5FA721A
:10FBB8008AF8E030A260FFF715BB00211748F3F779
:10FBC80069FB00287FF44BAB322384F8AA00A4F821
:10FBD800AC30FFF744BB00BF3C340020206D002050
:10FBE8006766666662220020DB0FC940E4CB1641D7
:10FBF800DB0F49C0E4CB16C1DB0FC93FDB0F49401F
:10FC080092E741B99730083C15A82ABE00000000C9
:10FC18007D580020926D0020D8520020383C0020EA
:10FC2800A4610020DB0FC9BF10570020D34D62101C
:10FC3800506D0020C94B1B78002B3EF47CAC9BF820
:10FC48000330002B7EF477AC94F8A7300133DBB295
:10FC5800032B84F8A7307EF66EACC14B5B7813B9E2
:10FC6800002E7EF468AC11F00BF9FEF75FBC002A99
:10FC78000CBF012002205CE707231A4602EB820230
:10FC8800174489F80030B97878780BF04DFC059B5B
:10FC98001E7806F00106FEF7D7BD08231A46EDE7E1
:10FCA800DAF8E400DFF8BC8290F8361098F80230F1
:10FCB80011446429A8BF642121EAE17180F8361053
:10FCC800002B40F09D8305F0FBFD20E5DAF8E40009
:10FCD800DFF8908290F8371098F802301144FE2926
:10FCE800A8BFFE2121EAE17180F83710002BEAD085
:10FCF80016201BF0B9FCDAF8E400E4E7DAF8E400CF
:10FD0800DFF8608281781144C829A8BFC82121EA98
:10FD1800E171817098F80230002BD4D014201BF0C8
:10FD2800A3FCDAF8E400CEE7DAF8E400DFF834827E
:10FD380041781144C829A8BFC82121EAE17141705E
:10FD480098F80230002BBED013201BF08DFCDAF897
:10FD5800E400B8E7DAF8E400DFF808820178114433
:10FD6800C829A8BFC82121EAE171017098F80230BA
:10FD7800002BA8D012201BF077FCDAF8E400A2E7E9
:10FD8800DFF8E081089898F8023041791144642935
:10FD9800A8BF642121EAE1714171002B40F03C8346
:10FDA800DAF8E4008FE7DAF8E400DFF8B881017ADE
:10FDB80098F802301144C829A8BFC82121EAE17186
:10FDC8000172002B3FF47FAF0B201BF04DFCDAF8DB
:10FDD800E40078E7DAF8E400DFF88881C17998F878
:10FDE80002301144C829A8BFC82121EAE171C171B4
:10FDF800002B3FF468AF0A201BF036FCDAF8E40069
:10FE080061E7DAF8E400DFF85C81817998F802307C
:10FE18001144C829A8BFC82121EAE1718171002BCA
:10FE28003FF451AF09201BF01FFCDAF8E4004AE761
:10FE3800DAF8E400DFF82C81417998F802301144AF
:10FE4800C829A8BFC82121EAE1714171002B40F0FF
:10FE58008E82112F7FF456AF35E7DAF8E400DFF829
:10FE68000481017998F802301144C829A8BFC82133
:10FE780021EAE1710171002B40F0D482102F7FF448
:10FE880057AF20E70899DFF8DC800F791744642F13
:10FE9800A8BF642727EAE7770F711BF0FFFB98F8E4
:10FEA8000230002B3FF47CAF032039461BF0DCFB0B
:10FEB800DAF8E40007E70898DFF8A8800178114429
:10FEC800FA29A8BFFA2121EAE171017098F80230F5
:10FED800002B3FF465AF01201BF0C6FBDAF8E40005
:10FEE800F1E60898DFF87C80817811446429A8BF7E
:10FEF800642121EAE171817098F80230002B3FF407
:10FF08004FAF02201BF0B0FBDAF8E400DBE60898FC
:10FF1800DFF85080C17998F80230114481F3080164
:10FF2800C171002B3FF43CAF05201BF09DFBDAF8B4
:10FF3800E400C8E6089BDFF82C80997998F802005D
:10FF480011446429A8BF642121EAE171997100284C
:10FF580040F015820D2F7FF415AF21E7BD54002026
:10FF68000C3E00204E6F0020DAF8E400DFF86C84C5
:10FF7800C17898F802301144C829A8BFC82121EADD
:10FF8800E171C170002B40F03F820F2F7FF4E6AE85
:10FF980099E60898DFF8448441781144B1F5967FD2
:10FFA800A8BF4FF4967121EAE171417098F80230C8
:10FFB800002B3FF4F5AE15201BF056FBDAF8E400F1
:10FFC80081E60E992AE435F912209978B2F5617F15
:10FFD8004FF4966393FBF1F33ADB40F63301914219
:10FFE800A8BF11460C2FA1F5617191FBF3F100F048
:08FFF800FB80182F7FF48BAB96
:020000040801F1
:10000000C9B2C8290B46A8BFC823DAF8E400C27DEC
:10001000DFB297423FF47FAB9A1ADFF8C883C77507
:1000200048BF0732D71098F802300137FFB23BB90A
:10003000002F3FF470AB384613F068FBFFF76BBB43
:1000400018201BF015FBF3E7F0EE477AFEF731BD01
:10005000B0EE677AFEF717BD0C2F00F0E080182F86
:100060007FF459AB00210B46CFE7B0EE667A6CE423
:10007000C84A0292FFF70EB9C74B1B6813F400334E
:1000800040F0D4801846C5490E5C0F2E00F10C00DC
:1000900031D00133152BF7D1049B1B68FA3A0021AC
:1000A000A4F8A42003F0040384F8A610FEF74BBACA
:1000B000F0EE476A5FE4BA4A049B1F68138823F096
:1000C00004031380012307F480578BF82130FFF7D6
:1000D000B9B904231A46D5E505231A46D2E5062305
:1000E0001A46CFE501231A46CCE502231A46C9E594
:1000F00003231A46C6E5AB4FD7F800E05800BEF11F
:10010000000F07D0C61801EB86069EF801E076784E
:100110007645C1D21844A44EA44B01EB80010020C7
:10012000396030801860B7E7A14BA2491A684FF4D4
:100130007A73B3FBF2F3C3EB431203EB8202049B2B
:100140001B68D200A1F8B42003F00403FEF7FBB94A
:10015000049B99491B680A6003F00403FEF7F3B996
:100160000021BB2A109100F0C680B72A00F0BF80A2
:10017000BE2A00F0BA80BD2A00F0A080792A00F0E3
:10018000E6807A2A00F0DC809E2A00F0D3809D2A47
:1001900000F0C980AE2A00F07081AD2A00F06681BF
:1001A000EF2A00F05D81FD2A00F05481FB2A00F067
:1001B0004B81FE2A00F04281F72A00F09F807B2AC3
:1001C0007EF4BDA94FF4FA6102201AF027F8FEF779
:1001D000B6B97A4B0022012079497A4C0B60227023
:1001E00013F094FA049B1B6803F00403FEF7ABB909
:1001F000CFB2744B09915B78BB423FF48CAADFF815
:10020000E48138461AF0D6F898F8023009991BB103
:10021000C9B20C201BF02CFA0137FFB208E7002707
:100220003946E6E7684B01220220D5E7674B1B7889
:10023000032B00F09B80034625E7654B0222032039
:10024000CAE7049B634A1B684FF4C871118003F02E
:100250000403FEF778B9002E3EF4EAA85E4C94F849
:10026000A130002B3EF416A913F054F9002384F8B2
:10027000A130FEF70FB911F0E7FCF2F7DFFB11F048
:10028000CBFCF5F72DFA012013F040FA94F8A220E8
:10029000FFF783BA94F8A820002A3ED194F8AA3038
:1002A00083F0010384F8AA3073BB0C2013F04EF9DD
:1002B000049B1B6803F00403FEF745B94FF6FE7379
:1002C000464AD0899689014433449381D18111F003
:1002D000BBFCF2F7B3FB11F09FFCF5F701FA01202C
:1002E00013F014FAB4F8A420D6E60223E8E70B468C
:1002F0004FF6FE71E4E70B460221E1E700210420FE
:1003000019F08CFFFEF71BB90B2013F01FF9049BAB
:100310001B6803F00403FEF716B984F8A80084F8FC
:10032000A910FEF710B90021FF201DF0AFF994F8D5
:10033000A2202FE701201DF0A9F994F8A22026E7BA
:10034000274A137A43F001031372FEF7F8B8244AE0
:10035000137A23F001031372FEF7F1B81E4C10F06C
:1003600093FD002384F8A130FEF794B813F0D2F87F
:10037000B4F9A42090E6112009921BF079F9DAF87B
:10038000E400099A69E50D2009921BF071F9099AB8
:10039000E4E500BF446A0020C8310020C407030818
:1003A000746D002014230020682300206C2300209B
:1003B000F4680020006200201C570020326E0020EC
:1003C0009C6C0020906C0020806E0020F254002075
:1003D000CE6E0020FA6D002078230020F03D002032
:1003E000786D00204E6F0020002B3FF437AF264978
:1003F000264A09684FF47A7000FB031313602DE757
:1004000003230393FEF778BD17201BF031F9CBE4EB
:100410000F2009921BF02CF9DAF8E400099AB8E5EC
:100420000E201BF025F9DAF8E40050E410200992C0
:100430001BF01EF9DAF8E400099A23E500210320F5
:1004400019F0ECFEFEF77BB80021022019F0E6FE61
:10045000FEF775B80021012019F0E0FEFEF76FB835
:100460000021084619F0DAFEFEF769B8FF210020E6
:100470001DF00CF994F8A22092E6012100201DF055
:1004800005F994F8A22088E6A461002018570020FE
:1004900030B4034600F12405064C07CC0C3343F876
:1004A0000C0C43F8081C43F8042CAB42F4D130BCCC
:1004B000704700BF3C020308034B33F80C2F028047
:1004C0009B788370704700BF3C020308084B196893
:1004D00061B130B45D68074C642202FB05F2B2FBE7
:1004E000F1F2228030BC002018605860704700BFD5
:1004F0006024002092340020704700BF2DE9F041B5
:10050000BC4CBD4D0E4630220021804620461FF0D7
:1005100088FBBA4A701CD37A927A4FF006013BD01E
:10052000B74FE2B1002B56D0B8F1000F40F0A180D8
:10053000FF2008E0012A0ED908F10108B8F1060FE2
:1005400004F1080444D017F90830A371A3F11E0286
:100550009E42D2B2EED10139C9B2A071ECE7002BB4
:1005600053D0B8F1000F40F0C480FF2008E0012A0A
:100570000ED908F10108B8F1060F04F1080427D0DC
:1005800017F90830A371A3F11E029E42D2B2EED138
:100590000139C9B2A071ECE7002B50D0002A00F05D
:1005A000D180B8F1000F40F00681954FFF2217F976
:1005B0000830A3711E3BDBB2012B08F1010802D801
:1005C0000139C9B2A271B8F1060F04F10804EED1E5
:1005D0002972BDE8F081B8F1000F5BD1FF2008E07F
:1005E000012A0ED908F10108B8F1060F04F1080438
:1005F000EED017F90830A371A3F11E029E42D2B2C9
:10060000EED10139C9B2A071ECE7B8F1000F59D1B0
:10061000FF2008E0012A0ED908F10108B8F1060F01
:1006200004F10804D4D017F90830A371A3F11E0215
:100630009E42D2B2EED10139C9B2A071ECE7704F3F
:10064000002A69D0B8F1000F40F0C480FF2217F9EA
:100650000830A3711E3BDBB2012B08F1010802D860
:100660000139C9B2A271B8F1060F04F10804EED144
:10067000AEE70023FF2003E0062B04F10804A7D017
:10068000FA56A271964203F10103F5D10139C9B2BC
:10069000A071F1E74FF0FF0E09E01F2A02D184F8A4
:1006A00006E0C1B20133062B04F1080490D0FA56DB
:1006B000A271964201F1FF30EFD10139C9B284F83D
:1006C00006E0EFE74FF0FF0E07E001280CD90133F9
:1006D000062B04F108043FF47BAFFA56A271A2F195
:1006E0001E00B242C0B2F0D10139C9B284F806E0AE
:1006F000EDE71346FF2007E01E2A09D00133062B41
:1007000004F108043FF464AFFA56A2719642F3D1A3
:100710000139C9B2A071F1E7B8F1000F39D1FF2258
:1007200017F90830A3711E3BDBB2012B08F1010859
:1007300002D80139C9B2A271B8F1060F04F1080458
:10074000EED145E72E4FB8F1000F12D1FF2217F975
:100750000830A3711E3BDBB2012B08F1010802D85F
:100760000139C9B2A271B8F1060F04F10804EED143
:100770002EE71346FF20FA56A2711E2A03F1010349
:1007800002D10139C9B2A071062B04F10804F2D1DB
:100790001EE71346FF20FA56A2711E3AD2B2012A72
:1007A00003F1010302D80139C9B2A071062B04F18B
:1007B0000804F0D10CE714230027012602201E2292
:1007C000A3711F23A773A675A07784F8262084F849
:1007D0002E30FDE6FF20FA56A2711F2A03F1010315
:1007E00002D10139C9B2A071062B04F10804F2D17B
:1007F000EEE600BFC84E00206024002040460020E6
:100800004C020308624B1B78002B3AD02DE9F041D3
:10081000604B614D9B79EC68E860013B82B0041B42
:10082000032B00F28380DFE803F0310229291AF05C
:10083000EDFE002800F08280584B59491B78B5F82E
:100840004620D1ED037A2A65DB0700F1848002FBA4
:1008500004F007EE900ADFED536A534BB8EEE77AE7
:10086000D5ED137A5A60E7EE267A1A60BDEEE77A84
:10087000C5ED137A85ED127A83ED027A02B0BDE8F8
:10088000F081494A1360536093607047474A484B70
:10089000D279DFF8308133F81220B8F902304548B8
:1008A000B8F9001092B207EE902A40F6E44707FB31
:1008B00002F6C3EB1633B8EE670A4FF47A7606FBFE
:1008C00003F393FBF1F3EB61EFF7B8FED5F81CE00F
:1008D000D5ED057ADFED336AB8F90220324BB8F96D
:1008E00000C0C3F804E00EFB04F007EE100AB8EEF7
:1008F000C77ABCEEC06AE7EE267A8DED016ABDF8D4
:100900000410C5ED057ABDEEE77A07FB01F7C2EBEF
:10091000173706FB07F683ED027A96FBFCF685EDAA
:10092000047AAE611E6002B0BDE8F0811E4B002269
:100930001A605A609A6002B0BDE8F0811E4B1B68D5
:10094000DE067FF579AF154BB5F846201B782A6592
:10095000D9070FD47BE7FDEEE77A184E17EE900A21
:10096000A0F57A7101FB01F386FB0306D817C0EBF3
:1009700026100844B5F94410114B00FB01F083FB2D
:100980000013C017C0EBA31002442A655FE700BF45
:100990000E440020406D002060240020FC6B0020ED
:1009A000104400202FE33E31AC530020AC61002006
:1009B000C861002080240020046900201F85EB51BD
:1009C000D34D6210E03D0020F0B5244B5B79012B44
:1009D00083B00ED0224900230B804B80214B1B7823
:1009E000022B04D1204B48880A8818805A8003B013
:1009F000F0BD1E4A1E4B92781E4D33F81240A4B231
:100A000007EE904A05F15800B8EE670AEFF716FEB8
:100A1000194A1349107896785378FCEEC07A00EBA7
:100A20004010CDED017ABDF8042044F6FB77C3EB0E
:100A3000033300FB027200FB0474B2FBF3F2B4FB5D
:100A4000F3F3B2FBF6F2B3FBF6F392B29BB2A5F866
:100A50005420A5F856300A804B80BFE7406D002037
:100A6000F8430020E8430020EC430020AC61002064
:100A7000C8610020602400201D6E0020F8B5254DBF
:100A800025496879254C264B264E042264270A7096
:100A900001284FF0000184F87C2084F88570A4F8C8
:100AA0007E10A4F8801084F88410C4F88810317087
:100AB0001980598020D0A9791B4A0023012913608D
:100AC00084F88C305360936007D0022904D1174A10
:100AD000A36453609360F8BDF8BD154A2361536069
:100AE0009360D3609FED130A02F110004CF2503175
:100AF000BDE8F840F2F774BB282204F154001FF05F
:100B000090F84CF250319FED0C0A04F15800F2F7C6
:100B100067FBD0E7406D0020F254002060240020E5
:100B2000F84300200E440020AC530020A8240020ED
:100B300070240020CDCCCC3ECDCCCC3D2DE9F04373
:100B40002F4DD5F8903083B01BB195F89430022B1F
:100B500002D003B0BDE8F0834FF020084046294C96
:100B600005F19809012655271AF024FDA0B199F83E
:100B700000300BB9217891B908F101085FFA88F8C3
:100B8000B8F1230F04F1010409F10109E1D0404655
:100B90001AF010FD0028EAD189F80000ECE7D5F83A
:100BA000900050B30DF1080EAA220EF8052D8DF815
:100BB00002108DF800708DF801608DF804306946E0
:100BC00055225340082213F0800F02F1FF324FEA02
:100BD000430318BF83F0310312F0FF02DBB2F2D1FE
:100BE000714502D011F8012FEBE7AA2269468DF872
:100BF00003308DF804200DF0AFFD89F80060BBE7ED
:100C000060240020540203081F4B1878002839D0B4
:100C10001E4A1389FBB11E4A9FED1E6AD2ED026A7D
:100C200007EE903AF8EEE66AF8EE677A07EE103AC9
:100C300077EEE66AB8EEC77A66EE866AC6EE877A1F
:100C4000FDEEE77A17EE900A6428A8BF642020EA38
:100C5000E070C0B2704710B40F4B54781B88117805
:100C600004FB1032091B642300FB01F003FB02F3B9
:100C7000B3FBF0F06428A8BF64205DF8044B20EAC1
:100C8000E070C0B2704700BF0E440020406D0020ED
:100C9000AC5300200000C842F84300202DE9F04F7B
:100CA000794D81B0F0F76CF9D5F8A0400022C5F875
:100CB0009C20002C00F0A580237D052B074617D92A
:100CC000216A23690B44C31A9342B8BF05F1A001FE
:100CD0000ADBD5E0137D052B0AD9136A1269134488
:100CE000FB1A002B80F2CC8051F8042F002AF1D19E
:100CF0004FF0010B0023B9461E46C5F89C309846BC
:100D00009A46274623E07A6A39693B7DA9EB0204BB
:100D1000B4FBF1F40134A4B213FB04F30133013644
:100D20009BB2B6B23C83FB82984506D2BBF1000F62
:100D300001D1012C5FD99846BA46D5F89C300133D1
:100D400005EB8302C5F89C30D2F8A07047B3BB68AE
:100D5000C3B1FC8A002CD6D1396A4846A9EB0101FF
:100D60009847D0B195F8F030002B52D13B7DC7F8B1
:100D70002490013601334FF00102B6B23A83FB8270
:100D80000124D1E73B6A3A69A9EB0304B4FBF2F40E
:100D9000A4B23C8334BBFB8AC6E73C83FB8AC3E72F
:100DA0002B686A683949013316443C4685E8480097
:100DB0004F46C1F800A0BAF1000F27D0DAF8203072
:100DC00095F8F020AAF81640FB1ACAF81C30CAF8A9
:100DD0002090002A35D1DAF80C30484601B0BDE841
:100DE000F04F18473B7D13FB04F3013301369BB2F0
:100DF000B6B2FB8298E73A7D062A04BF9846BA4607
:100E00009BE72B68214A01332B60146001B0BDE8D9
:100E1000F08FF0F7B5F81E4B1E4A1F4C11681A6888
:100E2000A0EB090002EB000E2268C3F800E090423C
:100E3000A1EB5111014438BF1046164A20601160E1
:100E400094E7F0F79DF8DAF80C3004469847F0F78D
:100E500097F8DAF82C20DAF82830DAF83010001B8E
:100E60009042A3EB53130344014438BF1046CAF821
:100E70002830CAF83010CAF82C0001B0BDE8F08F55
:100E80004FF0000B36E700BF602400201057002011
:100E900094340020983400209C340020F0B4342393
:100EA000184F194A03FB00F3D2F8F460FC58FD1800
:100EB000002E6B684B600C600DDDD2F8A0309D42B7
:100EC0001DD0A032002303E052F8044FA54216D0F3
:100ED0000133B342F8D10022342303FB00700A72BD
:100EE0000369CB60037D4B72836AC56A046BC26978
:100EF0000A615B094D618C61CB61F0BC70470122D6
:100F0000EAE700BFC4010020602400202DE9F04181
:100F1000244ED6F8F450122D27DC002D3DDDD6F8F6
:100F2000A030984221D005F1804106F1A007013997
:100F300007EB81013B4603E053F8042F904214D0A5
:100F40008B42F9D1D6F8A0409CB1237D017D8B4224
:100F50000ED3154A002405E052F8043F4BB11B7D27
:100F60008B4206D30134A542F6DA0020BDE8F081B9
:100F700000248046601C80002A1B011F06EB8404AD
:100F800039443844920001351EF031FEC4F8A08087
:100F9000C6F8F4500120BDE8F081E6D106F1A007C3
:100FA000D0E700BF6024002000250020142830D0A6
:100FB000122807D8184B342202FB003019B1C3683D
:100FC0000BB1A3E7704770B5144DD5F8F440002C71
:100FD0000FDDD5F8A03098420CD005F1A0063346BD
:100FE000002203E053F8041F884206D00132A242D7
:100FF000F8D170BD002205F1A0069000011DA21AD3
:10100000920031443044013C1EF0F1FDC5F8F4403B
:1010100070BD034B1868D1E7C40100206024002094
:101020001057002010B54FF4804082B012F0D0F974
:1010300000B30022032390F90200009301924FF4C1
:10104000E1334FF4804111F013FD0C4BC3F89000D5
:1010500070B1012402221220214683F8984083F8BF
:10106000994083F89A4083F89420FFF79FFF204629
:1010700002B010BD014BD3F89000E9E760240020D6
:10108000F0B50D4685B006460068F0F741F995E8E1
:101090001800E41A0023039324238DF808304D230D
:1010A0008DF80930B5F90A30FF2C2246A8BFFF227F
:1010B00001333DD02B7B002B0CBF3E233C238DF80E
:1010C0000A30FE2C2B898DF80B208DF80C3031DD89
:1010D00023128DF80D408DF80E3007273A4602A9ED
:1010E0003068F0F71BF902ABDA190DF10B010023A0
:1010F0008A4221D1002C8DF807300CDD2246296868
:101100003068F0F70BF92B689DF807201919994200
:1011100016D18DF8072001220DF107013068F0F794
:10112000FDF83068F0F7EEF804F1090005B0F0BD05
:101130002123C4E70527D1E711F8010B4340D7E786
:1011400013F8010B4240E2E72DE9F347012012F0CA
:101150003FF9174EDFF85CA00024CC2708B1022C21
:1011600002D902B0BDE8F08707FB04F856F8085032
:1011700015B10134E4B2F1E7C37890F902005AF8EE
:10118000233001950322009201212A4611F070FCC0
:10119000814648B104FB0760CC2229461EF041FD80
:1011A000013446F80890E4B213F00AFAD6E700BF1B
:1011B000284F0020A02003082DE9F04F2DED088BCB
:1011C000BE4CBF4BC4F80C3887B00023C4F81038AD
:1011D000F2F76CF9F0F79AFCF2F724F919F002F83B
:1011E000F1F7F6FB08B9F3F763FDF4F779FA052296
:1011F000B449B5481EF060FD08B1F3F759FD94F805
:101200001438B24D43F0010384F81438B04B9A7887
:10121000B04B1A70B04B1B682B600DF0EDF801213C
:101220000220F1F7DFF8F1F7D3F92B681F070BD590
:10123000AA4B1A7A0A2A07D80123934040F20342A4
:10124000134201D00CF06AFF6420A54EEFF768FD51
:10125000F3F71EFEA34ADFF8B8E20023B146995D1A
:1012600003F10F0003F11307304437440EEB010A7A
:1012700010F8018FB8F1000F05D09AF80CC0C445E2
:1012800008BF82F858C090F80480B8F1000F05D06C
:101290001EF801C0C44508BF82F859C0B842E7D162
:1012A000B2F8580040B104EB810109EB030050652E
:1012B000C1F8182802F517722033602BCFD12868A7
:1012C00042F2010318420CBF4FF0FF310121C0F37D
:1012D0008010FFF713F92B68DE0740F1CA8315F081
:1012E00045F9B4F83068804B94F82C081E80002E25
:1012F00040F0C583F0F7E4FB7C4A7D49106094F828
:101300002D28003218BF01220A7058B194F82E38E7
:10131000C671002B4FF02402827114BF11210121EC
:10132000F0F764FE0020F1F733F8724B724E03F1D0
:10133000300C4FF0000853F8057C77B313F9092CF3
:10134000A11806EB021091F832E891F8359891F85F
:1013500038A8991E11F801BFF34591F802B008BFF3
:1013600080F804E0CB4591F804B008BF80F8059000
:10137000D34508BF80F806A08B42EBD1110172184B
:10138000107950B1507940B1907930B17750597996
:10139000D1719979117282F80C8010339C45CAD1B1
:1013A0001F20F0F78DFB30B12C2282710022C27118
:1013B0002021F0F71BFE14F0C5FFDFF85891DFF88D
:1013C000588159F8063C0293002B3AD019F90A6C5F
:1013D000142303FB06871A46002138461EF021FC21
:1013E000A219A9F1030A92F83B3892F83DB8039389
:1013F0001AF8011F039B994203D11846F0F760FBCE
:10140000B8609AF80310594503D15846F0F758FBD5
:10141000F860D145ECD1142303FB06F108EB01027F
:10142000906870B1D06860B12644A9F10A0048F80C
:10143000010096F83F18029B117496F8411853600A
:1014400051742E4B09F110094B45BAD12C4F13F0B2
:10145000D5FD97F80890B9F1000F2DD04846F0F768
:101460002FFB284E8046706018B12F238371002314
:10147000C3713F78002F40F00683484613F0AAFE60
:101480000746C8B1B8F1000F04D0027A02214046E5
:10149000EFF790FFDFF884801B4A0023019300934D
:1014A00039468023404618F0FBFCB2688023336144
:1014B0001360012308F8083C144931E0602400203F
:1014C0008D13000892280308956C00200469002001
:1014D000906C0020E8430020806F0020446A0020C8
:1014E0005802030858250020C4640020C864002066
:1014F000C6640020C10203088464002012030308AC
:10150000546C0020406C002000A24A04406D002072
:1015100040460020F2020308D0610020486C002001
:10152000D64A4B795E1E7342734113708B795F1EEE
:101530007B427B4113712B68190400F1D48213F0B4
:10154000007305D0CE4BDB7AA3F108004342434140
:10155000937013F049FBD4F844383BB9D4F84828C9
:1015600022B9D4F84C28002A00F09F801BB208EE64
:10157000103ADFEDC4AADFEDC48AC44AB8EEC88AC7
:10158000002128EE2A8A117038EE280AFDEEC07A72
:1015900017EE903A2033402B00F2A782F1F7A6FD18
:1015A000F0EE409AFDEEC87A17EE903A2033402BC9
:1015B00000F29E82B0EE480AF1F798FDB0EE40AA24
:1015C000B4F9483809EE103AB8EEC99A29EE2A9AC9
:1015D00039EE280AFDEEC07A17EE903A2033402B00
:1015E00000F28982F1F782FDB0EE40BAFDEEC97AD1
:1015F00017EE903A2033402B00F28082B0EE490A79
:10160000F1F774FDB0EE409AB4F94C3808EE103A98
:10161000B8EEC88A28EE2A8A38EE280AFDEEC07A8B
:1016200017EE903A2033402B00F26B82F1F75EFD0B
:10163000F0EE408AFDEEC87A17EE903A2033402B48
:1016400000F26282B0EE480AF1F750FD69EE806A5E
:1016500068EE8A7AF0EE665AE7EE895A8C4B28EEED
:10166000A96A20EE0A7AC3ED035AF0EE465AE7EE75
:10167000495AE6EE897AA6EE497A68EE8B8A2BEE15
:10168000400A2AEE4BAA69EE8B9AC3ED008A83EDDD
:10169000010A83ED029AC3ED045A83ED05AA83ED96
:1016A000067AC3ED077AC3ED089A07F085FA064675
:1016B00018B1784B186807F08FFF07F06FFD46B937
:1016C00002210120F4F7CCF9734A138843F0010397
:1016D000138094F81438714F012143F00203084637
:1016E00084F81438F0F77EFE00210846F0F77AFE01
:1016F00000210220F0F776FE0A260120EFF74CFECB
:101700000020EFF749FE1920EFF70AFB3B68D903E9
:1017100002D40120F0F73CFE1920EFF701FB002076
:10172000F0F736FE013EE8D131463046F0F75AFE7A
:1017300031460120F0F756FEF3F7F2F9584B594EB7
:10174000186803F049FF584B188807F0CDFE574B37
:1017500032781A7004F0E6FD2A68554BD2049F8A4D
:1017600048BF544A9B7848BF9788042B04D14FF454
:101770008050F1F725F9002704F0F6FB4E4B384670
:10178000197813F055FF94F8143843F0040384F8E3
:10179000143802F07FFE02F037FE484B1B680BB195
:1017A00012F068FF02F03EFA04F0C8FE15F0EAFFFE
:1017B0004FF4197200214248424CDFF828811EF094
:1017C00030FAFFF7C1FC404B00271F809F7010F0DC
:1017D00053FA3E4BC8F800704FF0FF3A04F5056924
:1017E000C3F800A048463A4BC4F8503818F0EAFE57
:1017F000384A84F85E78012384F85C38537884F89A
:101800005DA80D3384F8583813781E3384F859389E
:10181000D8F80030042B474605D05A1CC8F80020E1
:101820002D4A42F823902B68980340F18E8094F85B
:101830006C382A4DDFF8B090C5F80090013B84F871
:101840006438C82094F86D3884F86538EFF768FA82
:101850002868DFF898800AF00FFB88F80000C8209D
:10186000EFF75EFA2B68C4F8743809F110051C4BC9
:10187000C4F87038284618F03BFE39E0C0610020FB
:10188000446A002035FA8E3CDB0FC93FF40000208B
:10189000343B0020F4680020746D0020C831002023
:1018A0009C6C00202C3E0020F03D0020402E0020AB
:1018B000B06500201C34002096430020A82F002093
:1018C000284F002060240020506D002034070020A5
:1018D00008030308706C0020B46B00208C6C00209F
:1018E00034030308B06B0020C02C0020916D002051
:1018F000012384F87C38002384F87E38FF2384F8A1
:101900007D38082384F87838152384F87938804B9B
:101910001D6098F800303BB13B68042B04D05A1C82
:101920003A607C4A42F823507B4D10220021284621
:101930001EF077F9002019F078FAEFF721FB07463F
:1019400019F08EFA754B3B44EB60754F754D0023D3
:101950003B702B68D90308D519F0CCF901233B70F3
:10196000714B93F8F1000AF085F92B685A0501D5FF
:101970000EF01CFB08F064F83378052B03D16B4B99
:101980004FF4C8721A806A4B6A4E1A684FF47A7321
:10199000B3FBF2F3C3EB431203EB8203664ADB00B3
:1019A000A2F8B4304FF4006011F012FD98B1634B0F
:1019B00090F9020093F83230002B14BF1823002353
:1019C00001930323009300224FF496534FF40061D8
:1019D00011F04EF83060336813B1594B594A1A6010
:1019E0004FF4005011F0F4FC574E98B1534B90F95E
:1019F000020093F83230002B14BF08230023019318
:101A00000323009300224FF416534FF4005111F0BA
:101A10002FF83060336813B1494B4C4A1A604C4A76
:101A2000137843F008031370FFF728F82B689B0323
:101A300006D5394B07225A721A7A42F001021A72FD
:101A4000444B1B682B6018F0EFF9434A138843F0AE
:101A50008003138011F0A2FEFFF7E4FA94F8143823
:101A600063F07F0384F8143807B0BDEC088BBDE841
:101A7000F08F98047FF535AC14F022FD31E4314647
:101A800018F0A4FB51E4012F7FF416AD404613F08B
:101A90004FF87068F0F76CFC4FF4E0733361377007
:101AA0003623002604A88DF810308DF811708DF8BB
:101AB00012608DF8137016F017FF372305A88DF804
:101AC00014308DF815708DF816608DF8177016F0BB
:101AD0000BFF224AD36943F03003D361204B1E85AC
:101AE000A3F82864E8E4012332E5DFED1E9A59E506
:101AF0009FED1CAA64E59FED1BBA77E59FED199A4F
:101B000082E5DFED188A95E59FED160A9EE500BF98
:101B1000886D0020B46B0020786D0020404B4C0095
:101B2000C254002004690020C0530020FA6D002038
:101B3000F46800202052002000620020BB32002008
:101B4000643F0020A8000020046C0020C400002096
:101B5000403C0020806F0020746D00200010024087
:101B6000001000400000000008B50E4B1978012954
:101B700013D00DD3022902D10020EFF70DFCEFF7AF
:101B8000FFF9094B00F5F42000F59070186008BDCE
:101B900000210846F0F726FCF1E70020F0F722FCD0
:101BA000EDE700BFFC6D0020006E00202DE9F04F36
:101BB00083B0484C484F0190019803685B6998478F
:101BC000002840F08380DFF818914448D9F80430A9
:101BD000DFF810E1C3F308034FF00A0A4FF0100CCE
:101BE0004FF47A75002B3BD1EFF31183002B37D1E3
:101BF0000168A26800BF03689942F9D1DEF800606D
